:020000040000FA
:040000006FD00400B9
:101000006F00907E00000000000000009020002093
:10101000AA220020A9BDF9F56C23002000000000E1
:10102000000000006C230020902000200000000041
:101030000000000090200020000000009020002010
:101040000000000090200020902000209020002030
:101050009020002090200020582F00209424002071
:101060000000000090200020902000201E2400207E
:1010700090200020D22300209020002090200020EB
:101080009020002090200020902000209020002020
:101090009020002001A04111B7170040985F3AC688
:1010A000945F3247E39CE6FE3245410182800111A4
:1010B00013078008F337078093F787083EC20100C3
:1010C0000100B7170040930570052380B70413068D
:1010D00080FA2380C7040100010083C6B70493F699
:1010E000F60DA385D704238007049246F3A6068055
:1010F0000100010093760502D5CEF336078093F602
:10110000860836C4010001002380B7042380C70489
:1011100001000100B70614007D89558D88C70100C4
:1011200001000100010023800704A246F3A6068007
:101130000100010073370780137787083AC6010062
:1011400001002380B7042380C704010001000100CF
:1011500001003727004093061005A303D7802380A2
:101160000704B247F3A70780010001009307800836
:10117000F3B7078093F787083ECE01000100B71749
:101180000040130770052380E704130780FA2380CB
:10119000E7040100010003C7B70413670708A3852C
:1011A000E70423800704F247F3A70780010001004A
:1011B0000561828093760504BDC6F336078093F6F9
:1011C000860836C8010001002380B7042380C704C5
:1011D00001000100B7061400938606047D89558D31
:1011E00088C7010001000100010023800704C246F6
:1011F000F3A6068001000100733707801377870884
:101200003ACA010001002380B7042380C70401000B
:1012100001003727004093062005A303D7802380D1
:101220000704D24781B773370780137787083ACC12
:10123000010001002380B7042380C70401000100DE
:1012400098471367070C98C723800704E24719BF24
:101250000111814601468145114506CE97000000E7
:10126000E780605893078008F3B7078093F78708F3
:101270003EC601000100B717004013077005238028
:10128000E704130780FA2380E7040100010003C785
:101290006704136717002383E70423800704B2471A
:1012A000F3A7078001000100F2400561828041112F
:1012B000814601468145114597000000E780A05214
:1012C00013078008F337078093F787083EC40100AF
:1012D0000100B7170040130670052380C70493066A
:1012E00080FA2380D70401000100FD552396B70240
:1012F00023800704A245F3A5058001000100733790
:101300000780137787083AC6010001002380C704CD
:101310002380D7040100010003C767041367170087
:101320002383E70423800704B247F3A70780010063
:10133000010001A0B1473305F50201007D1575FDDF
:101340008280411122C426C206C6AA8401446317C2
:101350009400B24022449244410182800504130566
:10136000803E420497000000E78000FD4180C5B741
:101370009305000273A04580824573901534924016
:101380002242B2424243D2436244F2440255925551
:101390002256B2564257D2576258F25806499649D9
:1013A000264AB64A464BD64B664CF64C065D965DD1
:1013B000265EB65E465FD65F09617300203041113C
:1013C000B7170040985F3AC6945F3247E39CE6FE49
:1013D000324541018280B71700401307000323887C
:1013E000E702854717170000232AF75473002030BF
:1013F000411122C42D6426C24AC006C637190040D6
:101400001304A4AAB704002023208900976000E0F9
:10141000E780003A9C408297976000E0E78040397F
:10142000E5B737370040834747009146BD8B639E41
:10143000D702B73600401306F00F973500009385AA
:10144000E52C9737000083D7673C03C7A6001377C6
:10145000F70F1DE3B7E70400BC4F09468945171590
:1014600000000345A5F7829731A099466394D70001
:10147000834757007300203003C786001377F70FA8
:10148000E365F6FC13851700AE9717380000231F9D
:10149000A8362380E70075B7B787004003C7670009
:1014A000098B6309071003C77700930600031377BE
:1014B0000703630DD708174800000348F884174650
:1014C0000000130666810547B30606012380E60087
:1014D00083C577001747000013070782429793F5EB
:1014E000F50F2300B70003C58700973500009385EB
:1014F000A57FC2951375F50F2380A500034707004C
:1015000089451377F703630CB70C63E7E50A6306B5
:10151000071A8545630CB7129737000083C7D77E3B
:101520003307F600034707001377F70F19CB85073A
:1015300093F7F70F3D476363F71A17370000A305CA
:10154000F77CB787004009472383E700B78700404F
:1015500083C77700E207E18763DE0704973700005F
:1015600083C7977A17370000130707773E9785469A
:101570002300D70017370000130707783E9793061C
:1015800000032300D700173700001307E7753E97C5
:10159000A14685072300D70093F7F70F3D47636403
:1015A000F71417370000A301F776B7870040094703
:1015B0002383E70073002030930610026300D70EE8
:1015C000930620026305D70693060002E316D7F4BC
:1015D00003C727021377C70F13672700D5A803C7D0
:1015E00067001377070465CB03C7A702173800000D
:1015F000130808501735000013054547134707081F
:101600002385E70203C7A7021377370F1367870005
:101610002385E702814713070004B305F5008C41D9
:10162000B306F80091078CC2E399E7FEF5B503C74E
:10163000A702134707042385E70203C7A70213770E
:10164000C70F136727002385E702F9B503C76700B3
:101650001377070449C303C767021738000013084C
:10166000E83C17350000130525341347070823838A
:10167000E70203C767021377370F136787002383D7
:10168000E702814713070004B305F5008C41B30658
:10169000F80091078CC2E399E7FEBDBD03C767025E
:1016A000134707042383E70203C767021377C70FB3
:1016B000136727002383E70285B503C76700137705
:1016C000070411CB03C727021377370F136787006F
:1016D0002381E70291B5238006003DBD97370000C6
:1016E000A3840762B9BD97370000A38F076075BD5B
:1016F0002303048015472303E48001002302A48010
:10170000828083076480E3CE07FE23030480828007
:1017100083076480E3CE07FE03454480828083070D
:101720006480E3CE07FE2302A4808280411126C498
:101730004AC24EC006C61377F50BAD47AA892E895B
:101740009544630CF700194597000000E78080FA84
:1017500097000000E78020FB8D444E859700000035
:10176000E78040F9FD59FD1463983401B240A2446A
:101770001249824941018280135509011375F50F01
:1017800097000000E780E0F92209F1BF011126CCA3
:1017900006CEB704080097000000E780C0F61545A4
:1017A00097000000E78000F597000000E78080F6D2
:1017B00097000000E78000F62AC697000000E78047
:1017C00080F432459377150089EB13651500137586
:1017D000F50FF240E24405618280FD14E9F0014515
:1017E000CDBF397126DC4ADA4ED852D656D45AD2F9
:1017F0005ED006DE62CE66CCB7E700E07D5783AAF6
:10180000070022C603AA470023A0E71823A2E7186F
:10181000B7170040130770052380E704130780FA09
:101820002380E70483C74704930B75FFB684E20760
:1018300093FBFB0F8546AA892E8B32893724004003
:10184000E187015763FA76016308D50089461307DB
:1018500000026313D5000157D98F93F7F70FB71C18
:1018600000402382FC0411472303E4801305F00F9A
:1018700097000000E78000E8094C97000000E7802F
:1018800080E863657C15B7050700DA9537870700A0
:10189000795563FEE504B3879500636AF704370B57
:1018A0000800A94733EB65016395F90881E8814495
:1018B00097000000E78020E5268515A8DA85094510
:1018C00097000000E780C0E605090345F9FFFD1415
:1018D000050B97000000E780C0E481C49377FB0FFD
:1018E000E5F797000000E780A0EA69F17D55B7179A
:1018F0000040130770052380E704130780FA238054
:10190000E70403C74704418B2382E704F250B7E79B
:1019100000E023A0571123A24711E2543244525948
:10192000C259325AA25A125B825B724CE24C21615C
:101930008280A547639BF90685691309F00FB306FA
:101940009900B3742B01B6941349F9FFB37499004D
:10195000856B33796901416B9387F9FFB3F72701F1
:1019600099E363FC340193D94900C147E3E637FFAB
:101970003DBF0569C1697D19D9B71305800D63881D
:101980006901130500026384790113051008CA85F3
:1019900097000000E780C0D997000000E78040DF93
:1019A00031D54E99B38434416DBFDA852D4597000A
:1019B0000000E780E0D7CA94E30B99EE0509970091
:1019C0000000E78020D5A30FA9FEFDB79387F9FF9C
:1019D00093F7F70F636DFC0C83C71C0413073008E3
:1019E0006315F706370708006361EB06B3079B0032
:1019F000B706100063FBD704334BEB0089476399AC
:101A0000F9068980D549E38404EADA850945970017
:101A10000000E780E0D111090327C9FF9147232087
:101A2000E48003076480E34E07FE23033481FD173F
:101A3000EDFBFD14110B81C49377FB0FE9FF9700B9
:101A40000000E780E0D461F155B5B717004003C747
:101A50005704B70708001377070219E3B787070091
:101A60007955E376FBE833079B00E3F9E7F841B5E6
:101A70008547E380F9F0DA852D4597000000E7807F
:101A800020CB9389F4FFE38404E297000000E78011
:101A900060C893F7390091EB83260480032709007F
:101AA00093074900E396E6E03E89CE84D9BFB54767
:101AB0006399F9001305900B97000000E78080C33D
:101AC000FDB3B1471305B00AE388F9FE9947639760
:101AD000F904B7050800B365BB002D459700000069
:101AE000E78000C581448D4BA14997000000E78045
:101AF00060C263967401832704802320F900850463
:101B0000E39534FF8327048013172B0163550700E7
:101B10002312F90069BB2322F90051BB9D47639F43
:101B2000F90281451305B00497000000E78040C02A
:101B3000BD442320090023220900FD59970000001D
:101B4000E78040BD93F77400CA9703C70700FD14F0
:101B5000398D2380A700E39334FF91BBA14763979E
:101B6000F90697000000E780A0C28144630D0B00D6
:101B70008D479304C0036308FB00930400056304CE
:101B80008B01930440041375C507E30295D21945F0
:101B900097000000E78000B697000000E780A0B63D
:101BA000054597000000E780E0B426859700000017
:101BB000E78020B7094597000000E78080B69700CE
:101BC0000000E780E0BCE31405CE0DB39147639FAE
:101BD000F9001305600697000000E780A0B19700A8
:101BE0000000E78040B213059009F9B5E38109CC04
:101BF000F1547DB9BD660147173600001306462E25
:101C0000938606A685458347060093F7F70F91C391
:101C100082800507E3F9E6FE973700002382B72CA0
:101C2000DDB77D166206618693178601E18763D46E
:101C3000070001458280931726003307F500AE9711
:101C400018439C4363E7E7007D16E37FF7FC7D556F
:101C5000828005458280FD15E205E18513978501A7
:101C6000618793F7F50F63480700FD15139725006B
:101C70002A97584365D713851700620561858280CE
:101C80003308B5021C4283A80600B335B502C297DB
:101C900033B50701AE98469585486367B5006394F0
:101CA000A50063E3070181480C43C6950CC388C2B5
:101CB0001CC2828081471397870161876343B70005
:101CC0008280139727002A97232007008507E5B70E
:101CD0008147014793968701E18663C5B6001335B6
:101CE0001700828093962700AA9694428507558F05
:101CF000D5B793D755408A07AA979C430545331516
:101D0000B5007D8D828017F3FFDFE702833D2A84D3
:101D100097000000E78060F405C5931725003E9406
:101D20000327C4FF814711EB7D1516053E9542053B
:101D3000418517F3FFDF6700033D05838507E5B79E
:101D40000145C5BF81471397870161876343C7007A
:101D5000828013972700B386E50094422A9785076F
:101D600014C3D5B77D1662066186014793178601B5
:101D7000E18763D50700133517008280931726008B
:101D8000B306F500AE9794429C437D16B58F5D8FE8
:101D9000F1BF8A05AA9501476363B500828083A6D7
:101DA000C5FFF11593D71600D98F9CC11397F60183
:101DB000E5B72A830148014701456343D700828084
:101DC000B387050183A80700B30706019C43C697A4
:101DD000AA976384F80033B517010507B308030118
:101DE000620723A0F80061871108C1BF2A83014759
:101DF0008147014563C3D70082803388E50083288B
:101E00000800330EE600032E0E003388A840330886
:101E1000C8416384080133B508018507B308E300AE
:101E2000E20723A00801E1871107E9B717F3FFDFF5
:101E3000E702232B0111B286B2842E86AA850A8579
:101E400097000000E780C0FA2A84A6850A859700DB
:101E50000000E78020E833348000060413351500C5
:101E6000018D056117F3FFDF6700E32917F3FFDF3B
:101E7000E702A3244111AA89AE8A328BB68402C23A
:101E800002C402C60144131C8401135C8C416349E3
:101E90009C02939B1400FD1B0549138CF4FFF15C1D
:101EA00033048901620461846340740792478E049D
:101EB000CE9423AEF4FE410117F3FFDF67006323E6
:101EC00013192400B30B2B01014A93172A00D6974C
:101ED00083A50B0088437800340050009700000071
:101EE000E78040DA050A93178A01E187F11BE35E78
:101EF000FCFC92474E9905042320F900A2473EC2FC
:101F0000B24702C63EC441B7131A8901135A8A4127
:101F1000131D240093178A01E18763CF970092472E
:101F20000A044E941CC0A24705091379F90F3EC25A
:101F3000B24702C63EC4ADB7B3079A0313152A00D1
:101F400056950841780034005000050AEA97DA9760
:101F50008C4397000000E780E0D26DBF197106C284
:101F600012C416C61AC81ECA22CC26CE2AD02ED219
:101F700032D436D63AD83EDA42DC46DECAC0CEC2C9
:101F8000D2C4D6C6DAC8DECAE2CCE6CEEAD0EED2F9
:101F9000F2D4F6D6FAD8FEDA971500009385859923
:101FA0008841E700050092402242B2424243D243B8
:101FB0006244F244025592552256B2564257D257C5
:101FC0006258F25806499649264AB64A464BD64BBD
:101FD000664CF64C065D965D265EB65E465FD65F45
:101FE0000961730020300000972100209381810156
:101FF000175100201301018117F5FFFF1305C500DC
:102000009705002093850500171600201306C6FDCE
:1020100063FAC5008322050023A055001105910530
:10202000E3EAC5FE17050200130545F997150020E0
:102030009385C5FB171600201306C66563FAC50015
:102040008322050023A0550011059105E3EAC5FE92
:102050001715002013050564974500209385053466
:102060006377B500232005001105E36DB5FEFD4241
:10207000739002BC8D4273904280B722000093821D
:10208000828873900230970200209382A2F793E235
:10209000320073905230975200009382428B7390BB
:1020A00012346FB0F47573002030397101436EC67D
:1020B00019A0397141536AC866CA62CC5ECE19A0B4
:1020C000397101535AD056D252D44ED64AD826DA54
:1020D00022DC06DE33016140828241114AC026C201
:1020E00022C406C68282B24D4101024D924C224C5E
:1020F000B24B4101024B924A224AB2494101024984
:1021000092442244B240410182803D432A87637356
:10211000C3029377F700BDEFADE5937606FF3D8AE6
:10212000BA960CC34CC30CC74CC74107E36BD7FE30
:1021300011E28280B306C3408A0697020000969699
:102140006780A6002307B700A306B7002306B700E1
:10215000A305B7002305B700A304B7002304B70005
:10216000A303B7002303B700A302B7002302B700FD
:10217000A301B7002301B700A300B7002300B700F5
:10218000828093F5F50F93968500D58D9396050182
:10219000D58D61B7939627009702000096968682A8
:1021A000E78086FA9680C1171D8F3E96E374C3F8C8
:1021B000A5B73367B500FD530D8B79E7B7877F7FF0
:1021C0009387F7F710419441B372F6003363F6003A
:1021D000BE92B3E262006397720C6318D606504158
:1021E000D441B372F6003363F600BE92B3E26200EC
:1021F0006398720A631BD60410459445B372F600C7
:102200003363F600BE92B3E262006391720A631E0A
:10221000D6025045D445B372F6003363F600BE9241
:10222000B3E26200639A72086311D60210499449BE
:10223000B372F6003363F600BE92B3E262006393BA
:1022400072085105D105E30FD6F6131706019397CF
:102250000601631CF7001357060193D706013305E7
:10226000F7409375F50F91E982804183C18333056F
:10227000F7409375F50F91E182801377F70F93F78D
:10228000F70F3305F74082800346050083C605003B
:10229000050585056313D60065FA3305D6408280AF
:1022A00011059105E312D6FE014582802105A105A5
:1022B000E31CD6FC014582803105B105E316D6FC4E
:1022C000014582804105C105E310D6FC01458280AD
:1022D000B717004003C777051377E70FA38BE70411
:1022E000130700F8A38DE7043D47238CE704130789
:1022F0005003A38CE70403C7A7051377D70F238DDB
:10230000E7048280B717004003C7E7020D89411137
:102310001377C70F498F93068008F3B6068093F6AC
:10232000860836C601000100930670052380D70495
:10233000930680FA2380D704010001002387E70277
:1023400023800704B247F3A7078001000100410181
:10235000828041112A83014E930E407E130F001993
:10236000930F400663E56E129308001913034006AD
:10237000B3781503854E0D4FA14F337365020D8958
:102380001335150063EFBE121308F6FF79467298F5
:102390004208135808013307C70213D61700BE07B7
:1023A00032976146B3F6C60213068070B386C60242
:1023B0003697A166F58F42075D8FB716004083C739
:1023C000F60293F70708A303F1000346710083C7E1
:1023D000F60293F70708E394C7FE83477100B71628
:1023E000004093F7F70F6388071293078008F3B74D
:1023F000078093F787083EC401000100B71700402B
:10240000930670052380D704930680FA2380D704AF
:102410000100010023AA070383C6170393E60608F9
:10242000A388D70223800704A247F3A707800100EF
:1024300001001166B71700407D16D45BC85F938515
:102440004703A98EF18EF5FA93068008F3B606804D
:1024500093F6860836C601000100930670052380B6
:10246000D704930680FA2380D7040100010098C1A5
:1024700003C7170313670704A388E7022380070431
:10248000B247F3A7078001000100410182807D135C
:102490003368E3039308E016630E08003368F30320
:1024A0009308D016630808009378330093B8180097
:1024B0009388D81633081E01131E0801135E0E01FF
:1024C00055B56393E5030548638608000148630337
:1024D00003002A8871087298FD15131E0801C205B1
:1024E000135E0E01C18179BD13F8150063F4BF00BE
:1024F0007908D5B713381800E5BF83C7F60293F7FC
:102500000708A303F1000346710083C7F60293F79F
:102510000708E394C7FE8347710093F7F70FF1DFD5
:10252000E9B531714AD966CB06DF22DD26DB4ED70D
:1025300052D556D35AD15ECF62CD6AC96EC7AA8C26
:1025400002D897100000E78020B12A8993078008FD
:10255000F3B7078093F787083EDA01000100B71749
:102560000040130770052380E704130780FA2380D7
:10257000E7040100010003C7F7021377770FA38771
:10258000E70203C7F70213678700A387E7022380E8
:102590000704D257F3A70780010001000545970003
:1025A0000000E78060D6130780C13347E902116A53
:1025B00093070AE893065002BD69930BA004814A71
:1025C000014B13048008930470057D1AB347F90288
:1025D0003307D7023EC0FD873ECC938709A69309F7
:1025E000803E3347F7023AC27D873AC43347390306
:1025F0008549B399990193D93940B306D702B30BF2
:102600007703B3C6F602B3CBFB0236C6FD8636C8E7
:1026100093D6FB4136CEB7460F0093860624334946
:10262000D9028566938606FAB3969601B389E902C4
:10263000130760553309D90293060010B389E902E4
:102640003349D902B3C9F9029316390036CA37198A
:102650000040FD8636D0930D090493D7F9413ED250
:10266000F336048093F6860836DC010001009307F8
:1026700070052380FD00930680FA2380DD000100B1
:1026800001008346390593F6860FA309D9048346D2
:10269000390593E61600A309D90423800D00E256FC
:1026A000F3A6068001000100130C80FA116DF336C9
:1026B000048093F6860836DE01000100930770055A
:1026C0002380FD0023808D01010001008346390530
:1026D000216693E60602A309D90483560905B3E6E9
:1026E000A6012318D90483560905D18E2318D904CD
:1026F00023800D00F256F3A60680010001008346F8
:10270000390593F606026381061A03463905218AC4
:102710006DDE081897100000E7800098733604807B
:1027200013768608B2C20100010023809D00238039
:102730008D0101000100B717004003C6370513766D
:10274000F60DA389C70403C6370513660602A389DD
:10275000C704835609052166B3E6A6012318D904E8
:1027600083560905D18E2318D90423800D0096467F
:10277000F3A60680010001008346390593F60602A0
:10278000638B061483463905A18AEDFE970000206D
:10279000E7806090AA8636D497000020E780A08F5B
:1027A000A256E30AD5FE835609054255B3E6A601B3
:1027B0002318D90497100000E780C08F834639059D
:1027C000A18AEDDE03560905834629058247337643
:1027D000CA00B306DA0293D5F641B296B388F64042
:1027E000E24733B8C6002E983308F840A247B3B684
:1027F00016013308D84063C70701631DF8009247EC
:1028000063FA1701C247634FF80E63950701B24799
:1028100063EAF80E894663E9660FF24693151800DD
:1028200013D3F8015E8613951800B365B30042D642
:1028300046D497C00100E78040DF3258050B137B78
:10284000FB0F63470001631A0838A25863870838F2
:1028500013081500B336A800B69513D6F5013298C3
:10286000B336C800AE9613581800FE06B3E606014C
:102870007336048013768608B2C6010001002380F7
:102880009D0023808D01010001000356C902B2960C
:10289000C206C1822316D90223800D00B646F3A6D4
:1028A00006800100010021B5F336048093F6860806
:1028B000B6C00100010023809D0023808D0101002E
:1028C00001008346390593E60602A309D904238053
:1028D0000D0086460DB5F336048093F68608B6C41F
:1028E0000100010023809D0023808D010100010073
:1028F0008346390593E60602A309D90423800D0017
:10290000A646BDB5E30B0BF0F336048093F68608BC
:10291000B6C801000100930680FA23809D00238041
:10292000DD00010001008346390593F5FC0F93F6A5
:10293000860FA309D90483463905CD8EA309D9048E
:1029400023800D00C646F3A6068001000100130592
:1029500080FA03463905930639051D8A631C9629BA
:102960007336048013768608B2CC0100010013068A
:1029700080FA23809D002380CD000100010003C662
:1029800006001376F60D2380C60003C60600136604
:1029900006022380C600835609051166D18E2318CE
:1029A000D904835609052166D18E2318D9042380C2
:1029B0000D00E646F3A6068001000100130680FA2A
:1029C0008346390593F60602638006268346390559
:1029D000130C3905A18AFDDA081897000000E7807A
:1029E000A06BF336048093F68608B6D00100010090
:1029F000930680FA23809D002380DD000100010002
:102A000083460C00116693F6F60D2300DC00834626
:102A10000C0093E606022300DC0083560905D18EE4
:102A20002318D904835609052166D18E2318D904A9
:102A300023800D008656F3A60680010001001306D0
:102A400080FA8346390593F60602638A0620834698
:102A50003905A18AEDFE97F0FF1FE780C0632A8C3D
:102A600097F0FF1FE7802063E30C85FF835609057D
:102A700011664255D18E2318D90497000000E780D3
:102A800060638346390513063905A18AFDDAF336FA
:102A9000048093F68608B6D401000100930680FAFC
:102AA00023809D002380DD00010001008346060095
:102AB00093F6F60D2300D60023800D00A656F3A64C
:102AC0000680010001008356090503462905D24707
:102AD000B376DA003306CA021305800C9355F6412B
:102AE0003696330DF6408257333CD6002E9C333653
:102AF000A601330CFC40330CCC40330885039256BE
:102B00004E86B335A5033305A503C29597C00100D2
:102B1000E780A0B163468001631E0C16630C0D169E
:102B2000130615003335A6002E959356F5013696FB
:102B3000B335D600AA959396F50105828585D18E89
:102B40006346B000639D051A638B061A0356C902DB
:102B500015823305D6003336C500B2956348B00000
:102B6000639105241306F00F637DA622894663F363
:102B7000561593078008F3B7078093F78708BED6EA
:102B80000100010037170040930770052300F70488
:102B9000930780FA2300F704010001008356C7025F
:102BA00089678117D58FC207C1832316F7022300D7
:102BB0000704B657F3A7078001000100FA506A54D2
:102BC000DA544A59BA592A5A9A5A0A5BFA4B6A4C49
:102BD000DA4C4A4DBA4D296182801308F5FF33352E
:102BE000A800FD152E951356F5013298B336C8008E
:102BF000AA9695B9F336048093F68608B6CA010002
:102C0000010023809D002380AD0001000100834668
:102C10003905CD8EA309D90423800D00D646F3A62D
:102C200006800100010035B3F336048093F6860870
:102C3000B6CE0100010023809D002380CD0001005D
:102C400001008346390593E60602A309D9042380CF
:102C50000D00F646F3A606800100010095B3F33699
:102C6000048093F68608B6D20100010023809D00FF
:102C70002380CD00010001008346390593E606025A
:102C8000A309D90423800D009656F3A606800100FF
:102C9000010045BB9306F5FF33B5A600FD152E9543
:102CA0009355F501AE96B3B5B600AA951396F50106
:102CB000858269B5F336048093F68608B6D801009C
:102CC0000100930680FA23809D002380DD0001002F
:102CD00001008356C9020566011693F6F60FD18EE0
:102CE000C206C1822316D90223800D00C656F3A660
:102CF000068001000100850A93FAFA0F95B233E6C7
:102D0000B60045C20356C9023305D0403338A0008F
:102D1000B305B040B385054115826345B000D1E1EC
:102D20006371A608894663F0560593078008F3B7D8
:102D3000078093F78708BEDA01000100B71700404B
:102D4000130770052380E704130780FA2380E70444
:102D50000100010003D7C7027D8B2396E702238081
:102D60000704D65781BDF336048093F68608B6DC97
:102D700001000100930680FA23809D002380DD007E
:102D8000010001008356C9020566011693F6F60F8D
:102D9000D18EC206C1822316D90223800D00E656C9
:102DA000B9B793078008F3B7078093F78708BEDEAB
:102DB0000100010037170040930770052300F70456
:102DC000930780FA2300F704010001000356C702AD
:102DD00093975600B297C207C1832316F7022300C8
:102DE0000704F657C1BB914763EEB70217D701003E
:102DF000130707218A05BA959C41BA978287B717AE
:102E0000004003A7470B1345F5FF698F23AAE70A84
:102E100003A7070B698F23A8E70A03A7070A798D81
:102E200023A0A70A8280B717004083A6470B134749
:102E3000F5FFF98E23AAD70A83A6070B558D23A881
:102E4000A70A83A6070A758F23A0E70A8280B7170F
:102E5000004003A7470B498F23AAE70A03A7070BE4
:102E60001345F5FF45BFB717004083A6470B13472F
:102E7000F5FF758F23AAE70A03A7070A598D4DB7F7
:102E8000B717004003A7470B498FEDB7914763EE93
:102E9000B70217D701001307E7178A05BA959C41B7
:102EA000BA978287B717004003A7470D1345F5FF70
:102EB000698F23AAE70C03A7070D698F23A8E70CE6
:102EC00003A7070C798D23A0A70C8280B7170040B9
:102ED00083A6470D1347F5FFF98E23AAD70C83A6C7
:102EE000070D558D23A8A70C83A6070C758F23A06B
:102EF000E70C8280B717004003A7470D498F23AA2C
:102F0000E70C03A7070D1345F5FF45BFB7170040B2
:102F100083A6470D1347F5FF758F23AAE70C03A778
:102F2000070C598D4DB7B717004003A7470D498FC0
:102F3000EDB7797122D43714004026D24AD0035914
:102F400024028354040206D64209C2044ECE52CC57
:102F500056CA13590901C1802DE11379F9F793F489
:102F6000F49F4209C20413590901C18093078008E4
:102F7000F3B7078093F787083EC401000100930769
:102F800070052300F404930780FA2300F404010081
:102F90000100231124032310940223000404A247F8
:102FA000F3A7078001000100B25022549254025945
:102FB000F249624AD24A45618280B7F507008146EC
:102FC0003000B105194597000020E7808081A247B5
:102FD00013972701E34A07FC1369090893E40440A7
:102FE00093098008F3B7098093F787083EC0010072
:102FF0000100930A700523005405130A80FA230088
:10300000440501000100231124032310940223002E
:1030100004048247F3A7078001000100294597F0C7
:10302000FF1FE7802031F3B9098093F989084EC268
:1030300001000100230054052300440501000100A4
:103040008357040293E707202310F40223000404AB
:103050009247B9B7B7170040884742054181937737
:10306000050491EB9377F5013755E80113050580C9
:103070003345F50282809377050C130700046397AC
:10308000E7009377F50137459C1CCDB72165130503
:1030900005D0828037E700E01C435443A183E20659
:1030A000D58F1CC1FD572320F7182322F7188280E3
:1030B00013178500B7E700E023A0E710618123A282
:1030C000A7108280B7F700E08847CC47828081470D
:1030D00037370040A14663C4C7003285828003456C
:1030E000B740E38EA6FE3385F5000345050085074E
:1030F0002304A740CDB797070020938727EF9C4371
:1031000017370020130787293E95636EE5001737B0
:1031100000201307274F6368A70017070020232705
:10312000A7EC3E858280FD57EDBF8280411122C40D
:1031300006C62A8497000000E78000F22947B307FB
:10314000E502B2408D83B3D7870222449507B3D7F7
:10315000E70237370040C207C1832316F700410159
:103160008280411137150E0006C697000000E780E7
:1031700020FCB7370040130770F82381E7000D47A4
:10318000A381E70013070004A380E7000547238716
:10319000E700B24041018280373700408347270073
:1031A0001A0593F7F703C98F93F7F70F2301F70079
:1031B0008280B737004003C7170019C9D98DA38093
:1031C000B70003C70700136787002380E7008280EA
:1031D00093C5F5FFF98DA380B7008280AE872A875B
:1031E000B736004021463738004089E71703000012
:1031F0006700E3F383C8B600E30916FF05078348B9
:10320000F7FFFD17C20723041801C183F9BF41115D
:1032100022C406C62A8497000000E780E0E329471D
:10322000B307E502B2408D83B3D7870222449507E6
:10323000B3D7E70237370040C207C1832316F740F0
:1032400041018280716541111305052006C6970072
:103250000000E78000FCB7370040130770F82381B7
:10326000E7400D47A381E74013070004A380E74030
:1032700005472387E740B24041018280CC4141119C
:1032800006C6328503C6150083C5050022064D8E8D
:1032900042068D654186138875A2630C0611634B47
:1032A000C804138845A26300060D634AC8009385CD
:1032B00035A26301B6082390060029464DA0138865
:1032C00055A26305060D938565A2E316B6FE8D45EE
:1032D0001D4663E6E5081146198E63F3C7003E8676
:1032E000B7E704002390C600FC4797D501009385FB
:1032F000A5D49DA0138895A263030611634E060D05
:103300001388A5A263000613938505A5E315B6FAF5
:1033100099451D4663E5E504198E63F3C7003E86B3
:10332000B7E704002390C600FC479705002093856B
:1033300025D61DA09D451D4663E3E5022146198E55
:1033400063F3C7003E86B7E70400FC472390C6003E
:103350009705002093858534BA9582970146B2403F
:10336000328541018280AD451D46E3EAE5FE3146E6
:10337000198E63F3C7003E86B7E704002390C600AA
:10338000FC4797D501009385A5CDF9B7B1451D46FA
:10339000E3E7E5FC3546198E63F3C7003E86B7E7E1
:1033A00004002390C600FC4797D50100938545CCC7
:1033B00065B78D451D46E3E4E5FA1146198E63F3C2
:1033C000C7003E86B7E704002390C600FC4797D5A8
:1033D0000100938525C749B78D451D46E3E1E5F812
:1033E0001146198E63F3C7003E86B7E704002390A9
:1033F000C600FC4797D50100938545C9B1BFA545D7
:103400001D46E3EEE5F42946198E63F3C7003E86B8
:10341000B7E704002390C600FC4797D501009385C9
:1034200025C31DBFB5451D46E3EBE5F23946198EB0
:1034300063F3C7003E86B7E704002390C600FC474D
:1034400097D50100938545BE01BFB7E7040003A3EC
:103450000713970600209386A6C24146A545170587
:1034600000201305E5B80283797126D252CCAE84D0
:103470002A8A97D50100938565C317D501001305E6
:1034800065C506D63AC622D44AD0368432894ECE95
:1034900056CA97B00100E7808064A28517D5010065
:1034A000130545C497B00100E7806063294597B0D4
:1034B0000100E780A06783C7840093F70702F9EF54
:1034C00083C904008947054532476391F90AD4400E
:1034D00083C7160083C60600A207D58FC166138670
:1034E00016FE638DC7028D16638BD7088D66938693
:1034F00026902945639CD706B7E70400A28622548C
:1035000003A34714B250F249D24A4A86A68502590B
:1035100092545285624A8547456102832D4539E7B9
:10352000130A700F354563638A04B7EA040083A762
:10353000CA04C8442286CA8582978149630A440125
:10354000C84483A78A0433068A408145229582971E
:10355000970700209387073D9C43014581CB9C43FF
:1035600091C74E852286CA8582970145B250225462
:1035700092540259F249624AD24A456182802D45ED
:1035800075F79307700F3545E3E287FEB7E7040050
:10359000FC47C8442286CA8582975DBF2145F9B79A
:1035A0002D455DE703C505000947631FE50803A82E
:1035B0004500411106C6034718003285034608003E
:1035C00022074168518F930828FE6307170563E9B6
:1035D000E80005186303070323900600294591A816
:1035E000130648FE630AC7041518E31707FF1546BC
:1035F0003E87637BF600154701A81306700F3E87D0
:103600006374F6001307700FB7E704002390E60019
:10361000FC471316070111A83E8691C30546B7E77C
:103620000400FC472390C6004206CC4541828297A5
:103630000145B24041018280130600083E87E375D0
:10364000F6FC13070008C9B72390060005458280E1
:103650008280416779176304E504411122C406C6DC
:1036600085472A84639FF500B7E70400228522443A
:10367000B24003A38713970500209385E5294101F4
:10368000028389476399F500B7E7040083A7070B16
:103690008545829771D9B24022444101828082805F
:1036A000411122C437E404008327841326C2AA846C
:1036B000416506C697050020938505267D158297EE
:1036C0008327C40A170500001305E5F8858882974B
:1036D00095C0032304132244B2409244970600206D
:1036E000938686AC4146C545170500201305C59A4B
:1036F00041010283B240224492440145410182804B
:1037000019C59707002023AFA720014582804545B2
:103710008280011122CC06CE26CA4AC84EC69147E5
:10372000094463EDA70417D701001307E7960A05BC
:103730003A951C41AE84B285BA9782879387F4FF8D
:10374000C207C1831307600F61446369F702B7E9D9
:10375000040083A7C904170900201309A9F42686C9
:103760004A8582971306700F01446389C40083A7BA
:103770008904058E81453305990082972285F240A0
:103780006244D2444249B24905618280854761441E
:10379000E396F4FEB7E70400FC4705461705002052
:1037A0001305C5FF82970144D1BF9307700F614491
:1037B000E396F4FCB7E70400FC471306700F170507
:1037C00000201305E5FDF9BF930700086144E39766
:1037D000F4FAB7E70400FC471306000817050020B9
:1037E0001305850BC1B795476144E399F4F8B7E732
:1037F0000400FC47154617050020130525125DB788
:10380000411126C2B7E4040083A7C41322C44AC0EE
:1038100006C62E8497050020938505102A89829775
:10382000058905C5970700209387078783D7A70BCE
:10383000A28503A3440D2310F4002244B240924415
:103840004A850249014641010283B2402244924422
:103850000249494541018280970700202386070CD1
:103860009707002023A4070CB717004003A7070CF5
:10387000B706C0FFFD16758F23A0E70C03A7070D41
:10388000B7064000558F23A8E70C03A7070C3D9B04
:1038900023A0E70C03A7070D1367070123A8E70C74
:1038A0008280B717004003A5470C83A7470C5981B6
:1038B00013451500C18B058999E31365250097070A
:1038C000002083C767066380A70297070020238D27
:1038D000A70411C9970700209387470503A3070092
:1038E0006303030002838280114517F3FFFF670023
:1038F00083C3011122CC06CE3714004026CA4AC821
:103900004EC652C483447405034AB40583498405F2
:103910000349940597F0FFFFE780C09B8347A40508
:1039200093F4F40F137AFA0F93E71700230DF404BE
:1039300093F9F90F1379F90FB717004003C7A705DB
:10394000058B6DFF03D5C705A38D4705238C370570
:10395000A38C2705A38B9704F2406244D2444249CA
:10396000B249224A0561828041119397050122C420
:1039700006C626C2C1872E8463DC0700B7E40400B4
:10398000FC54829719C1BC5482972165218D15A8DA
:1039900093F7150013C515008DE793F725009DC714
:1039A00097000000E78020F0B7E70400BC4F130643
:1039B000000A8945170500200345C5F7829713457E
:1039C0002400B24022449244410182809397250111
:1039D00063D80702B7E4040083A7C41E8297970048
:1039E0000000E780A0F0BC4C3756070013060630F5
:1039F0008965170500200345E5F38297096579B7C6
:103A0000939715010145E3DE07FA17C50100130579
:103A1000657597B00100E7806024B7E70400BC4FEC
:103A2000130600649165170500200345A5F08297F1
:103A30001165A9BF1D71A2CC37E404005C5C485835
:103A400086CE494697C501009385456D829711E959
:103A500017C501001305C56D97B00100E780002070
:103A600001A0B7F600E0795798CAFD57DCCA056790
:103A7000B7E700E023A0E7101306F00290C223A0EE
:103A8000E71801000100370700201847130600045B
:103A900081459706002023ADE6E84157A38AE74019
:103AA0003C4408088297971700209387A7853EC853
:103AB000856713870740938757D1231AE1002312A4
:103AC000F1021307B00F97F7FFFF9387E75F23100B
:103AD000E1023ED81547970700009387C7E1B7F585
:103AE0000700A30FE1003EDC05479707000093871E
:103AF000E7DF81463000E10519452301E1023EDEA2
:103B000097F0FF1FE780E0CD180881479946300005
:103B10003E960346060085070507A30BC700E398FA
:103B2000D7FEC24791C70357410185676373F7000A
:103B300001A0B7E7040083A7470A08088297AA856F
:103B400011C917C501001305E55F97B00100E780B3
:103B500000F901A0F640664425618280411126C229
:103B6000B7E4040083A7040806C622C417050000B2
:103B70001305C5DF8297170400201304A4DB23007C
:103B8000A40097000000E780800297000000E78013
:103B9000E0CC03450400224403A38405B2409244D0
:103BA00013060032896541010283797106D622D459
:103BB00013078008F337078093F787083EC2010098
:103BC0000100B7170040930570052380B704130662
:103BD00080FA2380C7040100010083C6F70293F630
:103BE000A60FA387D702238007049246F3A6068078
:103BF0000100010073370780137787083AC401007A
:103C000001002380B7042380C7040100010003C71B
:103C1000F70213672700A387E70223800704A24760
:103C2000F3A7078001000100054597E0FFFFE7804B
:103C3000A06D97000000E78060CB01478146814777
:103C4000054685451305407E97E0FFFFE780A0709D
:103C500037E404003C446800514681458297B70729
:103C6000C0A83EC8B787E803938707D03ECA97E746
:103C7000FF1F9387C7743EC67C5868008297B25076
:103C8000225445618280411197D501009385C5AFCB
:103C900017C501001305054406C697B00100E7806B
:103CA00000E417D501001305E5C697B00100E780D1
:103CB00000E3B2402945410117B30100670003E763
:103CC000411197D50100938565AD17C50100130516
:103CD000654006C697B00100E78060E017D5010097
:103CE000130505C297B00100E78060DFB2402945A7
:103CF000410117B30100670063E3411122C406C606
:103D0000834705002A849DC797D501009385C5AEDA
:103D100017C501001305053C97B00100E78020DCC2
:103D20004C4017D50100130525D197B00100E7805D
:103D300000DB3DA058410DEF97D501009385C5AB41
:103D400017C501001305053997B00100E78020D998
:103D500017D501001305C5CF97B00100E78020D823
:103D60002244B2402945410117B30100670003DC3A
:103D7000A1679386D7036313D70297D50100938574
:103D8000A5A717C501001305E53497B00100E7802A
:103D900000D517D501001305A5CC7DBFED0797D53C
:103DA0000100938565A517C501001305A532631BA6
:103DB000F70097B00100E78080D217D50100130506
:103DC00065CB59BF97B00100E78060D14C4017D553
:103DD0000100130525CC91BF411197D501009385B2
:103DE000259D17C501001305E52E06C697B00100F5
:103DF000E780E0CEB2402945410117B301006700DA
:103E0000E3D2797122D426D24AD02E842A898145E0
:103E1000B2844800714606D697E0FFFFE780202F66
:103E200097F7FF1F93874759DC4783D70700231471
:103E300021012313F10097500000E78020E585471A
:103E4000A305F1009307401F3EC6FD572305A100BF
:103E5000230AF10097500000E78080F72686A285AC
:103E6000480097500000E78040E5B2502254925439
:103E70000259456182809727002023980798972749
:103E8000002023810788B7E70400BC47411106C61C
:103E900041468145170500201305453582971707D0
:103EA00000200347A7369307F00A6315F70293072C
:103EB000F0F8894517050020130545351707002040
:103EC0002306F73497070020A38207349760000089
:103ED000E780209E97600000E78080C98145370514
:103EE00004009707002023A1073097070020239B99
:103EF000072E970700202388072E97070020239777
:103F00000726970700202395072497070020239A68
:103F1000072C970700202393072E97300000E78097
:103F2000202A014597600000E780A0A197D50100F5
:103F30009385858A17C501001305C51997B001003F
:103F4000E780E0B917D50100130505BB97B0010064
:103F5000E780E0B8B2402945410117B3010067008E
:103F6000E3BC4111814617F6FF1F13062642854523
:103F7000170500200355851D06C697C00000E78081
:103F8000C02715C997D501009385C58517C50100C0
:103F90001305451497B00100E78060B417D5010000
:103FA000130585A597B00100E78060B3294597B058
:103FB0000100E780A0B797D501009385A58217C5BA
:103FC00001001305251197B00100E78040B117D516
:103FD00001001305A5A397B00100E78040B0294573
:103FE00097B00100E78080B497F7FF1F9387C73C25
:103FF000DC47054797C501009385C57E2390E70000
:1040000017C501001305050D97B00100E78020AD2D
:1040100017D501001305C5A097B00100E78020ACBB
:10402000B2402945410117B30100670023B0411197
:1040300022C497C501009385657D2A8417C50100B8
:104040001305450906C697B00100E78040A94C401A
:1040500017D501001305C59797B00100E78020A888
:10406000294597B00100E78060AC0347040093073F
:10407000F00F631FF70297C501009385257917C5D7
:1040800001001305250597B00100E78040A54C40CD
:1040900017D501001305C59497B00100E78020A44F
:1040A0002244B2402945410117B30100670003A82B
:1040B000B240224441018280411122C426C22A8496
:1040C000AE8417C501001305E50097C5010093856F
:1040D000A56F06C697B00100E78060A017D5010064
:1040E000130505A097B00100E780609F294597B0B0
:1040F0000100E780A0A397C501009385E56C9707B1
:1041000000202395870417C501001305A5FC05446D
:1041100097070020239A970297070020239787028A
:10412000971700202393976E97B00100E780209B9C
:104130009715002083D5656D17D501001305C59A25
:1041400097B00100E780A099294597B00100E7806A
:10415000E09D971700202387875A97F7FF1F9387C3
:10416000A725DC4703D70700C167FD176312F702D5
:104170002244B7E70400B240924403A3870517F531
:10418000FF1F0345A57B1306000A854541010283F5
:10419000B2402244924441018280B1C1411122C403
:1041A00017C50100130505F32E8497C501009385FB
:1041B000E56006C697B00100E7806092A28517D53A
:1041C00001001305259197B00100E780409122443A
:1041D000B2402945410117B3010067002395828051
:1041E000011122CC06CE26CA4AC84EC693F7150046
:1041F0002E84BDC797000000E780E0D6930710F833
:10420000170700202304F7009707002083D7C7F380
:10421000914517070020A30BF7FE17050020130593
:10422000E5FEA183170700202303F7FE9707002070
:10423000A38F07FC97500000E780A06705459750C3
:104240000000E780007097200000E780600F1345B2
:104250001400F2406244D2444249B249056182806E
:1042600093F705108DC7054597500000E780606DF6
:10427000171500200355655997500000E780C03896
:1042800097200000E780C00B13450410D9B793F7BF
:104290002500E9CF170700200357C7F469C7AD64AD
:1042A000B71900409384A4AA23A099009706002080
:1042B000938686F3944297D701009387E785170684
:1042C0000020034646F2814517050020130505F23C
:1042D00097700000E780200E23A0990097F7FF1F3A
:1042E0002390A7FE2A8941C197C5010093854556B1
:1042F00017C50100130505DE97A00100E780207EA9
:10430000CA8517C501001305A5F497A00100E78031
:10431000007D294597B00100E78040819707002084
:10432000239207EC930710F8170700202300F7EEFD
:104330009707002083D747E117070020A308F7EC71
:10434000A183170700202304F7EC91458D4717053B
:1043500000201305A5EB17070020A30AF7EA9750E2
:104360000000E780005513452400E5B593F74500AC
:10437000D1C397C501009385A54D17C5010013054D
:1043800065D597A00100E780807517C5010013056A
:10439000E5ED97A00100E7808074294597A0010012
:1043A000E780C078930720F8170700202300F7E67E
:1043B0009707002083D787DB17070020A308F7E4BF
:1043C000A183170700202304F7E48547170700207F
:1043D000A30FF7E297500000E780809F17050020A9
:1043E0001305C5E2914597500000E780804C1345C6
:1043F000440085B593F78500A9C797C5010093854B
:10440000254517C501001305E5CC97A00100E780FD
:10441000006D17C501001305A5E697A00100E78010
:10442000006C294597A00100E780407097070020A5
:10443000239A07DA97700000E780C00713458400CD
:1044400009BD93F70501D1C3854517050020035524
:10445000E5D197600100E78080BD97C50100938595
:10446000253F17C501001305E5C697A00100E780A9
:10447000006717C501001305E5E197A00100E7807B
:104480000066294597A00100E780406A930730F84D
:1044900017070020230CF7D69707002083D707CDF6
:1044A00017070020A304F7D617050020130505D62B
:1044B000A1838D4517070020230BF7D497500000E8
:1044C000E780203F1345040169B393F70502D1C784
:1044D00097C501009385C53717C50100130585BF32
:1044E00097A00100E780A05F17C501001305C5DC98
:1044F00097A00100E780A05E294597A00100E78012
:10450000E062930740F8170700202301F7D09707D0
:10451000002083D7E7C317070020A309F7CEA183A4
:10452000170700202305F7CE854717070020A300B3
:10453000F7CE97070020239D07C097500000E78023
:10454000208917050020130565CC91459750000080
:10455000E780203613450402EDB993F70504FDC347
:1045600097C501009385C52E17C50100130585B6B3
:1045700097A00100E780A05617C50100130545D597
:1045800097A00100E780A055294597A00100E7808A
:10459000E0599707002083C767C71307700A63862F
:1045A000E7061307800A638CE7081307600A639322
:1045B000E704930760F8170700202309F7C497075B
:1045C000002083D707C217070020A301F7C4A183E7
:1045D00017070020230DF7C2854717070020A30CFB
:1045E000F7C2B14517050020130545C297500000DA
:1045F000E780202C97400000E780807D134504046D
:1046000097070020239F07BCA9B1930770F81707ED
:104610000020230DF7BE9707002083D787BC17071C
:104620000020A305F7BEA183170700202301F7BED2
:10463000854717070020A30DF7BC994565B7930779
:1046400080F8F1B793F705080145E38407C097C5E3
:1046500001009385E51F17C501001305A5A797A0C5
:104660000100E780C04717C501001305E5C797A003
:104670000100E780C046294597A00100E780004B74
:104680009307A0F8170700202302F7B89707002028
:1046900083D7C7B617070020A30AF7B6A183170769
:1046A00000202306F7B6854717070020A301F7B6B9
:1046B00097070020239407B497400000E7804071DB
:1046C00017050020130585B4914597500000E78039
:1046D000401E13450408B5BE011122CC37E4040086
:1046E0005C5C06CE354697C501009385E52317D55A
:1046F0000100130565F2829711E917C50100130542
:1047000025A397A00100E780605501A097F7FF1F40
:10471000938787233EC4B7F5070085679387078093
:10472000814617F6FF1F1306A621E10519453EC66F
:1047300097E0FF1FE780E00A7C44194697F5FF1FCA
:104740009385052017050020130585A28297340064
:1047500017F6FF1F1306C61E97C501009385456E09
:1047600017C501001305456F97700000E780A099F9
:104770002A841DCD97C501009385850C17C50100BE
:104780001305459597A00100E7806035A28517C500
:1047900001001305651A97A00100E7804034294500
:1047A00097A00100E7808038F24062440561828072
:1047B00097E00000E780A0FF17C501001305C50EB4
:1047C00097600000E780E08D97A00000E780E0534D
:1047D00097600100E78060B817F5FF1F130545BA21
:1047E00097600100E78000A117C501001305C50C03
:1047F00097600100E780E0B82A8497600000E780B6
:1048000020F497100100E780409097800100E78036
:10481000602997700000E780005097600000E780F3
:10482000206A97300100E780A05197C50100938569
:10483000250117C501001305E58919C897A00100D6
:10484000E780E029A28517C5010013052511A1B74E
:1048500097A00100E780A02817C5010013054512A5
:1048600097A00100E780A027294597A00100E780D5
:10487000E02B97300100E780802D97F00000E78063
:10488000404C7DC185453705040097300000E78026
:10489000209397C501009385A5FA17C5010013055C
:1048A000658397A00100E780802317C501001305E9
:1048B000A50E97A00100E7808022294597A001005E
:1048C000E780C02697F7FF1F9387879E83D707004F
:1048D00017170020231BF7F2854717170020230323
:1048E000F7E297F7FF1F938727ADDC4703D7070051
:1048F000C167FD176316F70097F0FFFFE780A0661A
:1049000097700000E78040CB1305C5149770000036
:10491000E78040CB97200000E78040B4972000005C
:10492000E78000A217150020035525EE97500000E0
:10493000E78080CD054597500000E780800097C54F
:1049400001009385E5EF17B501001305A57897A041
:104950000100E780C01817C501001305250697A0C0
:104960000100E780C01725BD97C50100938545ED7F
:1049700017B501001305057697A00100E780201602
:1049800017C501001305451797A00100E780201502
:10499000294597A00100E7806019014569BF4111D1
:1049A00022C437E404008327041A06C6829797506E
:1049B0000000E78020C983270408170500001305BD
:1049C0006582829797F7FF1F238AA7F617F5FF1FC7
:1049D0001305859E97400000E78020722244B24074
:1049E000410117030000670063CFB7E70400FC47ED
:1049F0001171A2DDCAD986DFA6DBCED72E8432891B
:104A00002E86AA851705002013054580829717F783
:104A1000FF1F1307A77F8347070093068002938732
:104A2000E70793F7F70FE3ECF610BA898A0717B791
:104A3000010013076773BA979C43BA9782878D4723
:104A400097C50100938505E217B501001305856838
:104A5000630FF40097A00100E780600817C501000C
:104A60001305059F97A00100E7806007BDA497A0EC
:104A70000100E780C00617C501001305E59E97A059
:104A80000100E780C005294597A00100E780000AE2
:104A9000930720F8114697F5FF1F938525774A85E0
:104AA00017F7FF1F2304F77697F7FF1FA3810776F9
:104AB00097F0FFFFE78020352A841DC997C50100C4
:104AC000938545DA17B501001305C56097A001006D
:104AD000E780E000A28517C501001305A59C97A0FB
:104AE0000100E780C0FF294597A00100E78000048E
:104AF00097C50100938505D717B501001305855D9E
:104B000097A00100E780A0FD17C501001305C59A15
:104B100097A00100E780A0FC294597A00100E7804D
:104B2000E0004165930730FA054697F5FF1F93852E
:104B3000E56D7D1517F7FF1F230AF76C97F0FFFF50
:104B4000E780602C2A841DC997C50100938585D113
:104B500017B501001305055897A00100E78020F85C
:104B6000A28517C501001305E59397A00100E78012
:104B700000F7294597A00100E78040FBB7E7040054
:104B8000BC4F0566130606C8A14517F5FF1F034570
:104B9000E5DA8297FE506E54DE544E59BE591161CB
:104BA000828091476303F40297C50100938585CB0A
:104BB00017B501001305055297A00100E78020F208
:104BC00017C501001305859271BDB7E70400FC4FBE
:104BD000914517F5FF1F034565D6829797C50100DC
:104BE000938545C817B501001305C54E97A0010070
:104BF000E780E0EE17C501001305059197A00100BD
:104C0000E780E0ED294597A00100E78020F297407A
:104C10000000E780E01B914535A485476303F4025B
:104C200097C50100938505C417B501001305854A92
:104C300097A00100E780A0EA17C501001305458E83
:104C400015B597F7FF1F23932753B7E704000566B1
:104C5000BC4F130606C8C1450DBF8D476303F40260
:104C600097C50100938505C017B50100130585465A
:104C700097A00100E780A0E617C501001305058C89
:104C8000D5B3930740F8114697F5FF1F9385055854
:104C90004A8517F7FF1F230BF75697F7FF1FA388C7
:104CA000075697F0FFFFE78000162A84E30405EE1D
:104CB00097C50100938505BB17B501001305854114
:104CC00097A00100E780A0E1A28517B501001305B8
:104CD000657D97A00100E78080E0294597A001004D
:104CE000E780C0E445BD9147E31CF4F6B7E7040054
:104CF000FC4F9305000217F5FF1F034525C482975B
:104D000097C50100938505B617B501001305853CCD
:104D100097A00100E780A0DC17C50100130585837B
:104D2000F1BD894763E3870297C50100938585B389
:104D300017B501001305053A97A00100E78020DAB6
:104D400017C501001305458231BB97F4FF1F83C4CB
:104D5000044C97F7FF1F83C7774B97C501009385D6
:104D600065B0A20417B501001305C536DD8C97A008
:104D70000100E780C0D6A28517C501001305058094
:104D800097A00100E780A0D5C204294597A00100A3
:104D9000E780C0D9C1849305D4FF93960401C182F2
:104DA0004A8693F5F50F17F5FF1F13055546972013
:104DB0000000E780A044E35F90DC930750F817F70A
:104DC000FF1F2305F74483C73900228697F5FF1F8D
:104DD0009385C54385074A8517F7FF1FA309F74247
:104DE00097F0FFFFE78020022A84E30505DA97C5E4
:104DF0000100938525A717B501001305A52D97A0E0
:104E00000100E780C0CDA28517C50100130585CB41
:104E1000C9B5894763E3870297C50100938585A4D7
:104E200017B501001305052B97A00100E78020CBE3
:104E300017B501001305457635B197400000E780AE
:104E400020F9A28517F5FF1F1305453C9750000078
:104E5000E78020A681B38D476303F40297C5010064
:104E6000938545A017B501001305C52697A001003D
:104E7000E780E0C617B501001305C573E5B6B76650
:104E800002000146B7750200054597E0FF1FE78065
:104E90004095930760F817F7FF1F2309F73697F738
:104EA000FF1FA38607369307000617F7FF1F23018E
:104EB000F736894717F7FF1FA30CF73497F7FF1F43
:104EC0002389073497F7FF1FA3850734C14717F7D6
:104ED000FF1F2301F734930720F917F7FF1FA30BD8
:104EE000F732314697F7FF1FA387A73297F5FF1FC9
:104EF0009385C5314A8597F7FF1F238E073097F0BA
:104F0000FFFFE78040F02A84E30605C897C501004B
:104F10009385459517B501001305C51B97A00100A2
:104F2000E780E0BBA28517B501001305256A55B3DC
:104F3000B1476303F40297C501009385A59217B5A5
:104F400001001305251997A00100E78040B917B5A6
:104F500001001305656939B6B7E70400FC4F9305F6
:104F6000000417F5FF1F0345659D829797400000D9
:104F7000E78000E6B145F9B5914763E3870297C53D
:104F800001009385258E17B501001305A51497A080
:104F90000100E780C0B417B501001305A566D9B4B8
:104FA00097F4FF1F83C4C42697F7FF1F83C73726D4
:104FB000A204DD8C8E04B77702006D14BE942286A5
:104FC000A68517B501001305256597A00100E780A8
:104FD00000B1B7E70400FC47228697F5FF1F9385D1
:104FE00035232800829793160401C1823000A685DC
:104FF000094597D0FF1FE780C07E2A8409C917B5ED
:1050000001001305256397A00100E78020C59307E1
:1050100070F8194697F5FF1F9385451F4A8517F7C6
:10502000FF1F2305F71E97F7FF1FA383871E97F027
:10503000FFFFE78040DD2A84E30E05B497C5010039
:105040009385458217B501001305C50897A0010097
:10505000E780E0A8A28517B501001305A55E95B904
:105060009947630BF41297B501009385A57F17B597
:1050700001001305250697A00100E78040A617B59B
:1050800001001305A55DF9BA914763E3870297B55F
:1050900001009385257D17B501001305A50397A091
:1050A0000100E780C0A317B501001305A55C5DBA38
:1050B00097F4FF1F83C4C41597F7FF1F83C73715E5
:1050C000A204DD8C8E04B77702006D14BE94228694
:1050D000A68517B501001305255B97A00100E780A1
:1050E00000A0B7E70400FC47228697F5FF1F9385D1
:1050F00035122800829793160401C1823000A685DC
:105100000D4597D0FF1FE780C06D2A8409C917B5E8
:1051100001001305255997A00100E78020B49307EB
:1051200080F8194697F5FF1F9385450E4A8517F7B6
:10513000FF1F230DF70C97F7FF1FA38B870C97F02A
:10514000FFFFE78040CC2A84E30605A497B5010061
:105150009385457117B501001305C5F797A00100A8
:10516000E780E097A28517B501001305E55495B6D1
:1051700099476303F40297B501009385A56E17B5AF
:105180000100130525F597A00100E780409517B5AC
:1051900001001305E553F9B0B7E70400FC4F930590
:1051A000000417E5FF1F03456579829797400000CB
:1051B000E78000C2994579B18D476303F40297B542
:1051C00001009385256A17B501001305A5F097A086
:1051D0000100E780C09017B501001305E55059B0F4
:1051E00017B501001305455197A00100E78000A7FE
:1051F0001305C01297D0FF1FE780A014014597E068
:10520000FFFFE78060E90D4597100000E780A0A050
:10521000294597D0FF1FE780C01297D0FF1FE78076
:1052200020038DBA99476303F40297B50100938573
:10523000656317B501001305E5E997A00100E78054
:10524000008A17B501001305E54B29B817F7FF1FB2
:10525000034717FC97F7FF1F83C787FB22075D8F64
:105260009166BA96C2061166C1821306F6EF8D47A3
:105270006365D60297E7FF1F938707149C4B17F6C9
:10528000FF1F0346D6F89386C7002DC203D607003A
:1052900069CA8907E39CD7FE89471307A0F811461E
:1052A00097F5FF1F938585F64A8597F6FF1F238F95
:1052B000E6F417F7FF1FA30CF7F497F0FFFFE78062
:1052C00080B42A84E308058C97B50100938585593D
:1052D00017B50100130505E097A00100E7802080C5
:1052E000A28517B5010013052543E5B203D60700D3
:1052F000630EE60A8907E39BF6FE8D4779BF914767
:105300006304F40297B501009385C55517B50100F4
:10531000130545DC97900100E780607C17B501001C
:10532000130505416FF00FF4B7E70400FC4F930538
:10533000000817E5FF1F034565608297C9B897B558
:1053400001009385255217B501001305A5D8979044
:105350000100E780C07817B501001305E53E6FF046
:105360006FF02390E70017E5FF1F1305E504973062
:105370000100E78040A397B501009385A54E17B5BE
:105380000100130525D597900100E780407517B5FA
:1053900001001305653C97900100E78040742945A2
:1053A00097900100E78080788147C5BD2390070072
:1053B00017E5FF1F1305450097300100E780A09E09
:1053C00097B501009385054A17B50100130585D0EF
:1053D00097900100E780A07017B5010013054539CB
:1053E0005DBF411122C406C6834705002A849DC7BC
:1053F00097B501009385C54217B50100130585CD0A
:1054000097900100E780A06D4C4017B5010013058F
:10541000A57197900100E780806CE1A05841B70723
:10542000CF009387777D631DF70697B501009385BD
:10543000253F17B501001305E5C997900100E780E6
:10544000006A1C448356E4008355C40003C6070069
:1054500017B501001305C56E97900100E78020681D
:10546000294597900100E780606C0357E400970797
:10547000002083D787396309F7008355C4000844A7
:1054800097E0FFFFE780C0D50356E4008355C400D2
:1054900008442244B240410117F3FFFF670023553F
:1054A000B707CC009387777D6315F70497B50100A4
:1054B0009385053717B501001305C5C19790010005
:1054C000E780E0611C448356E4008355C40003C6B2
:1054D000070017B501001305A56697900100E78046
:1054E00000602244B2402945410117930100670042
:1054F000E363B707CE009387777D6304F70297B520
:1055000001009385E53117B501001305A5BC9790FF
:105510000100E780C05C4C4017B5010013058557BA
:10552000CDBDB240224441018280411122C44AC013
:1055300006C626C29307D00D2A892E841306D00DE5
:1055400063E3B7002E86B7E70400FC4742064182BA
:10555000CA8517F5FF1F130565CB829797B5010024
:105560009385053217B501001305C5B69790010064
:10557000E780E05697F5FF1F83C545C917B50100C1
:10558000130505D897900100E7806055294597904D
:105590000100E780A05997F4FF1F938424C783C7B5
:1055A000040041479387070693F7F70F636CF75A98
:1055B00017B70100130787C58A07BA979C43BA97A4
:1055C0008287994763E7870297B501009385452B4A
:1055D00017B50100130505B097900100E780205032
:1055E00017B50100130545D297900100E780204FC1
:1055F0008DA497F7FF1F83C777C1DDCB17F7FF1F78
:105600000347F7C097F7FF1F83C767C022075D8F67
:1056100097F7FF1F83C7C7BFC2075D8F97F7FF1FAD
:1056200083C717BFE207D98F17F7FF1F232EF7BADB
:1056300083C7640097B501009385852417B50100E1
:10564000130545A917F7FF1F230FF7B8979001001F
:10565000E780E04897F7FF1F938707B98C4317F659
:10566000FF1F034646B817B501001305A5CB979059
:105670000100E780C046294597900100E780004B74
:1056800097F7FF1FA38407B82244B240924402490F
:10569000930700F817F7FF1F230AF7B69D4517F584
:1056A000FF1F1305A5B641011743000067006320E3
:1056B00097600000E78080EF97F7FF1F2389A7B46A
:1056C0009357850017F7FF1FA303F7B493570501FE
:1056D0002A8417F7FF1F230DF7B293578501014561
:1056E00017F7FF1FA306F7B297600000E78060F08E
:1056F00097F7FF1F238FA7B097B501009385451833
:1057000017B501001305059D97900100E780203D26
:1057100017F6FF1F0346E6AFA28517B50100130574
:10572000E5C1B1B7C94763E3870297B50100938527
:10573000251517B501001305E59997900100E7803D
:10574000003A17B501001305E5C079BD37E4040040
:105750007C44414697F5FF1F938555AB17F5FF1F16
:105760001305C5A8829797F7FF1F83C747AB17F7A5
:10577000FF1F0347B7AAA20703238405D98F17F792
:10578000FF1F2311F7A61306000A89452244B240E1
:105790009244024917E5FF1F0345451A4101028360
:1057A000894763E3870297B501009385650D17B5B7
:1057B00001001305259297900100E780403217B54C
:1057C00001001305E5C80DB517F4FF1F034424A419
:1057D00097F7FF1F83C797A397B501009385450AE5
:1057E000220417B501001305E58E5D8C979001002A
:1057F000E780E02EA28517B50100130525B7979025
:105800000100E780C02D294597900100E780003214
:105810000D4697F5FF1F9385659F228597E0FFFF53
:10582000E780605EAA8421C197B501009385450594
:1058300017B501001305058A97900100E780202A1B
:10584000A68517B501001305A5B397900100E78061
:1058500000292244B240924402492945410117934C
:1058600001006700A32C97F7FF1F23918790B7E7EC
:105870000400116603A38705130606E8914539B7AE
:10588000894763E3870297B50100938565FF17B5E4
:1058900001001305258497900100E780402417B587
:1058A00001001305A5C989B317F4FF1F034424960B
:1058B00097F7FF1F83C7979597B50100938545FC20
:1058C000220417B501001305E5805D8C9790010057
:1058D000E780E020A28517B501001305A5AB9790DE
:1058E0000100E780C01F294597900100E780002450
:1058F0000D4697F5FF1F93856591228597E0FFFF81
:10590000E7806050AA841DC197B50100938545F7D3
:1059100017A501001305057C97900100E780201C66
:10592000A68517B50100130525A805B797F7FF1F32
:1059300023908782B7E70400116603A38705130647
:1059400006E89305000299B5894763E3870297B596
:1059500001009385E5F217A501001305A57797903F
:105960000100E780C01717B501001305E5BFADB909
:1059700097F4FF1F83C4A48997F7FF1F83C7178974
:1059800097B501009385C5EFA20417A50100130583
:105990006574DD8C97900100E7806014A68517B5CB
:1059A00001001305E5A197900100E7804013294508
:1059B00097900100E7808017228697F5FF1F938557
:1059C000E584268597E0FFFFE780E0432A84630CA7
:1059D000051A97B501009385A5EA17A501001305DF
:1059E000656F97900100E780800FA28517B50100D1
:1059F0001305459E99BD854763F7871883451900B0
:105A00002244B24092440249B335B00097E7FF1FE9
:105A10002388B77617B501001305059D410117933B
:105A200001006700C30BA2852244B24092444A851C
:105A3000024941011703000067002324954763E3EF
:105A4000870297B501009385A5E317A5010013050B
:105A5000656897900100E780800817B5010013057D
:105A600065CA59B617E4FF1F0344647A97E7FF1F1E
:105A700083C7D77997B50100938585E0220417A5E0
:105A80000100130525655D8C97900100E7802005D6
:105A9000A28517B501001305A59697900100E78030
:105AA0000004294597900100E7804008194697E5D2
:105AB000FF1F9385A575228597E0FFFFE780A0343F
:105AC000AA841DC197B50100938585DB17A5010048
:105AD0001305456097900100E7806000A68517B523
:105AE00001001305E59295B397E7FF1F2398877090
:105AF000B7E70400116603A38705130606E89305BC
:105B0000000869B197B50100938585D717A50100F5
:105B10001305455C11E897900100E78040FC17B53C
:105B2000010013052590C9B497900100E78020FB80
:105B300017B501001305859097900100E78020FAC2
:105B4000294597900100E78060FE2244B2409244CC
:105B5000024997E7FF1F2397076841011763000079
:105B60006700439597B50100938585D117A501007E
:105B70001305455697900100E78060F617B50100C0
:105B8000130585BC95B4B2402244924402494101B8
:105B90008280411106C622C497E0FFFFE780A0265D
:105BA00021CD97E7FF1F83D7C75D85072A8417E7B5
:105BB000FF1F2318F75C97B501009385E5CD97E7A4
:105BC000FF1F2391A75C17A501001305A55097900F
:105BD0000100E780C0F0A28517B50100130585EE2E
:105BE00097900100E780A0EF2244B240294541018F
:105BF00017930100670083F397E7FF1F83D7A75828
:105C0000B2402244850717E7FF1F231EF7564101C4
:105C10008280411122C491462A8417E6FF1F130691
:105C2000E66C9D652D4506C697D0FF1FE78060BBDB
:105C3000B7F7070003C70701A5476313F70001A0E3
:105C40009306001001469D65254597D0FF1FE7800C
:105C500040B997E7FF1F238B87682244B2409146E3
:105C600017E6FF1F130686689D652945410117D376
:105C7000FF1F670003B71171CED7B7E9040083A7F0
:105C8000C904CAD917E9FF1F13094958A2DD2E8696
:105C900086DFA6DB2E84AA854A85829797E7FF1FB9
:105CA00083C7C7561307700A6385E710636DF70053
:105CB0001307600A6385E704FE506E54DE544E59A4
:105CC000BE59116182801307800A6385E7161307A6
:105CD000900AE393E7FE8D476306F41C97B5010035
:105CE000938585F117A501001305C53E9790010026
:105CF000E780E0DE17B50100130545ED25A08D47CF
:105D0000630CF40297B50100938505EF17A5010018
:105D10001305453C97900100E78060DC17B5010052
:105D2000130505E497900100E78060DB2945979013
:105D30000100E780A0DF49B7854717B501001305CB
:105D4000E5E317E7FF1F230DF74297900100E78077
:105D5000E0F0B7750200B76602000146054597D02E
:105D6000FF1FE78000A8930760F817E7FF1F230FC6
:105D7000F74897E7FF1FA38C07489307002617E70C
:105D8000FF1F2327F748E5779387072117E7FF1FB2
:105D90002312F748B14597E7FF1F238E074697E781
:105DA000FF1FA38AA7464A8597000000E780E016F8
:105DB00021B7914763E3870297B501009385C5E357
:105DC00017A501001305053197900100E78020D148
:105DD00017B50100130585DCB1B797E4FF1F83C435
:105DE000244397E7FF1F83C79742A204DD8C83A754
:105DF000C9046D14228697E5FF1F9385754128001D
:105E000082978E0493160401B7750200C182300098
:105E1000A695094597D0FF1FE780A09C930770F8CF
:105E200017E7FF1F2304F73E994597E7FF1FA3815C
:105E3000A73E95BF914763E3870297B5010093851D
:105E4000A5DB17A501001305E52897900100E78061
:105E500000C917B501001305E5D5E9B597E4FF1FA3
:105E600083C4043B97E7FF1F83C7773AA204DD8C06
:105E700083A7C9046D14228697E5FF1F93855539C2
:105E8000280082978E0493160401B7750200C18220
:105E90003000A6950D4597D0FF1FE78080949307AB
:105EA00080F8BDBF17B50100130585D39790010099
:105EB000E780C0DA930790F82304F10083471900C4
:105EC0008D452800A304F100834729002305F10034
:105ED00097000000E78060041305C01297C0FF1F01
:105EE000E7802046014597D0FFFFE780E01A0D4587
:105EF00097000000E78020D2294597C0FF1FE78068
:105F0000404497C0FF1FE780A0347DB397E7FF1F91
:105F100023A6A73E828097E7FF1F9387273E03A310
:105F200007006303030002831743000067006398C0
:105F300041114AC09706002083D6268D328917D694
:105F4000FF1F0356864922C426C206C62A84AE8491
:105F500097000000E780C05B35C12DC0994763FF03
:105F600097048347140003470400A207D98F1397AF
:105F70008700A183D98FC2073167C1831307C75533
:105F8000639EE70297D7FF1F83D72745A301F4003D
:105F9000A1832302F4009707002083D7078791C7C6
:105FA000A302F400A1832303F400A68517B5010022
:105FB000130585C897900100E78060B297F7FF1F2F
:105FC00083C74774A5C797D5FF1F83D5054117B56C
:105FD0000100130525C897900100E78040B0268690
:105FE000A28517D5FF1F0355453F97000000E780A6
:105FF00080BA6306090497F7FF1F83C7A770A1E360
:1060000097E7FF1F83C7C72F9DCB95C897E7FF1F53
:1060100083C707178DE722852244B2400249A6852F
:1060200092444101174300006700A38817B501009F
:10603000130545C397900100E78040C25DBFB240A1
:10604000224492440249410182808347550083459E
:10605000450017B501001305E5BCA207DD8D1793B8
:1060600001006700C3A717B501001305A5BA179370
:1060700001006700A3BE8D4763FBB70A011126CA62
:1060800006CE22CC0344350097E4FF1F83C4542777
:1060900097B501009385C5BDB337800017E7FF1F93
:1060A000A300F72609C497B50100938525BD17B550
:1060B0000100130525BD97900100E78040A297E7F6
:1060C000FF1F83C7F7236386970097000000E780D0
:1060D000E02C97E7FF1F83C7B7228DC785472306AC
:1060E000F100B7E7040083A7471770008545130543
:1060F0005030829717B501001305C5B9979001007C
:10610000E780C0B59967938757EE2316F1006800C2
:1061100085479145A30781002307F1009700000000
:10612000E780A0DFF2406244D24405618280828031
:10613000894763F7B708011122CC06CE26CA8344EB
:10614000250085472A84639DF404914763F5B704CD
:10615000034545008347340022055D8D97D7FF1F17
:10616000239DA72697000000E780604399679387E7
:1061700067EE2314F1008347340023059100A30543
:10618000F10083474400954528002306F10097005D
:106190000000E78080D8F2406244D24405618280EA
:1061A000FDF89967938767EE2314F10097D7FF1FD7
:1061B00083D7A722A305F10023050100A183E1B73E
:1061C00082800111996722CCD51717F4FF1F1304A1
:1061D00064532314F1008347040026CA97F4FF1F79
:1061E0009384A4622305F10083D704002800954519
:1061F000A305F100A18306CE2306F100970000005D
:10620000E780A0D103D604008345040017B5010040
:106210001305C5A997900100E780608CF2406244A5
:10622000D244056182809D677971D9172316F100E8
:1062300097F7FF1F83C7074D06D62307F100A9C3B1
:10624000B7E70400FC47414697E5FF1F938505FA31
:106250001305F10082976800CD4597000000E780A4
:10626000C0CB97F5FF1F83C5E54917B5010013059E
:10627000E5A697900100E7808086B2504561828054
:10628000B7E70400BC47414681451305F1008297FA
:10629000D9B745C5411106C622C4930750FA230059
:1062A000F5009307A005A300F50089472301F50039
:1062B0009147A301F5009307B003A302F50097F7F8
:1062C000FF1F9387274483C70700230205002A8402
:1062D0002303F50097E7FF1F9387970283C7070003
:1062E000414697E5FF1F938565F0A303F50097F7F7
:1062F000FF1F83D787512304F500A183A304F50072
:1063000097D7FF1F83D7670D2305F500A183A3054A
:10631000F500B7E70400FC47310582972285F14577
:1063200097000000E780C01A230EA4002181A30E6D
:10633000A400B240224441018280828079710A85A2
:1063400006D697000000E78000F50A86F94501456A
:1063500097D0FFFFE780203CB25045618280411119
:1063600022C426C24AC02A84AE843289AA858566A0
:106370000146254506C697C0FF1FE7808046A285D7
:106380002244B240CA8626860249924429454101E8
:1063900017C3FF1F6700E3440111B7C7A55A22CCFA
:1063A0009387C73317E4FF1F130494F53EC4834754
:1063B00004002C002146196506CE3EC69700000059
:1063C000E78020FA8345040017B50100130505A0F6
:1063D00097800100E780A070F240624405618280EE
:1063E0000111A146300099652D4522CC06CE97C0FB
:1063F000FF1FE780003FA24737C4A55A1304C433E8
:1064000063958702B24517B501001305658FB33553
:10641000B00097E7FF1FA385B7EE97800100E780E4
:10642000006CF2406244056182809165A1463000B3
:10643000938505F02D4597C0FF1FE780803AA2475E
:10644000E38287FC97E7FF1FA38C07EA814517B516
:1064500001001305258DD1B77971D1467000916582
:106460002D4522D406D697C0FF1FE7808037B2475C
:1064700037C4A55A1304F43563988702B7E70400BC
:10648000FC4717E5FF1F130565D641460C088297A8
:1064900017B501001305058F97800100E780007C88
:1064A000B2502254456182809165D1467000938537
:1064B00005E82D4597C0FF1FE780A032B247E38F64
:1064C00087FA17B501001305E58DF9B7C16769763D
:1064D0008146FD1705061397060141836364B700E3
:1064E0003E8582803307D50003470700B98F2147D7
:1064F00013F81700858363050800B18FC207C183B5
:106500007D171377F70F6DF78506F1B741C5A547DE
:10651000054763F2B7088347150003470500316854
:10652000A207D98F13978700A183D98FC207C18390
:106530001308C855054763900707411106C622C4D2
:1065400026C203442500914763F087049307540053
:1065500063ECF502A301C50021822302C500930468
:10656000340091C6A302D500A1822303D5002A845A
:10657000A68597000000E780A0F526942300A400DC
:106580002181A300A4000147B240224492443A85ED
:106590004101828005473A8582800111B7C7A55A1B
:1065A00022CC9387E7342A842AC621462C0015651D
:1065B00006CE3EC497000000E780A0DAA28517B59A
:1065C00001001305A58297800100E78040519700E4
:1065D0000000E780E0D6F24062440561828001114C
:1065E000A146300095652D4522CC06CE97C0FF1FF1
:1065F000E780201FA24737C4A55A1304E4346395EB
:106600008702B24517A501001305C57397D7FF1F71
:106610002395B7DCC205C18197800100E780204C3B
:10662000F2406244056182809165A1463000938505
:1066300005EE2D4597C0FF1FE780A01AA247E38211
:1066400087FCD14717D7FF1F2319F7D8D14517A5C6
:10665000010013052571C9B721C1411126C206C623
:1066600022C4AE848DC52A8497000000E78080662E
:1066700097E7FF1F83C7C7C899CB22852244B24042
:10668000A685924441011733000067008322B2407F
:106690002244924441018280828001114AC806CE80
:1066A00022CC26CA4EC693F715002E899DCBAD6726
:1066B000371700409387A7AA1CC3B7E70400BC4F55
:1066C00013060019854517D5FF1F0345E5D08297AE
:1066D00013451900F2406244D2444249B24905616F
:1066E000828093F72500638A071C17F7FF1F035763
:1066F000A711954763F9E70C014417F6FF1F13062E
:10670000A6009306300513055004130810049308DF
:10671000B00413039005930764006374F7043A848C
:10672000FD5997F4FF1F83C424FE97F7FF1F83C70B
:10673000B7FDA204DD8CAD679387B755638BF41466
:1067400063E3970AA9679387A755638EF414A2851C
:1067500017F5FF1F130545FB97000000E78000F0C9
:1067600031A2B307860083C50700639AD50483C5A9
:1067700017006396A50483C527006392050583C5AA
:106780003700639ED50283C54700639A150383C70C
:10679000570063966702A2890DE897F5FF1F83D51E
:1067A000A506B3853541C20517F5FF1F1305C5F5CD
:1067B000C1814E9597000000E78040EAE1A0050402
:1067C0004204418089BF3A84FD598547E3EB87F451
:1067D0005DC4854517F5FF1F130505F397000000FD
:1067E000E780C0E769A8B1679387C7556380F40461
:1067F000B5679387D755E39CF4F4A28517F5FF1F7F
:10680000130585F097300000E780A00A8947630FE1
:10681000F4049305E4FFC205C18117F5FF1F1305BA
:10682000C5EE97000000E780E04A89A097200000AD
:10683000E780C0F797000000E780204911C9A285D2
:1068400017F5FF1F130545EC97000000E78080480F
:106850000546A28517F5FF1F130505EB97F0FFFF0F
:10686000E780406D97200000E78040F4A68517A5DB
:1068700001001305655997800100E7804026FD5708
:10688000E39DF9F097F7FF1F239007F813452900C0
:1068900091B5A28517F5FF1F130505E797F0FFFFD8
:1068A000E780E07AE1B7A28517F5FF1F1305C5E57C
:1068B00097F0FFFFE780607B55BF93F745000145E8
:1068C000E38A07E017A501001305455597800100ED
:1068D000E780C03897300000E780402B134549001F
:1068E000D5BB411122C437E404005C5C06C63546C2
:1068F00097A501009385450317B501001305C5D180
:10690000829711E917A50100130505529780010030
:10691000E780C03401A08327041C82972A840545A0
:1069200097C00000E78000E897600100E780206DD5
:1069300097600100E780204297B00000E78080F96F
:106940002285B2402244410182804111054506C69C
:1069500022C426C297C0FFFFE780E05D1305A004B4
:1069600097B0FF1FE780A074757585457D1597C0AA
:10697000FFFFE78080477D7585451305F53697C095
:10698000FFFFE780E050371400408327840A8D45DD
:106990001305002093E707202324F40A97C0FFFF84
:1069A000E780A044B7E4040097D0FFFFE780C089E8
:1069B000C85897800100E780602A17B501001305C9
:1069C000A5C597800100E78060298327840C854551
:1069D000414593E707082324F40C97C0FFFFE780A5
:1069E000204B8D451305000897C0FFFFE780404A04
:1069F00097C0FFFFE780207737A507001305051232
:106A000097C0FFFFE780C072014597C0FFFFE78096
:106A1000E07895450545894717F7FF1F2308F7DEFE
:106A200097C0FFFFE7802079B7E700E01307000673
:106A3000238DE7403707000423A0E71097D0FFFF1E
:106A4000E78080FF97D0FFFFE7808011970000006C
:106A5000E78060E997000000E780C0989700000099
:106A6000E78020B897E0FFFFE780A0F397000000E1
:106A7000E780802797000000E780801083A7040844
:106A8000170500001305A5C1829797D7FF1F23851F
:106A9000A794BC4C130600648545829797C0FF1FDE
:106AA000E780009501458280AD67371700409387E6
:106AB000A7AA1CC3B7E700E03707400023A0E718E8
:106AC00001000100B7F7070003C70701A5476316D8
:106AD000F7009397450191C301A04111AE8601468D
:106AE000AA85254506C697C0FF1FE78080CFB24024
:106AF000B7E700E03707400023A0E710410182809C
:106B00004111B2862E86AA852D4506C697C0FF1F65
:106B1000E78020CDB2400145410182809307000407
:106B200063ECC7041D71A2CC2A840808A6CACAC88F
:106B300086CE32C697800100E78000EFAD67371739
:106B400000409387A7AA1CC3B7E400E037094000C0
:106B500023A0241901000100B2461008A28529458E
:106B600097C0FF1FE780E0C7F640664423A02411CA
:106B7000D6444649256182803955828041110D6590
:106B80008D4506C697C0FFFFE7802026B717004057
:106B90008D6623A6D70A17F5FF1F130565C7138750
:106BA000C70A9387870A1CC15CC5856689675CC96B
:106BB00058C114C518C9B7E70400B24003A3871E23
:106BC000410102838145B307B5008387070089E748
:106BD00017230000670023C48505C205C181E5B7FE
:106BE00097A701009387473E1357C5003E97034779
:106BF0000700011106CE2304E100135785003D8BE9
:106C00003E970347070023060100A304E100135742
:106C100045003D8B3D893E97AA970347070083C7F0
:106C2000070028002305E100A305F10097000000FC
:106C3000E78080F9F24005618280411126C2E97740
:106C400097F4FF1F938444CD22C49387A7552E84C5
:106C50002381B4002E86AA8517F5FF1F130505CCE6
:106C600006C62390F400A381040097800100E7800A
:106C7000A0DB93052400C205C18117F5FF1F130592
:106C8000C5C997000000E780A084B38784002382F1
:106C9000A7002181A382A700930564002244B2408B
:106CA00026859244C205C181410117230000670077
:106CB00083B609C99307800263E6B7001703000093
:106CC0006700E3F7828017F5FF1F0345E5B5828073
:106CD00097F7FF1F83C707C489E7172300006700E2
:106CE00083B3828097F7FF1F83C7E7C599EF4111F0
:106CF00006C697200000E780E0A9B240854717F755
:106D0000FF1F2302F7C44101828082806307054A86
:106D10006385054A5D71CAC04EDE86C6A2C4A6C29E
:106D200052DC56DA5AD85ED662D466D26AD0B947F7
:106D30002A89AE8963F9B706394697A5010093857C
:106D4000651697800100E780C0CB31ED8347E900ED
:106D5000130710036394E702854717F7FF1F230B00
:106D6000F7BA17A501001305E51497F7FF1F239243
:106D700007BA97000000E78020E571A01307000321
:106D800017A5010013050516E395E7FE97F7FF1F0A
:106D9000238207B897F7FF1F239D07B617A50100A9
:106DA0001305C512F9B797F7FF1F83C7A7B6638707
:106DB0000722BD6AB96B938CFA55014A17FBFF1F76
:106DC000130BCBA6138CEB65938AFA6605A8B30761
:106DD000490183C6070097F7FF1F83D787B3B1E345
:106DE0009307A005639BF600854717F7FF1F231243
:106DF000F7B297F7FF1F238BD7A2050A93170A0153
:106E0000C183E3E637FDB640264496440649F2596D
:106E1000625AD25A425BB25B225C925C025D616153
:106E20008280054D639BA7039307500A639EF6007B
:106E3000894717F7FF1F231EF7AC930750FA17F780
:106E4000FF1FA305F79E55BF9307A005E387F6FA3A
:106E500097F7FF1F239F07AA4DB713871700420715
:106E6000DA9741832380D70017F6FF1F2313E6AA82
:106E70008D47E3F4E7F817F4FF1F0344549B97F79B
:106E8000FF1F83C7C79A22045D8C9307F4FFC207D4
:106E9000C1839306F00DE3EDF6FA93076400C20791
:106EA000C183E31CF7F493052400C205C18117F5E3
:106EB000FF1F1305C59797F0FFFFE7806061330759
:106EC0008B008347570003474700A207D98F17F766
:106ED000FF1F231007A46318F50E8144630CA4015F
:106EE00097F4FF1F83C4C494A20497F7FF1F83C7BE
:106EF0003794DD8C170500001305E5DB97F0FFFFE5
:106F0000E780000163878407636D9C029387EB55DC
:106F10006382F40497F7FF1F83C78791054763894E
:106F2000E70681CB1387A7051377F70F8D4663F22A
:106F3000E6081307F0072300E100A300F1008945EC
:106F40009DA063829405E39754FD97F0FFFFE780CF
:106F5000C02D11A8A28517F5FF1F1305658D97F0A9
:106F6000FFFFE7808011014597F0FFFFE78040FABF
:106F700069B5A28517F5FF1F1305858B97F0FFFFF5
:106F8000E780401BCDB797F0FFFFE780C023E1BF4C
:106F9000930710F8130511002300F10097F0FFFF8D
:106FA000E780602FFD450A8597000000E78020C933
:106FB0005DBFA28517F5FF1F1305858797F0FFFFBB
:106FC000E780A0CB4DB79307F00789450A852310CA
:106FD000F10097000000E78080C605B5BD4763F863
:106FE0003717414697A50100938505F24A8597809A
:106FF0000100E78000A1631C051417A5010013051B
:10700000E5F197000000E78020BC17E5FF1F03555E
:10701000C57F97000000E780E0BC97E7FF1F83C7AC
:10702000676E17A501001305E5E689E717A50100BE
:107030001305C5E697000000E78000B917A5010019
:10704000130545EF97000000E78000B817C5FF1F44
:107050000355453697000000E780C0B817A501002A
:10706000130585ED97000000E78000B617C5FF1FE8
:107070000355A53697000000E780C0B617A50100AC
:10708000130505EC97000000E78000B417D5FF1F3B
:107090000355650F97000000E780C0B417A50100F5
:1070A000130585EA97000000E78000B217D5FF1F9F
:1070B0000355250D97000000E780C0B217A5010019
:1070C000130505E997000000E78000B017D5FF1F02
:1070D0000355450B97000000E780C0B017A50100DD
:1070E000130545E797000000E78000AE17C5FF1FB6
:1070F0000355051D97000000E780C0AE17A50100ED
:107100001305C5E597000000E78000AC97D7FF1F87
:1071100083C7C70DA20717D5FF1F0345350D5D8D2A
:1071200097000000E78000AC97D7FF1F83C7270CAC
:10713000A20717D5FF1F0345950B5D8D9700000033
:10714000E78040AA17950100130585551DB1C14779
:1071500063FE3705414697A50100938565E04A85A2
:1071600097800100E780E08931E183470901130737
:107170001003639CE700854717E7FF1F2306F76AA4
:1071800017A50100130505DFEDB61307000317A5CA
:107190000100130525E1E39EE7BC97E7FF1F238568
:1071A000076817A50100130565DEE1B6CE854A859F
:1071B00097C0FFFFE780C002B9B18280411126C2AB
:1071C000AE848D4522C406C62A8497C0FFFFE7809F
:1071D00020CCB717004099C803A5C70C418D23A642
:1071E000A70CB240224492444101828003A5870C3F
:1071F000418D23A4A70CF5B783470500034715006D
:10720000A207D98FC2076177C18713072720639A26
:10721000E7008345250037050400170300006700D9
:1072200023FA828017E6FF1F130646728147B28653
:107230001303F00FA9483308F6000348080013F7BA
:10724000F70F6307A80C630668008507E39517FF2F
:107250002947B387E6002380A70097E7FF1F93879E
:10726000A76F5DA8411113D765001347170006C625
:1072700093F63500058B954791CA05469947638774
:10728000C60009469D476383C600A14713F6450023
:107290003336C00093F68503050685C2A145638B8E
:1072A000B604E145638AB604930580026388B60498
:1072B000930580036393B600914697F5FF1F2382E1
:1072C000F59097F5FF1F238DC58E97F5FF1FA389B6
:1072D000D58EBE8517A50100130505D39770010053
:1072E000E780E07FB240854717F7FF1FA30BF78CBD
:1072F000410182808546D1B78946C1B78D4675BFA9
:1073000017A501001305C5D2177301006700237D7F
:1073100017E7FF1F13074764BA972380B700E147B9
:10732000E302F5F493077002E30CF5FC82802A87F0
:1073300023800500814717E5FF1F1305256113080A
:10734000F00F2946B306F50083C606006396E602F1
:1073500097E6FF1F93864660B69783C707000545EB
:107360002380F5009947636EF7029D4763FDE700B0
:10737000E147630DF7008280638506018507E3938B
:10738000C7FC0145C5B7238005008280B7370040A0
:1073900003C7370083C7050093F70704D98F2380FD
:1073A000F50082805D7152DC56DA5ED6716A97FB19
:1073B000FF1F938B2B928D6AA6C24EDE62D486C6C7
:1073C000A2C4CAC05AD866D26AD06ECEC1495E8CF9
:1073D00097E4FF1F93840459130A0A20938A7ADCE6
:1073E00017F9FF1F03490992B3872B0183C70700D1
:1073F00093F7F70FC9EFB787004003C76700058B06
:10740000E310077C03C76700118BE30D077E83C77A
:107410005700918B99E36F10200317F7FF1F034765
:10742000878E85476304F7006F10400197E7FF1FC1
:10743000A389E77897E7FF1F2386075E97E7FF1F7B
:107440002384076A97E7FF1F2382077697E7FF1FCA
:10745000238F077497E7FF1FA386075C97E7FF1F3B
:10746000A384076897E7FF1FA382077497E7FF1FAE
:10747000A38F077297E7FF1FA386077497F7FF1F75
:10748000A3830788B787004011476F007077930781
:10749000190093F7F70F3D476364F70617F7FF1FCF
:1074A0002302F78697F7FF1F9387C784CA9783C77E
:1074B00007001307100293F7F703638EE71E636656
:1074C000F70405446385871CE38C07620947638ED4
:1074D000E71013070002E384E74EB7E700E0370741
:1074E000400023A0E7180100010062992300090071
:1074F000FD1923A0E71093F9F90FE39309EEE5BD19
:1075000097F7FF1F2380078071BF1307300263883E
:10751000E70C63E8E71613074002638CE70A1307DA
:107520000003E39CE7FA97E7FF1F9387A77BCA97BF
:1075300003C70700A1471377F70FE31BF71483C7AF
:10754000640097E6FF1F2385F66697E7FF1F83C752
:10755000D74191C7FD5797E6FF1F238BF66497E548
:10756000FF1F83C5354097E7FF1FA383B76497E7E5
:10757000FF1F83C7273F13FB07089306000493F7F9
:107580000706639FD74C9307A009638DF51663EA3E
:10759000B7129307F0056386F54A93075009638491
:1075A000F52A014497E7FF1F83C797601547E392C9
:1075B000E736B7E700E03707400023A0E7180100EF
:1075C0000100B786004023808602130680FC6F000E
:1075D000500EFD5717E7FF1F230BF75CFDBDFD574E
:1075E00017E7FF1F2304F75CCDBD17A501001305A6
:1075F000A5B597700100E780606697E7FF1F938746
:10760000676ECA9703C40700014B97ECFF1F938C6A
:10761000EC4D1374F40F17AD0100130D6DB36347F8
:107620008B04294597700100E7804050854717E794
:10763000FF1FA30BF74A17E7FF1F2308874A17E727
:10764000FF1F2301F75837E700E0B706400023206B
:10765000D71801000100378600408347A60293F740
:10766000370F2305F6022320D71085BDB3876C01A1
:1076700083C507006A85050B97700100E7802046E7
:1076800079BF854717E7FF1F2300F746B9B517E70E
:10769000FF1F130727654A970347070097E6FF1F59
:1076A000A382F63897E6FF1F238FE63617E7FF1F02
:1076B000230AF7501DB5854717E7FF1F2304F73648
:1076C00029BD9307400A6389F5349307200B63842F
:1076D000F5369307100AE396F5EC838724000144FE
:1076E000E3D207EC97E7FF1F83C7F72793F637002E
:1076F000638A061A0546638AC62209466395C61A36
:107700001D4755A217E5FF1F0345E525C94797EC1F
:10771000FF1F83CC5C2597E5FF1F83C5E52417E495
:10772000FF1F034474246315F510CD476392FC10CA
:1077300093077008639CF5021307300FB7170E000C
:107740006308E4001307900DB7B704006314E4085E
:1077500017E7FF1F2324F746BE8517A50100130571
:10776000A59F97700100E780803725BD93078008AB
:10777000639DF500B307804013F4F70FB777460019
:10778000938787CDB3D78702E1B793079008639AB1
:10779000F500B307804013F4F70F91679387C7662E
:1077A000D5B79307A008639BF500B307804013F497
:1077B000F70FB7173D0093870790E9B79307B00815
:1077C000639AF500B307804013F4F70F916793872E
:1077D00097D04DBF93F5F5078D47639BF500B30731
:1077E000804013F4F70FB7975B00938707D859BF12
:1077F0008947639BF500B307804013F4F70FB77711
:107800000B009387071BBDBF8547639AF500B3073D
:10781000804013F4F70FDD67938767E3A5B7D2873E
:1078200085F9B307804093F7F70FB3D7FA020DB786
:1078300097000000E780409FA285668597000000C2
:10784000E780809EB9BB9305610017E5FF1F0345E4
:10785000851117E4FF1F0344141197000000E7800F
:1078600040AD93057100228597000000E78060AC71
:107870003C0017E7FF1F232DF744834761002304D3
:10788000F10083477100A304F100894717E7FF1F48
:107890002300F7328357810017E7FF1F2314F70CEB
:1078A000094409B3154793F64700B336D00093F760
:1078B0008703850685C32146638BC7066146638AB5
:1078C000C706130680026388C70613068003639306
:1078D000C700914717E6FF1F2304D62E97E6FF1F28
:1078E000A380F62E97E7FF1F238DE72C17E7FF1FD6
:1078F000034787079376070497E7FF1F83C7D706D9
:107900008DEE1377770C93067008630CD70213770C
:10791000F7078D466312D70CB307F040B7955B00AD
:1079200093F7F70F938505D849A81947ADBF854749
:1079300055B7894745B78D4771BF930670086311E6
:10794000D7021307300FB7150E006389E70213073C
:10795000900DB7B504006383E7021307700845BFB5
:107960009306800C6311D702B307F040B775460049
:1079700013F7F70F938785CDB3D5E70297E7FF1F7E
:1079800023AEB722D9BB9306900C631CD700B30774
:10799000F04093F5F70F91679387C766B3D5B702A9
:1079A000F1BF9306A00C631DD700B307F040B715D5
:1079B0003D0093F7F70F93850590B3D5F5027DBF92
:1079C0009306B00CE315D7F4B307F04093F5F70F27
:1079D0009167938797D0D9B78946631BD700B307C0
:1079E000F040B7750B0093F7F70F9385051BF1B7C0
:1079F0008546631AD700B307F040DD6593F7F70FAC
:107A0000938565E35DBFD28535FBB305F04093F503
:107A1000F50FB3D5BA029DB783C72400C18B99C7B0
:107A2000854717E7FF1F2308F718A5BE97E7FF1F35
:107A300023830718BDB6854717E7FF1FA303F71871
:107A40008DB63C0017E7FF1F2324F728094793074B
:107A500000032314F10097E6FF1F238BE6142DBDCE
:107A600063940756A94763E5B742179701001307C8
:107A7000E7568A05BA959C41BA97828717E4FF1F9B
:107A8000034474EE894C6306940D63E68C068547C7
:107A90006303F4089307F00F17E7FF1F034747112D
:107AA00063F6E70017E7FF1F2304F71097ECFF1FAB
:107AB00083CC0C109307000413F4FC0F63F49701BC
:107AC0001304000497E7FF1F9387872003AD070087
:107AD00022862685EA85B38C8C40229D9770010012
:107AE000E78080F497E7FF1F2384970D97E7FF1F38
:107AF00023A0A71F45BC8D47630CF40A9947E31BDD
:107B0000F4F8979701009387E75317E7FF1F2321A6
:107B1000F71CA94751B717E7FF1F0347C71E97E791
:107B2000FF1F9387E70A4946979501009385855A79
:107B300063068700979501009385C5553E8597702C
:107B40000100E78060EE17E7FF1F2323A718C9474E
:107B5000A1B797E6FF1F83C6061B054797E7FF1FE0
:107B6000938707076394E6023E8513067002979594
:107B700001009385A55397700100E780E0EA17E7BD
:107B8000FF1F2327A7149307700239B73E851306FA
:107B90003004979501009385A54B97700100E7800D
:107BA000A0E817E7FF1F2325A71293073004EDB5C0
:107BB00097E5FF1F83C525DB179501001305055BBE
:107BC00097700100E780A0F1054D97EDFF1F83CD71
:107BD0008D1397E5FF1F83C505D917950100130580
:107BE000E5586398AD0B97700100E78040EF97E789
:107BF000FF1F83C747D7B5CBE36EF4E817940100A6
:107C000013048451638CB701179401001304445189
:107C1000638697011794010013040452228597701C
:107C20000100E780E0041375F50F93071500860740
:107C300017E7FF1F230EF7F88D4717E7FF1FA3096C
:107C4000F7F897E7FF1F9387A7F80147BE861376DB
:107C5000F70F89076365A60297E7FF1F23AAD706D8
:107C600097E7FF1F83C7C7F605BD97970100938766
:107C7000A74317E7FF1F232DF704914731BD3306B4
:107C8000E40003460600A380070005072380C70021
:107C90007DBF97700100E78080E497E7FF1F83C7EF
:107CA00087CCE1D7E368F4DE179401001304C443E2
:107CB000638CA70117940100130484436386970122
:107CC0001794010013044444228597700100E78053
:107CD00020FA1375F50F93071500860717E7FF1FA6
:107CE0002308F7EE8D4717E7FF1FA303F7EE97E78B
:107CF000FF1F9387E7ED0147BE861376F70F8907CD
:107D0000E37CA6F43306E40003460600A3800700E4
:107D100005072380C700D5B797E5FF1F83C5A5C416
:107D2000179501001305454597700100E78020DB9A
:107D300097E7FF1F83C797E993E7470017E7FF1F00
:107D4000A306F7E883C7240017E7FF1FA30EF7E693
:107D500089B8179501001305654397700100E78006
:107D6000E0EF97E7FF1F938727E683C7070017E732
:107D7000FF1F2309F7BE17E4FF1F034464E33334F6
:107D800080000DB017950100130585419770010023
:107D9000E780C0EC97E7FF1F83C757E393E707012E
:107DA00017E7FF1FA304F7E283C7240017E7FF1FAD
:107DB000230CF7E06FF0EFFE179501001305853FE8
:107DC00097700100E78080E903C704007D8B51EFC5
:107DD000B787004003C767021377C70B13672700F5
:107DE0002383E70203C7A7021377C70B1367270094
:107DF0002385E70203C7E7021377C70B1367270042
:107E00002387E70203C727031377C70B13672700EE
:107E10002389E702854717E7FF1F2305F7C017E708
:107E2000FF1F2303F7CC17E7FF1F2301F7D817E73E
:107E3000FF1F230EF7D697E7FF1FA38507BE97E71F
:107E4000FF1FA38307CA97E7FF1FA38107D697E702
:107E5000FF1FA38E07D497E7FF1FA38507D697E7D9
:107E6000FF1FA38207EA6FF0CFF389476312F7027F
:107E700097E7FF1F83C747AF9146638CD70863E03E
:107E8000F604638EE70C6369F70A05476380E70E23
:107E9000FD5717E7FF1FA30DF7D037074000B7E7DF
:107EA00000E023A0E71801000100B7860040130698
:107EB000F0FC2381C60223A0E7106FF00FE2130746
:107EC00020086382E7086362F70213071008E39152
:107ED000E7FC378700408347670293F7C70B93E7B8
:107EE00027002303F7026FF0CFEB130730086389F5
:107EF000E70213074008E39DE7F837870040834710
:107F0000270393F7C70B93E727002309F7026FF0C6
:107F10004FE9378700408347270393F73707F5B7C3
:107F2000378700408347E70293F7C70B93E72700A3
:107F30002307F7026FF0EFE6378700408347E70239
:107F400093F73707F5B7378700408347A70293F7C2
:107F5000C70B93E727002305F7026FF08FE43787FD
:107F600000408347A70293F73707F5B737870040EC
:107F70008347670293F73707ADB7179501001305DD
:107F8000652497700100E78060CD97E7FF1F238B82
:107F9000079CD5B3179501001305C5239770010001
:107FA000E780C0CB97E7FF1F239E079A97E7FF1F45
:107FB000938707C003C40700894763F38700094418
:107FC0001374F40F6FF00FDE13070002E392E7EC77
:107FD000631B0B0A638FF500930720026383F50888
:107FE000179501001305852297700100E78020AFE7
:107FF00045B5179501001305A51E97700100E78090
:10800000E0C50144179D0100130DCD1EA14CB3879F
:10801000840083C507006A85050497700100E78026
:1080200000ACE31694FF178501001305656D97708A
:108030000100E780A0C217E4FF1F0344E49201E8B7
:1080400097E7FF1F23820790014B6FF0AFD5894759
:10805000E310F4E4854717E7FF1F2307F78E6FF05F
:108060004FD417E6FF1F0346169097E5FF1F83C501
:10807000858F179501001305651897700100E7803B
:1080800000A66FF00FD26380F50693071002E39904
:10809000F5F497E5FF1F83C5258D1795010013059E
:1080A000E51797700100E78080A397E7FF1F23A1E2
:1080B00097C297E7FF1F938767B0944383D7470022
:1080C00017E7FF1F0347E7AF17E6FF1F232CD688EC
:1080D0001D4497E6FF1F2399F68897E7FF1F238625
:1080E000E7886FF02FCC97E5FF1F83C5E5871795CD
:1080F00001001305251497700100E780409E97E763
:10810000FF1F2383078497E7FF1F239D07846FF0DA
:108110002FF92547638FE7C8994637870040639456
:10812000D70223008702B7E700E0B706400023A08C
:10813000D71801000100130600FC2301C70223A089
:10814000D7106FF08FB99306100A639FD7002300F2
:108150008702B7E700E0B706400023A0D718010068
:108160000100130680FCD1BF9306A009E381D7FE6E
:108170009306400AE38DD7FC93062002639DD70047
:10818000B7E700E0B706400023A0D71801000100C0
:1081900023008702F9B78546E384D7FE93070008DA
:1081A000E300FBFEB7E700E0B706400023A0D718C6
:1081B00001000100130620FC23008702BDBF17E762
:1081C000FF1F0347F79E6302F71E63E7E702954729
:1081D0006300F7109947630AF704B78600402380CD
:1081E0000602B7E700E03707400023A0E7180100C8
:1081F00001001306A0FC75B99307F005630AF700A8
:10820000930750096306F70093071002E317F7FC82
:10821000B7E700E03707400023A0E718010001009E
:10822000B7860040130620FC69B117EBFF1F034B14
:108230002B98930700045A8D63F46701130D000413
:1082400097E7FF1F9387C7A883AC07001374FD0F40
:108250002286E685268597600100E780E07CB307EB
:108260008B40669417E7FF1F2304F79497E7FF1FDF
:1082700023A087A6B7870040630C0B022380A703C7
:10828000B7E600E03706400023A0C6180100010051
:1082900003C72702134707042381E70203C7270206
:1082A0001377C70F2381E70223A0C6106FF0EFA258
:1082B0002380070237E700E0B70640002320D718E5
:1082C00001000100130620FC2381C7026FF0AFB943
:1082D000378700408347370097E6FF1F83C6D68E57
:1082E00093F70708D58FA301F700B7064000B7E75B
:1082F00000E023A0D718010001001306A0FC35BD43
:1083000097E7FF1F9387079ECA9783C7070093F7D6
:10831000F70FC1CF97E7FF1F83C7E79ED9E717E79E
:10832000FF1F0347F788930700026310F70883AD28
:10833000040017DDFF1F034D2D6397DCFF1F83CC67
:10834000BC6217DBFF1F034B4B62E6876A87DA8646
:108350006E8697D5FF1F83C5255F1795010013050E
:10836000E5EE97600100E780807797E7FF1F23A77E
:10837000B78597E7FF1F2385A78597E7FF1FA38191
:10838000978597E7FF1F238E678397D7FF1FA38CDF
:10839000875AB7E700E03707400023A0E71801003D
:1083A0000100B78600406FF04FA2B7E700E0370743
:1083B000400023A0E71801000100B786004015BD6A
:1083C00097E6FF1F83C626940547639CE60429476A
:1083D0002381E70209472383E7022385E70297D732
:1083E000FF1FA381077E97E7FF1FA38E0790B78724
:1083F0000040A381070017D7FF1FA307077C05478D
:108400002383E700B640264496440649F259625A4F
:10841000D25A425BB25B225C925C025DF24D6161BA
:10842000828029472381E70209472383E7022385C6
:10843000E7022387E7022389E70255B717D7FF1F13
:10844000A303F7506FE01FFF854717D7FF1F230BCC
:10845000F75C17D7FF1F2309F76817D7FF1F2307FC
:10846000F77417D7FF1F2304F7746FE0BFFE85472B
:1084700017D7FF1F2308F75A17D7FF1F2306F766E2
:1084800017D7FF1F2304F77217D7FF1F2301F772B7
:1084900017D7FF1FA308075817D7FF1FA3060764A6
:1084A00017D7FF1FA304077097D7FF1FA38107707B
:1084B0008280411106C697000000E78080FBB787E5
:1084C000004023800700130740FC2386E7001307C2
:1084D000C004A386E70017D7FF1F1307A7482398F8
:1084E000E70017D7FF1F1307E74B239AE70017D7BB
:1084F000FF1F13076757239CE70017D7FF1F1307BA
:10850000E762239EE70029472381E7020947238387
:10851000E7022385E7022387E7022389E702A38195
:108520000700930600F8A380D700930690022380EB
:10853000D700FD562383D7002381E700930600056B
:1085400037E700E0230BD740B70640002320D710C1
:1085500003C7170013671700A380E700B24097D73F
:10856000FF1F2393076641018280411106C69700D1
:108570000000E78000F0B787004023800700130762
:1085800000FC2386E7003147A386E70017D7FF1FCB
:108590001307473D2398E70017D7FF1F13078740AE
:1085A000239AE70017D7FF1F1307074C239CE70008
:1085B00029472381E70209472383E7022385E7024E
:1085C000A3810700930600F8A380D70093069002CA
:1085D0002380D700FD562383D7002381E70093062D
:1085E000000537E700E0230BD740B7064000232003
:1085F000D71003C7170013671700A380E700B24026
:1086000097D7FF1F2392075C41018280F167938710
:10861000072017D7FF1F2323F75A854717D7FF1FB8
:108620002310F75AA14717D7FF1F230CF75897D7E6
:10863000FF1FA388075897D7FF1F2385075897D791
:10864000FF1F2383073097D7FF1FA38E072E814775
:1086500017D5FF1F1305852FFD5517D6FF1F1306CE
:10866000A62F2947B306F5002380B600B306F6000F
:10867000238006008507E397E7FE97D7FF1FA38AAD
:10868000075297D7FF1FA388075297D7FF1F23834F
:10869000075297D7FF1F238E075097D7FF1F238DB1
:1086A000075097D7FF1FA387075097D7FF1F238433
:1086B0000750814717D6FF1F1306C6614147B3060F
:1086C000F600238006008507E39BE7FE828017D72C
:1086D000FF1F0347476385476316F7001703000032
:1086E0006700E3E8170300006700E3DC411122C4E0
:1086F00006C617D7FF1F0347076185472E8613F469
:10870000F50FAA856317F70417D5FF1F1305C539A1
:1087100097600100E780403197D7FF1F2386073C11
:10872000B787004023848702B7E600E037064000A1
:1087300023A0C6180100010003C7A7021377C70FC3
:108740002385E702B240224423A0C610014541011F
:10875000828017D5FF1F1305E52897600100E78089
:10876000A02C97D7FF1F238F072AB78700402382AB
:108770008702B7E600E03706400023A0C6180100D4
:10878000010003C767021377C70F2383E7025DBFAA
:10879000411106C697000000E78080E7B240410122
:1087A000170300006700E3F2411106C697F0FFFFD0
:1087B000E78080BF97D7FF1F83C7D726A1CB97D568
:1087C000FF1F83C5452689C917D5FF1F1305C5257A
:1087D00097E0FFFFE780C05397D7FF1FA3840724CC
:1087E00097D7FF1F2380073E37E700E0B70640001A
:1087F0002320D71801000100378600408347660216
:1088000093F7370F2303F6022320D710B24041011C
:10881000828041C9D9C597D7FF1F83C7E73AD1C323
:10882000011122CC4AC84EC656C25AC006CE26CA2C
:1088300052C42E89AA890144930A0004371B0300FD
:1088400063772403B3078940C207C183BE8463F4FE
:10885000FA0093040004C204C180130A1BD497D702
:10886000FF1F83C7271C9DE37D1A631C0A00F2408B
:108870006244D2444249B249224A924A024B0561BB
:10888000828097F0FFFFE78020B2D1BF3385890057
:108890002694A685420497000000E78060E54180A9
:1088A00045B7828097D7FF1F9387874918429C431B
:1088B00083D645000345070083C5C700035646001D
:1088C0006396A50083D5E700638DD502011106CE1E
:1088D0002386A7002397D700B705CF00DC4B9385ED
:1088E000757D05077D162EC2230001003AC42316AC
:1088F000C1002317D10099C30A858297F240056110
:1089000082808280DC4DDC4B81CFB7E7040090454C
:1089100003A38705914517D5FF1F0345A542028391
:1089200082806D713C083EC6B707E5002322911096
:108930003EC8AA843C083285232611103ECA23244F
:108940008110232021112E8997300000E780806359
:108950002A84979501009385E59217750100130508
:10896000657797600100E7808017A2851795010061
:108970001305C5A197600100E7806016294597603F
:108980000100E780A01AB705CB009385757D6800CC
:1089900097100000E7800069A2856800973000000A
:1089A000E780A050014781467000CA852685972040
:1089B0000000E780808C05CD2A849795010093857F
:1089C000658C177501001305E57097600100E7805D
:1089D0000011A285179501001305059C9760010001
:1089E000E780E00F294597600100E780201483208D
:1089F000C110032481108324411003290110516107
:108A0000828097D7FF1F9387A73318429C437971C1
:108A100022D406D60348070083C807012A8483D6D8
:108A20004500035546006396080183D82701638DEE
:108A3000D8022388070105072399D7003708CC00FF
:108A4000DC4B1308787D3ACC1307F5FF42CA2308A4
:108A50000100231EE100231FD10099C7080832C678
:108A60002EC482973246A245228597000000E780F7
:108A700080EBB2502254456182806D713C083EC04B
:108A8000B707E5003EC23C083EC42326111023244C
:108A900081102322911023170100231801002319AC
:108AA0000100231A0100231B010097B7FF1F83D782
:108AB000279599E3C167FD172316F10097B7FF1FAC
:108AC00083D7279491EB97D7FF1F938767279C4302
:108AD0009C43DC4783D7070017B4FF1F130444925D
:108AE000584C2317F10083574400484B2318F100DA
:108AF00031E1978501009385E57F17750100130526
:108B0000655D97600100E78080FD17850100130512
:108B1000A57F97600100E78080FC294597600100F0
:108B2000E780C0008320C1100324811083244110FA
:108B30005161828097B7FF1F83C7F78C89EBB7E736
:108B40000400BC5782975C4C23AA0700E1BFFD17C5
:108B500097B6FF1FA389F68A0356070183470401CE
:108B60004C470A85230BF10097300000E780003165
:108B700097D7FF1F9387C71C9C43014781468843B3
:108B80000A866C0097100000E780206FAA8429C134
:108B900097850100938505761775010013058553A8
:108BA00097600100E780A0F3A685178501001305F3
:108BB000657697600100E78080F2294597600100A3
:108BC000E780C0F6584CB7E70400BC57484B9DBF40
:108BD00097B7FF1F83C73783F5D7B7E70400BC4FAC
:108BE0001044854517D5FF1F0345C51582971DBF46
:108BF0005C4EDC4BB9CFB1CD411122C417750100D9
:108C00001305454D2E84978501009385E56C06C6B6
:108C100097600100E780A0ECA2851785010013058D
:108C2000257297600100E78080EB2945976001007D
:108C3000E780C0EFB7E704002244B24003A38705F2
:108C400017D5FF1F03450510130640069145410146
:108C500002838280411122C417A4FF1F13040478E9
:108C60001C4C06C689C7DC4399C34C488297584CB4
:108C7000B7E70400BC57484B82975C4CB240224493
:108C800023AA07004101828017A7FF1F1307077758
:108C9000834707009306F00B850793F7F70F63E907
:108CA000F60097A6FF1F238BF6740345070082800A
:108CB000930700F8FDB7835745006386071001113D
:108CC0004AC817A9FF1F1309A97352C4032AC9016F
:108CD00006CE22CC03274A0126CA4EC656C2F157F9
:108CE00035E31307D00DFD57636EC704B7E90400E1
:108CF00083A709072A841305860042054181B284AF
:108D0000AE8A8297232AAA000325C9015C49A9E7F4
:108D1000978501009385455A177501001305853B1A
:108D200097600100E780A0DB1785010013058569C6
:108D300097600100E780A0DA294597600100E7808D
:108D4000E0DEDD57F2406244D2444249B249224A51
:108D5000924A3E850561828093874400B705CF0023
:108D60002319F5009385757D310597100000E78084
:108D7000602B0325C901834564003105973000004D
:108D8000E780A0120325C9012686D68531059730D4
:108D90000000E780A00E7146A2854A859760010019
:108DA000E78080C8504419CA83A78905854517D52F
:108DB000FF1F034525F98297814769B79700000097
:108DC000E780E0CBD5BFFD573E858280411126C2AA
:108DD00097A4FF1F9384C462D84C22C437E40400D4
:108DE0003C54484B06C68297DC4C0323C4052244FE
:108DF000B240924423AA070017D5FF1F034585F40C
:108E0000854541010283411126C297D4FF1F9384F7
:108E100024F39C4006C622C44AC0D5C3DC43C5C364
:108E20005CC12300B5002A84978501009385054421
:108E3000177501001305052A97600100E78020CA15
:108E4000294597600100E78060CE9C4023A407007D
:108E500023A2070097A7FF1F93874758DC4FDC4BDF
:108E600091C7295597000000E78000DF97A7FF1FF3
:108E700093870759DC4FDC4B89C797000000E780D8
:108E800020F537E904008327C905894517D5FF1F59
:108E9000034545EB82978327C905914517D5FF1FE9
:108EA000034545EA82979C4003A3470163090300F9
:108EB00022852244B2409244024941010283B240D9
:108EC000224492440249410182800111328506CE3A
:108ED00022CC26CA2E8497300000E780A00AAA84FC
:108EE000978501009385C53B177501001305851E05
:108EF00097600100E780A0BE03078400035664006A
:108F000083554400A68617850100130565459760C3
:108F10000100E780C0BC294597600100E78000C1DF
:108F200097A7FF1F83C7E74B639D970001459700F5
:108F30000000E78060D281450A8597000000E78045
:108F4000C0ECF2406244D244056182806D712324FA
:108F50008110232611102322911093F745002E84AF
:108F6000638707143C083EC0B707E5003EC23C08D3
:108F70003EC4231701002318010023190100231AFE
:108F80000100231B010097A7FF1F83D7274599E303
:108F9000C167FD172316F10097A7FF1F83D727444A
:108FA00091EB97D7FF1F9387A7D99C439C43DC473E
:108FB00083D7070017A7FF1F130747422317F100A6
:108FC000544F835747002318F100DC4AA1E79785E7
:108FD000010093852531177501001305A50F9760D2
:108FE0000100E780C0AF178501001305E5319760E8
:108FF0000100E780C0AE294597600100E78000B31B
:10900000134544008320C1100324811083244110A0
:109010005161828097A7FF1F83C7B73C2555D9C3ED
:10902000FD1717A6FF1FA30EF63A03D606018347C6
:109030000701CC460A85230BF10097300000E7803A
:10904000E0E397D7FF1F9387A7CF9C4317A7FF1F86
:109050001307C738978601009386062E88430A8631
:109060006C0097100000E7804021AA8451D99785B1
:10907000010093852527177501001305A505976045
:109080000100E780C0A5A685178501001305852886
:1090900097600100E780A0A4294597600100E78060
:1090A000E0A8268597000000E78000BB91BF93F7FA
:1090B00025009DC7B7E70400BC4741468145280805
:1090C0008297255597000000E78000B9280893058E
:1090D000F00F97000000E78040D3134524001DB730
:1090E00093F71500014599DF97000000E78020996C
:1090F0001345140001BF5C4D411106C688C317D744
:10910000FF1F232FF7C2B7E7040083A7070817053F
:1091100000001305E5E38297B24097D7FF1F238332
:10912000A7C201454101828001113335A000A30788
:10913000A100B7E7040083A7471706CE1306F10086
:109140008545130550308297F24005618280828008
:10915000411122C406C697D7FF1F83C727C0014409
:1091600089EF97B7FF1F83C7B719054499E717B46D
:10917000FF1F0344E41813441400228597000000E5
:10918000E780C0FA178501001305C52E09E417858D
:1091900001001305252F2244B2404101176301004D
:1091A0006700E393797122D4A30F010037E4040030
:1091B0008327841726D24AD006D6AA842E8913057F
:1091C00050309305F10132C6829732468347F10150
:1091D00093150601C18185CB01452EC6970000007D
:1091E000E780C0F483274417B2454A8626858297D4
:1091F000054597000000E78060F3B2502254925476
:10920000025945618280832744174A8626858297C2
:10921000EDB741119397050122C406C626C2C18746
:109220002E8463D40702B7E40400FC5417A5FF1F83
:1092300003450520829719C1BC5482972165218D71
:10924000B240224492444101828093F715008DC7B9
:10925000B7E7040083A7471A17A6FF1F1306461C8B
:1092600097D5FF1F9385C5AE17A5FF1F0345451C66
:10927000829713451400E9B793F7250099CFB7E714
:109280000400BC4F13060064894517A5FF1F034562
:10929000251A82971345240065B793F7850085CF7B
:1092A00097D7FF1F83C747AC85E7B7E7040003A83C
:1092B000871A1307401F97A7FF1F83C767178146A9
:1092C00013064006994517D5FF1F035565A9029857
:1092D00013458400B5B793F745000145B5D3B7E40E
:1092E000040083A7041817D5FF1F035565A78297AD
:1092F000BC4C13060064914517A5FF1F0345451399
:109300008297134544002DBF97D7FF1F83D747A5EA
:109310006398A70217D7FF1F2315B7A417D7FF1FFE
:109320002312C7A417D7FF1F231FD7A22E86178586
:1093300001001305A51BBE85175301006700237AA2
:10934000178501001305051C1763010067000391D1
:109350000357450097D7FF1F83D787A0631EF704E5
:10936000C1674111F91722C417D7FF1F232AF79E9F
:1093700037E4040097D7FF1F23A6079E97D7FF1F48
:10938000A38E079C97D7FF1F2380079E7C4C06C6A1
:10939000894517A5FF1F0345A50982977C4C914578
:1093A00017A5FF1F0345C50882972244B24041011B
:1093B00017030000670003DA178501001305851401
:1093C00017630100670083897D15954763E2A71C39
:1093D00017870100130787080A053A951C410111F8
:1093E00022CC06CEBA972E848287178501001305FA
:1093F000E51197600100E7806086A1A203C7250000
:1094000099476311F7022E8597000000E78080F4EA
:10941000834564001785010013054510975001002E
:10942000E780E06B97B7FF1F238C07EC17850100DF
:10943000130585107DBF03C7250095476319F70203
:10944000C16717D7FF1F0357A791F91703D5A500C9
:109450006309F702B7E7040083A7C7178297178548
:1094600001001305650E97500100E780207F8547B6
:1094700017B7FF1F2306F7E8178501001305450FEF
:109480008DBF97D7FF1F239DA78C83D7E50097D665
:10949000FF1F2398F68C83D7050197D6FF1F2393D0
:1094A000F68C83D7250197D6FF1F239EF68A97D780
:1094B000FF1FA385078A631BE502B7E70400BC4FC3
:1094C000096613060690A14517A5FF1F034545F63B
:1094D00082970356E4008355A40017850100130505
:1094E000E50797500100E780805F51B79307700F41
:1094F0002316F100B7E7040083A7870D17A6FF1F07
:10950000034606F36C0082974DF9854717D7FF1F76
:10951000A306F7845DB71785010013052506D1BDA5
:1095200083C5250091476392F50217850100130555
:10953000650697500100E780607297000000E780A1
:1095400060C1F24062440561828099476392F502EE
:10955000228597000000E780E0DF834564001785DF
:1095600001001305A5FB97500100E7804057D1BFCC
:109570009547639AF50083471400E1F317850100CE
:1095800013058503BDB51785010013056503E1BF0C
:1095900082803757315F97A7FF1F9387A7EA13078A
:1095A00077D598C39356C500178701001307C7F0F6
:1095B000BA9683C5060093568500BD8ABA9603C63F
:1095C000060093564500BD8A3D89BA962A9783C600
:1095D000060003470700238407002383D700A383E3
:1095E000E7002382B700A382C70097A7FF1F9387D6
:1095F00067E62383B700A383C7002384D700A3842F
:10960000E7008280411106C697000000E780A0F8BD
:10961000B7E7040083A7871417A6FF1F130686E287
:10962000D54501458297B2404D4697A5FF1F9385CA
:1096300065E2130570304101170300006700C3B6EF
:1096400061712324811A37E4040083270408232648
:10965000111A2322911A2320211B232E31191705B9
:109660000000130545BB829717A9FF1F130949DCAA
:10967000994785442300A900231CF1009785010028
:10968000938585E29307400617750100130585A4AD
:10969000231CF1082308910097C9FF1F9389E9163D
:1096A00097500100E780A04383D50900178501008A
:1096B000130585DE97500100E780604229459750E9
:1096C0000100E780A04603D50900896997000000E2
:1096D000E78060EC83274417100885451305503058
:1096E00082978327441717A6FF1F1306A6D6CD45DA
:1096F0001305703082978327441717A6FF1F1306A0
:1097000066D3B54513056030829783274417300828
:1097100089451305103182978327441730098945FD
:1097200013052031829783274415938509900D45B1
:109730008297832744159385099011458297A30545
:1097400091002306910002CD23080100230C0100A3
:10975000832784163009914513057040829783272B
:1097600084161306B10085451305004082978327B0
:109770008416700085451305104082978327841650
:1097800030088545130520408297832784161008EA
:109790008545130550408297832704157D55829790
:1097A000832744137D5582977D5597A0FFFFE7805F
:1097B00060EF8327440C829797A0FFFFE78020C9C2
:1097C0008327841417A6FF1F1306C6C7D545014576
:1097D000829789471306700F814528092306F100F7
:1097E0009790FFFFE780A0928D4713060008814500
:1097F0002808230CF1089790FFFFE78040919147DC
:10980000230CF100976701009387477E984383C735
:1098100047003AC8230AF10097D0FFFFE78040B223
:1098200070008545054597A0FFFFE780C0EE300931
:109830009305700F094597A0FFFFE780C0ED300842
:10984000930500080D4597A0FFFFE780C0EC1008C6
:109850009545114597A0FFFFE780E0EBC16717C76B
:10986000FF1F1307E74FF9171CC32322070017A593
:10987000FF1F1305A5BB97A0FFFFE780A0E8832784
:10988000C41D17C5FF1F1305254C82973C4803458F
:109890000900854582978320C11A0324811A8324F5
:1098A000411A0329011A8329C1195D618280C167A8
:1098B00017C8FF1F0358C84AF9176301F8083DCDC0
:1098C000B5CD011126CAB7E4040083A7841222CCC7
:1098D0002E862315B10006CE2A8401478146ED4528
:1098E000428582972AC611ED17850100130505BE32
:1098F00097500100E7808036F2406244D24405610F
:109900008280FC440356A100A28582972C0017C5D3
:10991000FF1F0355E54497A0FFFFE780A0EE69DD38
:10992000178501001305C5BB97500100E780003380
:1099300083A7C412ED45280082977DBF82800DC5A4
:10994000854717A7FF1FA30CF7AE97A7FF1F238913
:1099500007AE354697A5FF1F9385C5AD130560304B
:10996000170300006700438497A7FF1FA38907AC74
:10997000E9BF97C7FF1F83C7273FA9EFC16717C775
:10998000FF1F0357E73DF9176306F70441118547A9
:1099900022C417C7FF1F2309F73C37E404007C4C9F
:1099A00006C6A14517A5FF1F034585A88297032377
:1099B000841A2244B24097A7FF1F83C767A717C521
:1099C000FF1F0355E5391307401F8146314699456E
:1099D0004101028382806D7123248110232611109E
:1099E00023229110328401CD8947630AF502832036
:1099F000C110032481108324411051618280178596
:109A000001001305A5BCAE8497500100E780002536
:109A1000A285268597C0FFFFE78060B1C9BFB7E781
:109A20000400FC4728008297178501001305C5BA7A
:109A300097500100E78080228347810039C41307D3
:109A4000000B6380E7021387A7051377F70F8D4696
:109A500063EDE602A285280097C0FFFFE780E021C2
:109A600079B78547E3F587F88345910017750100BD
:109A700013058597B335B00097A7FF1F2382B770F2
:109A800097500100E780A0059DB703479100A2070A
:109A9000D98F35671307D7556385E7086368F702E1
:109AA0002D671307B7556387E70631671307C75557
:109AB000638AE70429671307A7556394E702A28521
:109AC000280097C0FFFFE780405A15B73967930613
:109AD000E7656381D70863E9F6001307E7556384F8
:109AE000E706A28528003DB73D679306F755638AD0
:109AF000D7061307F766E396E7FE97C0FFFFE780F8
:109B0000C072F5B50146A285280097C0FFFFE78027
:109B10006042F1BDA285280097C0FFFFE780205377
:109B2000F9B58947E3F587EC97000000E780A0E4EA
:109B30009305E4FFC205C1811305A1009790FFFFC3
:109B4000E780006A6DB5A285280097C0FFFFE78017
:109B5000C05271BDA285280097C0FFFFE780805DDD
:109B600079B597C0FFFFE780006651B5C16717C59B
:109B7000FF1F0355E51EF9176307F500B7E704005B
:109B800003A3C71702838280854717C7FF1F2307D8
:109B9000F71C014517F3FFFF670043591783FFFFC9
:109BA000E70243522A8408452E89B28919C900C1A7
:109BB000971500009385A586610597300100E78021
:109BC000200581447D5A97100000E780E03963C783
:109BD000A404814497100000E780003A63C8A404FD
:109BE00097C7FF1F938787189C43DC47B307F9404B
:109BF00091872302F400638309048327C900B30714
:109C0000F4409587A302F4001C4C89C79C4799C374
:109C1000228582971783FFFF6700034E5C441397EA
:109C200014008504BA972390470171BF1C4813970D
:109C300014008504BA972390070069BF8327890021
:109C40000547B307F4409587A302F4008357040047
:109C5000638EE7028DC309476384E7040D47E395EC
:109C6000E7FA978701009387E7E91CCC9787010003
:109C7000938747EA11A897870100938727B01CCCE8
:109C800097870100938787B05CC8BDBF97870100A5
:109C90009387C79B1CCC978701009387279CEDB7C0
:109CA000978701009387C7EA1CCC978701009387A9
:109CB00027EBD9BF95E51783FFFFE7024342004634
:109CC00018448347940075839D8B6317F7009710A2
:109CD0000000E78060B448C41783FFFF6700634259
:109CE00082801783FFFFE702E33D13893500C164DB
:109CF00042094111AA890144F11413590901054A85
:109D00002EC697100000E7802026B2456348A400C5
:109D1000014541011783FFFF6700033E83A7090048
:109D200013171400BA9783D707006388B7006394AA
:109D3000970063742A010504E1B70545D9BF17836D
:109D4000FFFFE7024337AA892E89328BB6843A8A0D
:109D5000BE8A97A00000E780C0FE71C926859720C3
:109D60000000E780C00C8D4763E7A7007D5517838F
:109D7000FFFF6700C33783DB440097100000E780D4
:109D8000A0242A8497100000E780402593077400E0
:109D900031443305850263CDA70297100000E780A8
:109DA000A02297100000E78020222A84971000004C
:109DB000E780C0229307740031443305850263C3F2
:109DC000A70497100000E78020209307450029A8EA
:109DD00097100000E7808020330585021307F017F5
:109DE0009307C017E35FA7FA2D55E3C277F9630421
:109DF0000B02D6865286A6854A8597200100E78009
:109E0000C0BDB5B797100000E780401D330585023F
:109E10009307C5FFD1BF832749001385C90083D5A8
:109E2000270097000000E78000EC61F581B76955D5
:109E30003DBF97C7FF1F239DA7F297C7FF1F9387BB
:109E4000E7F2904381470C463307F5004207418310
:109E50006393B70082805446139847008507C296E3
:109E60002390E600D5B797C7FF1F938727F09C4341
:109E700003C58700828017C5FF1F035565EF8280E9
:109E80001783FFFFE702A325C1671387D7FF630B83
:109E9000E502636AA700F1176300F5020145178325
:109EA000FFFF670003261387E7FF6302E502FD1744
:109EB0001D8D13351500E5B797500000E780602A27
:109EC0007D15C5BF97500000E780E0FED5BF9750D5
:109ED0000000E78000FDEDB71783FFFFE7022320B6
:109EE0004111AA8401442EC697100000E780C008E3
:109EF000B2456348A400014541011783FFFF670095
:109F000043209C48131514003E9583570500E385B4
:109F1000B7FE0504C9BF03485500814693F7F60F05
:109F200063E5070181473E85828058459397560037
:109F3000BA9703D727006316B70003D70700E304D7
:109F4000C7FE8506E1BF8346450001479377F70FBB
:109F500063E4D700814711A81C4513165700050775
:109F6000B29703D60700E313B6FE3E8582801783BF
:109F7000FFFFE702231593170501C18797CAFF1F4B
:109F8000938ACADE635BF00883A70A00C0479C4738
:109F900003570400198D420541816368F5000144AF
:109FA00022851783FFFF6700231512052A94CDBF72
:109FB000DC4713944900014A3E94834744006341BF
:109FC000FA02014A834754006349FA028509C2092B
:109FD00093D9090183A70A009847E3EBE9FCC1B7CD
:109FE0001C4413195A00A6853E994A859700000023
:109FF000E780C0EE05E1050AC9B75C4413195A00B1
:10A00000A6853E994A8597000000E78020ED19E17A
:10A01000050A4DBFE30C09FA61B7AA8481495DBF07
:10A020001783FFFFE702A30B1C452A8481E79307F0
:10A03000C5001CC51C44231204001CC09307F00F6C
:10A0400063EDB70093F5F50F228597200000E780B8
:10A05000C0E51783FFFF6700C30A93940501C1673A
:10A06000C18063F9F500A685228597200000E7806E
:10A07000E0E8C5B7C18193F5F50F22859720000070
:10A08000E780A0E2A685228597200000E780E0E334
:10A09000C9B797C7FF1F938767CD884382801C4548
:10A0A00099C797C7FF1F23A3A7CC014582807D5581
:10A0B000828097C7FF1F938767CB984383474500EC
:10A0C000484792073E9582801783FFFFE7022301EE
:10A0D000617100451C183EC6B70780013EC81C18B8
:10A0E0003ECA8357440002CE02D002CC231EF100A8
:10A0F000834784002A8902D22301F1023C083ED41E
:10A1000002D697000000E78000FB83570500231666
:10A11000F10297500000E78000C82307A1025C40CD
:10A1200003556400F18313F717008347F1025205CA
:10A130005181F99BD98FA307F10297100100E780A5
:10A14000207939CDAA840355050097A00000E78047
:10A1500020C083D704002AD26800231CF10083D7D3
:10A160002400231DF1001C4803D647008C43972090
:10A170000000E780A0D08347B400CA8617760100AC
:10A18000130646468117A305F4006C00481097207B
:10A190000100E78080845D611783FFFF670063F63D
:10A1A0002155D5BF1C45B1CF03C5A700894613571C
:10A1B0006500630BD7028D46630ED70285466300A8
:10A1C000D702130740063305E50203C7B700418BEA
:10A1D00015CB83C7B700BD8B3355F540828013750F
:10A1E000F5031307803EC5B709671375F503130719
:10A1F0000771D1BF372709001375F5031307077CD3
:10A20000D9B7014582801783FFFFE70243ED03A919
:10A210008500630C09048347B900AE8493F7070EE9
:10A2200085C303459900930520030D810505B305FA
:10A23000B5028844610597300100E78080AD35A004
:10A240002E8597000000E78020F62A8419CD97001C
:10A250000000E780605C8325C900B307B54063FA5E
:10A2600087002E94B305A440E9F51783FFFF67002C
:10A2700043E985457DBF1783FFFFE70243E62A8454
:10A2800003D50500011132C636C43AC22EC002CA37
:10A2900002CC02CE97A00000E78080AB82452ACA9C
:10A2A00022852ECC97000000E780E0E003570500F0
:10A2B000231EE10097500000E780E0ADA246324641
:10A2C0009247230FA10036874C08B28622850146AB
:10A2D00097000000E780E0A605611783FFFF670095
:10A2E00043E21783FFFFE70283DF61711C183EC65C
:10A2F000B70780013EC81C183ECA3C0800453ED442
:10A30000AA8402CC02CE02D002D202D6970000006C
:10A31000E78060DA8357050035592316F10297501C
:10A320000000E78040A72307A10209C48357440027
:10A3300081EB21594A855D611783FFFF670063DC6C
:10A34000035564005205518197100100E780405881
:10A350002A8965D18347B40093F7070E99C713057F
:10A36000840197300100E780009D83574400231E3D
:10A37000F100834784002301F1025C40035509008A
:10A38000D98313F7070883471102231CA10093F711
:10A39000F707D98FA300F10283572900231DF1008D
:10A3A0005C40F18313F717008347F102F99BD98FC3
:10A3B000A307F10297A00000E78080992AD235D93F
:10A3C000834794006800139757008347B400FD8BC0
:10A3D000D98FA305F4001C4803D647008C4397206F
:10A3E0000000E780A0A9A687177701001307871F41
:10A3F000740005464C10268597000000E7806094A5
:10A400002A890DD98347B400A685FD8BA305F400E6
:10A4100097000000E78060DF31BF1783FFFFE7028E
:10A4200003CC832485FE2A844111268597000000F1
:10A43000E78080D7834734FF93F7070E8DCB2AC67A
:10A44000268597000000E78060C809CD834734FF68
:10A45000B245FD8BA309F4FE91C52285973001001A
:10A46000E780208B41011783FFFF670083C97DD9F7
:10A470008327C4FF2685829775F5834734FF93F7BA
:10A48000070E91C7228597300100E780C08A032517
:10A4900084FE97000000E78000E5E9B71783FFFF1F
:10A4A000E702E3C09C4141112A8903C7070089479D
:10A4B0002E84935667006380F6040D466388C604B5
:10A4C0009307F0076304F7022E8597200000E780CA
:10A4D00060ABAA848149C16B130C490097C7FF1F69
:10A4E0009387C7889C43984763E4E9044101178335
:10A4F000FFFF670083BF03D745008547E3F8E7FE0A
:10A500002E8597200000E78040ADE1B703D74500D6
:10A51000E3FEE7FC2E8597200000E780A0A6AA8432
:10A52000228597200000E78000A8C204C98C5DB78F
:10A53000DC470355A900139A49003E9A9317050179
:10A54000C187635DF00083570A006397A70263E742
:10A5500074038327CA00034D5A002DA0A167216709
:10A56000A98F1307F7EFE374F7FE639709009700CD
:10A570000000E780209161FD85098DB783278A005F
:10A58000034D4A00835DA90003576900216A138BBC
:10A59000C7003AC6814A33CA4D01631E5D0197B7B1
:10A5A000FF1F9387277D9C43E1DBA286628681455E
:10A5B00026858297D1B7A1679387F7EF930C4BFF5E
:10A5C00063F24703B2455A8597F0FFFFE780A07119
:10A5D0000DC103278B00104709CE10436382C402CC
:10A5E0003107D5BFEE85668597000000E780008FB4
:10A5F00071F993861A0093FAF60F130B0B0271BFD1
:10A60000835644005C43E3E9F6F622853AC6972078
:10A610000000E7802081A1679387D7042A8A035D21
:10A620004400324763E897008347D90093E707F86F
:10A63000A306F9001C4766852286E2858297C167DA
:10A640000844FD17337AFA00529508C02312A4017A
:10A6500025B797B7FF1F938767719843814715C345
:10A660001447814763FFD500939745004C47BE953B
:10A6700019C903C7550081476375E600DC45160616
:10A68000B2973E85828003C745008147E37BE6FEA3
:10A6900016069C45F5B71783FFFFE702A3A2AA8918
:10A6A0002E8A814497BAFF1F938A4A6C83A70A00B7
:10A6B000984763E6E4001783FFFF6700E3A3DC47E6
:10A6C0001394440001493E9413BB14008347440093
:10A6D000634BF900014913BB140083475400634FD7
:10A6E000F9008504E1B70844931759005287DA86C8
:10A6F0000146A2853E9582990509C9BF4844931732
:10A7000059005287DA860546A2853E958299050949
:10A71000E9B71783FFFFE702839C814517F5FFFF29
:10A720001305054897B7FF1F23940764970000009F
:10A73000E780A0F61783FFFF6700A39C97B7FF1F72
:10A740009387C7629C4395C31783FFFFE702239952
:10A75000814517F5FFFF1305A54497000000E7802A
:10A76000C0F31783FFFF6700C39982801783FFFF41
:10A77000E702439537E4040083278412411123152F
:10A78000E100AE893289368A3A8681460147ED4535
:10A79000AA8482972AC621C90356A100D285974070
:10A7A0000100E78060288327C413CE852685829721
:10A7B000058905C98327440D2314210101462C0076
:10A7C000268582972A8401C9B7E7040083A7C712A8
:10A7D000ED4528008297228541011783FFFF67001E
:10A7E000A3914944D5B76554FDB75C41FD175CC1E1
:10A7F00082801783FFFFE702838EB7E70400FC5FC8
:10A80000829795473305F50281450D811783FFFF38
:10A810006700238F1783FFFFE702638CB7E704000D
:10A82000FC5F829795473305F5020D811783FFFF83
:10A830006700238D1783FFFFE702638AB7E70400F1
:10A8400083A7870B0355050082971783FFFF6700D7
:10A85000438B1783FFFFE702838803550500328788
:10A86000AE861796FF1F035606C597B5FF1F938543
:10A87000A55097000000E780A0EF1783FFFF670057
:10A8800043881783FFFFE7028385B7E7040083A7A8
:10A89000C71782971783FFFF6700A3861783FFFF01
:10A8A000E702E383B7E7040083A7871397B5FF1F89
:10A8B0009385854C829701451783FFFF670063846A
:10A8C0001783FFFFE702A381B7E7040083A7C71F31
:10A8D00081451795FF1F035505BA82971783FFFF20
:10A8E000670023821773FFFFE702637FB7E7040067
:10A8F00083A7871397B5FF1F938505498297014565
:10A900001773FFFF6700E37F1773FFFFE702237DE5
:10A91000B7E7040083A7C71F81451795FF1F03559D
:10A9200085BB82971773FFFF6700A37D1773FFFF37
:10A93000E702E37A2E8597800000E78080B3978056
:10A940000000E78080F01773FFFF6700837B1773B9
:10A95000FFFFE702C37897800000E78080FA177353
:10A96000FFFF6700037A5C49E1175CC95CC5835748
:10A970002501A1072319F50083570501A107231815
:10A98000F5008280F1473305F50297B7FF1F9387E3
:10A99000A7419C433E9582808D476315F60803D7F7
:10A9A0004600854763F0E7081773FFFFE70223734C
:10A9B000368536842E8997100000E780A05C29C96F
:10A9C0008357440093140501C18063E397042285F3
:10A9D00097100000E780005BFD142312940093079A
:10A9E000A0026300F5029307B0026307F502930724
:10A9F0009002631FF500228597000100E7806089BF
:10AA000001A80146CA85228597A00000E78000B40E
:10AA10001773FFFF6700E36E228597100000E78041
:10AA20006007FDB7828097B6FF1F938626389C4249
:10AA3000014599CF9843D44217B6FF1F2328E63625
:10AA40006396D70097B6FF1F23A4E6361385C7FE8B
:10AA500082801773FFFFE702836897000000E7809A
:10AA6000A04B714433058502914597900000E78023
:10AA7000C0EC11E565551773FFFF6700836897B752
:10AA8000FF1F23A1A73297000000E780E0483305AD
:10AA90008502914597900000E78020EA61DD97B735
:10AAA000FF1F23A3A73097000000E780E04697B779
:10AAB000FF1F2393A72E97000000E780E04597B77C
:10AAC000FF1F239CA72C977701009387E7B617B742
:10AAD000FF1F2327F72C97070000938707E917B775
:10AAE000FF1F232DF72A014579B71773FFFFE702F0
:10AAF000035FAA8517B5FF1F1305052A97100000ED
:10AB0000E780605F1773FFFF6700A35F1773FFFFA6
:10AB1000E702E35C97000000E78060FD971000000B
:10AB2000E780E05E97B7FF1F938747289C4391CF4C
:10AB30001387C7FE19CB83D5C7FF17B5FF1F1305B2
:10AB4000652797200100E780C01C1773FFFF67008F
:10AB5000435B1773FFFFE702835897000000E7800D
:10AB6000C0EC09CD834785002A8493F7070499EB4D
:10AB70000355E50097000000E78080F91773FFFF99
:10AB8000670023588347C5009304450117B9FF1F89
:10AB90001309C92185E3832709005CC997B7FF1F03
:10ABA00023A6972083274900F1FB97B7FF1F23A116
:10ABB0009720E9B7FD172306F5006105978000008F
:10ABC000E78060DA8307840063CB0704834784004F
:10ABD00093E707F82304F400B7E704009C5F82972B
:10ABE0004205A94741813375F5028347840093F7F5
:10ABF00007FCC98F2304F4008347D4003E951C4012
:10AC00002318A40089CF984319CB8347C400504030
:10AC1000814585073305F502420541810297832767
:10AC200009005CC897B7FF1F23A297188327490024
:10AC300089E797B7FF1F23AD97168347C4009DDFB1
:10AC40008355040117B5FF1F1305C5169720010092
:10AC5000E780200C25B71773FFFFE702434897B73B
:10AC6000FF1F9387673A9C4701448583858B85E363
:10AC7000AE84B2853A8697100000E780204F2A8480
:10AC800019C597100000E7806045829408CC2285A2
:10AC90001773FFFF6700E3461773FFFFE702834266
:10ACA00041112E8932C6AA8997000000E780C03181
:10ACB000324713060502CA86970500009385C5CC66
:10ACC00017B5FF1F1305450D97000000E780E0F85A
:10ACD0002A8425C99304C50097000000E780E0415D
:10ACE0001946AA85268597100000E780201985451A
:10ACF000268597100000E7800015177501001305E1
:10AD000065914E9583450500268597100000E780E4
:10AD1000C0195C4831468145A1075CC85CC48357B3
:10AD20002401E1172319F40083570401E1172318C4
:10AD3000F4001C4C3E859770FFFFE780403DA30464
:10AD40002501228541011773FFFF6700E33A17735E
:10AD5000FFFFE702C3384111AA842EC632C4971000
:10AD60000000E780003A004DB24522468347840048
:10AD70000CC050C093F7F70393E707042304F400D3
:10AD800023180400268597100000E78020358347AC
:10AD90009400A9462317A40013D7370005073307EB
:10ADA000D7029D8B85072306F400A306E40083C722
:10ADB0000401D8488507230FF7FE17B7FF1F1307B5
:10ADC000E7FE5843232A04009307440129E317B7F9
:10ADD000FF1F232FF7FC17B7FF1F2329F7FC17B41A
:10ADE000FF1F130424FD228597200100E780A0E4C3
:10ADF0001C44858B5D8D19E58145228597200100D6
:10AE0000E78020F141011773FFFF6700832F1CC308
:10AE100017B7FF1F232EF7F8D9B71773FFFFE70205
:10AE2000032C97050000938565B701459700000046
:10AE3000E78000B001451773FFFF6700832C17738D
:10AE4000FFFFE702C32997000000E78080B0177377
:10AE5000FFFF6700032B8347C500A5E31773FFFFC0
:10AE6000E702E3272A840355E50097000000E78006
:10AE700000C821C18347840093F7F7FB2304F40043
:10AE80001C4091C7DC4381C74C4001458297970025
:10AE90000000E78080B917B5FF1F1305A5F19720C3
:10AEA0000100E78040E90355E40097000000E780D7
:10AEB00020C61773FFFF6700C32482801773FFFF4C
:10AEC000E702E32197B7FF1F938747EE970500003E
:10AED000938565C817B5FF1F1305C5ED23A00700AF
:10AEE00023A2070097200100E78080D21773FFFF9D
:10AEF000670023211C4D91CFDC4381CF1773FFFFE7
:10AF0000E702E31D8345070082971773FFFF670081
:10AF1000431F828097B7FF1F938707EC9C4303C5AD
:10AF20000700828097B7FF1F938707EB9C4303C5F9
:10AF30001700828097B7FF1F938707EA9C4303C5DA
:10AF40002700828097B7FF1F938707E99C4303C5BB
:10AF50004700828097B7FF1F938707E89C4303C58C
:10AF60003700828097B7FF1F938707E79C4303C58D
:10AF70005700828097B7FF1F938707E69C4303C55E
:10AF80006700828097B7FF1F938707E59C4303C53F
:10AF90007700828097B7FF1F938707E49C4303C520
:10AFA0008700828097B7FF1F938707E39C4303C501
:10AFB0009700828097B7FF1F938707E29C4303C5E2
:10AFC000A700828097B7FF1F938707E19C4303C5C3
:10AFD000B70011E11D45828097B7FF1F9387C7DF38
:10AFE0009C4303C5C700828097B7FF1F9387C7DEC6
:10AFF0009C4303C5D700828097B7FF1F9387C7DDA7
:10B000009C4303C5E700828097B7FF1F9387C7DC87
:10B010009C4303D50701828097B7FF1F9387C7DB47
:10B020009C4303C52701828097B7FF1F9387C7DA28
:10B030009C4303D54701828097B7FF1F9387C7D9E9
:10B040009C4303D56701828097B7FF1F9387C7D8BA
:10B050009C4303D58701828097B7FF1F9387C7D78B
:10B060009C4303C5A701828097B7FF1F9387C7D66C
:10B070009C4303C5B701828097B7FF1F9387C7D54D
:10B080009C4303C5C701828097B7FF1F9387C7D42E
:10B090009C4303C5D701828097B7FF1F9387C7D30F
:10B0A0009C438857828097B7FF1F9387E7D29C43C2
:10B0B00003D5C702828097B7FF1F9387E7D19C43D0
:10B0C00003D5E70219E11305800C828097B7FF1FB3
:10B0D000938787D09C4303C50703828097B7FF1FE0
:10B0E000938787CF9C43C85B828097B7FF1F938766
:10B0F00027CE8843828097B7FF1F9387A7CD8843C9
:10B10000828019E17D558280F5DE984265DFFDD9A8
:10B1100017B7FF1F130747EF1847AA877155058B0D
:10B12000631D072403C507001547E37DA7FC03C77C
:10B1300037001305F0057D171377F70FE364E5FC7F
:10B1400003C35700E30003FC83C86700E38C08FADD
:10B1500003C77700494579171377F70FE364E5FADA
:10B1600003C7A70011481305F7FF1375F50FE36B2D
:10B17000A8F803CE97000D481305FEFF1375F50FD1
:10B18000E362A8F803C8B7006309080065181378DC
:10B19000F80F1305600DE36705F703C5C70079488D
:10B1A00079151375F50FE36FA8F403C8D7000D45A3
:10B1B0007D181378F80FE36705F503D80701930EA0
:10B1C00040175118420813580801E3ED0EF303C865
:10B1D000E7007D181378F80FE36605F303C827012D
:10B1E0007D181378F80FE36F05F103C88700C54E8B
:10B1F00075181378F80FE3E70EF103D86701856E31
:10B20000938EBEE06D18420813580801E3EC0EEF70
:10B2100003D847016D18420813580801E3E40EEF04
:10B2200003D887017918420813580801E36C05ED2B
:10B2300003C8A7017D181378F80FE36505ED03C572
:10B24000B7011D487D151375F50FE36DA8EA03C519
:10B25000D701714879151375F50FE365A8EA03D591
:10B26000E7011308E00F7D1542054181E36CA8E872
:10B2700003C50702494879151375F50FE364A8E87B
:10B28000C85301C937C834005915130858BFE36BB8
:10B29000A8E603A8870237C53400130555BF59181F
:10B2A000E36205E717B5FF1F2326C5B203C60501F4
:10B2B00017B5FF1F2322F5B20545E375C5E403D892
:10B2C0002501D04933760603E31E06E203C61501C5
:10B2D000E30A06E217B6FF1F232CB6AE83C527008C
:10B2E00001466387A50003C61700F1453306B60281
:10B2F00083C707039305C00272971A071307C70590
:10B3000016031A9796084697B387B70241553E979A
:10B310003297420741836362E8061773FFFFE70233
:10B3200003DC368597800000E780406C97000100C1
:10B33000E780C04B2A8497A00000E780205E2A9413
:10B3400097F00000E780002A2A9497900000E78099
:10B3500040852A9497F0FFFFE780E06F2A9497409A
:10B360000000E78000972A9497700000E78040A0D3
:10B3700022951773FFFF6700C3D882801773FFFF02
:10B38000E702E3D54111A307A10097A00000E780E1
:10B3900040C99305F100170500001305E5B597F0C6
:10B3A000FFFFE780802F014541011773FFFF670012
:10B3B00043D51773FFFFE70203D017B4FF1F130431
:10B3C000A4C40328840079599368180097B4FF1F18
:10B3D00023A014C51378180063100802BA84BE892C
:10B3E000368B328A2E89AA8A97F0FFFFE780E0A782
:10B3F0007D15269519E531594A851773FFFF6700BA
:10B4000003CF97F0FFFFE78040A67D152695A16743
:10B41000E353F5FE97B7FF1F9387C7F598433E8C1C
:10B42000814B01CB014597F00000E780C047933B7B
:10B4300015004A85DA865686D28597900000E78007
:10B4400060512A8911CD1C44F99B17B7FF1F232196
:10B45000F7BC83270C00CDD3E3800BFA829769BF3A
:10B46000268597B7FF1F23A307BA97F0FFFFE78052
:10B47000809C4146CE8517B5FF1F130565C29730E6
:10B480000100E780605A97D00000E780E09C032528
:10B49000040B97D00000E780A0A0054597D00000DE
:10B4A000E780A0A7054597000000E78060EDA9B7F9
:10B4B00097B7FF1F938747B59C47858BEDC71773D9
:10B4C000FFFFE702C3C117B5FF1F1305A5BB97B761
:10B4D000FF1F23AB07B297B7FF1F23A907B297B788
:10B4E000FF1F23A707B297200100E780C084975071
:10B4F0000000E78080F997100100E7804050971026
:10B500000100E780405697B7FF1F938767AE9C43C3
:10B5100091C7054597800000E780E02397B7FF1F9C
:10B520009387C7969C4399C741657D159770000026
:10B53000E780E0A597F00000E780804197D0000009
:10B54000E780209397B7FF1F9387C7C09C4313974B
:10B5500017016356070097F00000E780A0B097B787
:10B56000FF1F23AF07B297B7FF1F23AD07B297B7EF
:10B57000FF1F23AB07B297B7FF1F23A907B297009E
:10B580000000E780008C97000000E780A07597F02E
:10B59000FFFFE780401897F00000E780E0D91773BD
:10B5A000FFFF670003B6828097B7FF1F9387C7A589
:10B5B0008843828097B7FF1F938707A5C84382807F
:10B5C000B7E7B0009387075063E1A70297B7FF1F63
:10B5D000938787A3D843FD576367E50097B7FF1F9D
:10B5E00023A6A7A281473E858280B957EDBF177376
:10B5F000FFFFE702C3AE97800000E7806075978089
:10B600000000E780C0771773FFFF670083AF1773F1
:10B61000FFFFE70223AB2A849304140201112E8555
:10B62000B289A685214636C63A8997300100E7805F
:10B63000403D0DE9B24638082686CE8513059404B0
:10B6400097500000E780604121462C084A859730DA
:10B650000100E780003B1335150005611773FFFFFC
:10B66000670083A90145D5BF1773FFFFE70223A732
:10B670009305450617A5FF1F130545769710010092
:10B68000E78020691773FFFF6700A3A71773FFFF09
:10B69000E702E3A441112EC697F0FFFFE780C01731
:10B6A000B24588C141011773FFFF670083A5177377
:10B6B000FFFFE70223A1AA842E8497800000E78081
:10B6C000006CAA898545228597000000E780E07D0F
:10B6D00083C7E4011389940899E313890403CE8591
:10B6E000228597000000E780407C214693051902DF
:10B6F000228597000000E780607897B7FF1F938747
:10B70000A7908C43228597100000E780C0822146D5
:10B7100093858402228597000000E78020761773C6
:10B72000FFFF6700639D1773FFFFE702C39839713E
:10B7300097F00000E780E0B49305400661E9978048
:10B740000000E78000606302051497A7FF1F83C70E
:10B75000A76A13B7170097A6FF1F238FE668014457
:10B7600099CFC16417B9FF1F1309098A9309400EC5
:10B77000FD1497000000E78020836342A40A97F03D
:10B78000FFFFE78060094169B7290900096AFD7A6E
:10B790002A8B81447D199389F97B130A0A71938A54
:10B7A0008AC797000000E780208063D7A4041304B1
:10B7B000400EB387840217B7FF1F1307E7840324E3
:10B7C000070B3E948357C4016382270B184033074D
:10B7D000EB4063EAE900834744008507B3874703EA
:10B7E000D6976365F70801468145094597F0FFFF45
:10B7F000E780C04AAA8B29E597400000E780808354
:10B8000085476317F50689659385057117A5FF1FA1
:10B810001305C55C97100100E780A04F95A0B30702
:10B8200034030327090BBA9703D7C70163089700AE
:10B8300003C75700A38207002382E700050415BF52
:10B840009305C500228597000000E78080E65E85AD
:10B85000228697650100938525DD97F0FFFFE7803D
:10B86000404F5E8597100000E780608A850415BF11
:10B8700097A7FF1F938747799C478D83858BC1F7D7
:10B8800021611773FFFF67008386014685450945DF
:10B8900002D002D202D402D697F0FFFFE780004028
:10B8A000AA8479DD97F00000E780E09C1389C4004A
:10B8B0002A8481454A8597000000E780005F0C409C
:10B8C00041464A8597000000E780405B8329440099
:10B8D0006385090C4E8502D802DA02DC02DE97305D
:10B8E0000100E780E0382ACE141005462C0808181D
:10B8F0004ECC97500000E780E00A1375F50F51ED2C
:10B900008355840093E525004A8597000000E78071
:10B91000E05E11460C104A8597000000E780005653
:10B920000146976501009385A5D0268597F0FFFF16
:10B93000E7802042268597000000E780407D5C403C
:10B94000A1D3014685450D4597F0FFFFE7800035FF
:10B95000AA841DD548401389C40097300100E780B0
:10B9600020312AC64A8597000000E780404C3246C5
:10B97000636FC5004C404A8597000000E780005087
:10B9800001468145268597F0FFFFE780803C2685AC
:10B9900097000000E780A077E5B583558400ADB738
:10B9A0001763FFFFE702A37397A7FF1F9387C7657E
:10B9B0009C471DC193E7870017A5FF1F130505428C
:10B9C00017A7FF1F2326F76497100100E780403276
:10B9D0001763FFFF6700E372DD9B17A7FF1F232993
:10B9E000F76297300000E780E0647DF117A5FF1F44
:10B9F0001305C53E97100100E780E033D1BF176300
:10BA0000FFFFE702436B4169AA892E8AB28A368B0F
:10BA1000BA8B814417ACFF1F130C0C5F930C400EC4
:10BA20007D1997F0FFFFE780205863C4A40001440C
:10BA30003DA03384940383270C0B3E948357C401A9
:10BA4000638627055A87D6865286CE85130504035A
:10BA500097000000E780E0BB01C923800B0022852E
:10BA60001763FFFF6700A3688347F40185C35A8704
:10BA7000D6865286CE851305940897000000E7808D
:10BA800040B909C585472380FB00D1BF850451BF5C
:10BA9000835745006380071E1763FFFFE702836239
:10BAA00001112A8497000000E780C04D09C985472D
:10BAB0006309F50605611763FFFF6700E36397E01D
:10BAC0000000E780007C7DF5835744004947ED9BEB
:10BAD000E392E7FEC145228597000000E7804033EE
:10BAE000AA84228597000000E780204F0357440076
:10BAF00002CE91472A89631AF70022859700000039
:10BB0000E780A0513C082ACC3ECE97E00000E780B9
:10BB100080765C55C5D374084A86A685054582970C
:10BB200051BF03574400D147E3F6E7F8032A040066
:10BB3000C169014997AAFF1F938A0A4D130B400E52
:10BB4000FD1997F0FFFFE7802046634FA90E22857D
:10BB5000032A040097000000E780C042A1452A891B
:10BB6000228597000000E780A02AAA8422859700FA
:10BB70000000E780804A14402A86AA897808268532
:10BB8000CA8597000000E780C0E7AA8405D503C7EF
:10BB9000F40189476315F7008347C10181DF5546EA
:10BBA000D2851385640097300100E780E0E7014506
:10BBB00097800000E780C01901C583D7C401A5E7BD
:10BBC00097A7FF1F938747449C4793551900858982
:10BBD00013D73700058B01CF8983858B6399B70015
:10BBE00001452EC697000000E780C0DBB2454E85B8
:10BBF00097800000E780601F0346C1012A84937587
:10BC00001900268597900000E780E03935C1268528
:10BC100097800000E780E018268511C001459780D5
:10BC20000000E780004C97300000E780A040854787
:10BC3000E312F5E883C754001307F00FE38CE7E63F
:10BC40008507A382F400BDB5B304690383A70A0B7B
:10BC5000BE9483D7C401638B37015546D2851385C3
:10BC6000640097300100E780C0D955DD0509D1BDDA
:10BC70005DD86DB782801763FFFFE702A34497800A
:10BC80000000E780000C05C1C164014417A9FF1F33
:10BC9000130989379309400EFD1497F0FFFFE780E1
:10BCA000A030634EA40017A5FF1F1305251397109E
:10BCB0000100E780E0031763FFFF6700E3433305FC
:10BCC00034038327090B3E958357C501638897008A
:10BCD0002312050097800000E780A00C050475BFC3
:10BCE00097A7FF1F938747329C478D83858B8DE3F2
:10BCF0001763FFFFE702A33E17A5FF1F1305050EFD
:10BD000097100100E78020031763FFFF6700633F80
:10BD100082801763FFFFE702833C9705000093854D
:10BD2000C5A017A5FF1F1305650B97100100E7803D
:10BD300020EE1763FFFF6700C33C1763FFFFE702B6
:10BD4000033A8841B7E70400BC5B05054205418121
:10BD5000829709C585472300F50005051763FFFF96
:10BD60006700233A83C7F5FF2E858507A38FF5FE6D
:10BD7000828083C7F5FFFD1793F7F70FA38FF5FEBA
:10BD800099EF1763FFFFE7028335B7E70400BC575D
:10BD90001385F5FF82971763FFFF67008336828064
:10BDA0001C41035745008D8FBA951CC12312B50065
:10BDB0003E85828093D78500A2051441DD8D83578F
:10BDC00045001387E6FF18C189072312F50013D633
:10BDD00085004111238FB6FEA38FC6FE41018280EC
:10BDE00018419307F7FF1CC18357450085072312AD
:10BDF000F500A30FB7FE8280835745008D8F231275
:10BE0000F5001C41BE950CC12E858280AA8703D700
:10BE1000470008410D8FAA952392E7008CC38280CA
:10BE2000184108453305A7408280835745000357D2
:10BE300065001D8F1C4108453385A7403305A74089
:10BE400082801763FFFFE702832941112EC62A84EF
:10BE500097000000E780A0FDB2456373B50001A024
:10BE6000835744000840BE952312B4003E9541011B
:10BE70001763FFFF6700E3281763FFFFE70223262E
:10BE800041112E84B28532C697000000E780A0FBE6
:10BE90003246A28597300100E78000B9410117635F
:10BEA000FFFF670003261763FFFFE70243232E848B
:10BEB000854597000000E78000F92300850017639F
:10BEC000FFFF670003241763FFFFE70243214111CF
:10BED0002317B100894597000000E780C0F683472B
:10BEE000E1002300F5008347F100A300F5004101C4
:10BEF0001763FFFF6700E3201763FFFFE702231EBE
:10BF000093D78500A2054111DD8D2317B100894526
:10BF100097000000E78020F38347E1002300F5004D
:10BF20008347F100A300F50041011763FFFF67009D
:10BF3000431D1763FFFFE702831A1397850193D709
:10BF40008501C166938606F0D98F13D78500758F5A
:10BF5000D98FA2053707FF00F98D4111DD8D2EC65F
:10BF6000914597000000E78000EE6C001146973085
:10BF70000100E78060AB41011763FFFF67006318B2
:10BF80001763FFFFE702A3151C41854503C40700A3
:10BF900097000000E78080E622851763FFFF6700B7
:10BFA00043161763FFFFE70283131C4141118945C4
:10BFB00003C7070083C717002307E100A307F100A9
:10BFC00097000000E78080E30355E100410117631B
:10BFD000FFFF670003131763FFFFE70243101C41D5
:10BFE0004111894503C7070083C717002307E100F4
:10BFF000A307F10097000000E78040E08357E100CD
:10C00000410113D58700A2075D8D42054181176369
:10C01000FFFF6700030F1763FFFFE702430C0C41AC
:10C0200041112A841146680097300100E780C09FC3
:10C030009145228597000000E78040DCB247C16649
:10C04000938606F01397870113D58701598D13D76F
:10C050008700758F598DA2073707FF00F98F5D8D17
:10C0600041011763FFFF6700C3091C45BE950CC162
:10C070008280AE87944391E6584101EF0CC15CC1C8
:10C08000828003C7570013671700A382E700B687B3
:10C09000D5B70CC3EDB7AA87084119CD1841D443D1
:10C0A00098C36313D500D8C32A87034657009376F5
:10C0B000160081E6232007008280944381CA8C42C7
:10C0C00003A847008CC363930601CCC3799A14C3B9
:10C0D000A302C7003687D1BF1C45DC471D8DB7774B
:10C0E000DBB6938777DB09853305F502420541818D
:10C0F0008280F147B385F50248452E9582808347BB
:10C10000450085072302F50082801763FFFFE702E1
:10C1100003FD2A8409E41763FFFF670083FE83475A
:10C120004400F5DBFD1793F7F70F2302F400E5F762
:10C130001C4403D7270005072391E700DC4399C37C
:10C14000228582974C4889CD83475400898B99E793
:10C150001C4422859C479C439C478297232A0400C9
:10C160000040232004007DB71763FFFFE70223F799
:10C170008357250041112EC681EB014422854101E0
:10C180001763FFFF6700E3F7035705008147F14698
:10C19000E305F7FEB385D702404585072E94834516
:10C1A000440008C4F5F5B247AA8481E7232A0400B5
:10C1B00009A81C456C0022859C439C43829748C873
:10C1C0004DDD85472312F400B247232004002318D5
:10C1D00004002319F4005C485CC483D72400FD17D5
:10C1E0002391F40061BF1763FFFFE70243EF97A7B6
:10C1F000FF1F9387A7C0884323260500232405003B
:10C20000410597100100E78000B31763FFFF670047
:10C2100043EF1763FFFFE70283EC17A4FF1F13042C
:10C22000E4BD1C40411199CF9C472300B5002AC6AC
:10C230005CC197000000E78040FB1C40DC4399C3D1
:10C240003245829741011763FFFF670083EB034785
:10C25000450029E3584DAA877D551DCF1763FFFF81
:10C26000E702E3E71CC3DC4797A6FF1F23A8E6B855
:10C27000F156130507012390D70097050000938519
:10C28000050297100100E780A09801451763FFFFA2
:10C29000670023E77D55828082801763FFFFE702F6
:10C2A00003E401116146814528009760FFFFE780A4
:10C2B00000E697A7FF1F938767B49C432800930568
:10C2C000F00FDC473EC697000000E780C0F4056130
:10C2D0001763FFFF6700E3E297A7FF1F938707B28B
:10C2E0009C43D847A1679387C702631EF70A397139
:10C2F00006DE22DC26DA80004AD84ED652D456D248
:10C300003285B28497000000E780C0C7AA892685DD
:10C3100097000000E78020C92318A4FC2685970019
:10C320000000E78040C82319A4FC26859700000080
:10C33000E78060C783D744000A8A231AA4FC858358
:10C3400093F7F70F230EF4FC8607BD0793F7073F1B
:10C350003301F1408A8A01498347C4FD6367F902CA
:10C36000CE85130584FC232C54FD97000000E78044
:10C3700080EA5281130104FCF2506254D2544259B3
:10C38000B259225A925A2161828026859700000074
:10C39000E78060C193171900D69705092390A7007D
:10C3A0001379F90F55BF828097A7FF1F938707A5C1
:10C3B0009C43D847A1679387A702631AF70A39718C
:10C3C00006DE22DC26DA80004AD84ED652D456D277
:10C3D0003285B28497000000E780C0BAAA8926851A
:10C3E00097000000E78020BCFD572318A4FC268599
:10C3F0002319F4FC97000000E780E0BA83D74400DB
:10C400000A8A231AA4FC858393F7F70F230EF4FC02
:10C410008607BD0793F7073F3301F1408A8A014938
:10C420008347C4FD6367F902CE85130584FC232C82
:10C4300054FD97000000E78000DE5281130104FCE8
:10C44000F2506254D2544259B259225A925A21613E
:10C450008280268597000000E780E0B493171900DA
:10C46000D69705092390A7001379F90F55BF82804D
:10C4700097A7FF1F938787989C43D847A167890791
:10C480006310F70A397106DE22DC26DA80004AD80A
:10C490004ED652D456D23285328997000000E780BA
:10C4A00060AEAA894A8597000000E780C0AF835735
:10C4B00049000A8A2318A4FC858393F7F70F230CFD
:10C4C000F4FC8607BD0793F7073F3301F1408A8AE2
:10C4D0008144834784FD63E7F402CE85130584FC21
:10C4E000232A54FD97000000E780E0D25281130117
:10C4F00004FCF2506254D2544259B259225A925A10
:10C50000216182804A8597000000E780C0A9939747
:10C510001400D69785042390A70093F4F40F55BF19
:10C52000828097A7FF1F9387678D9C43D847A16799
:10C530009387E704631EF70A397106DE22DC26DAE8
:10C5400080004AD84ED652D456D23285B284970053
:10C550000000E78020A3AA89268597000000E780D5
:10C5600080A42318A4FC268597000000E780A0A3E0
:10C57000231AA4FC268597000000E780C0A283D779
:10C5800044000A8A2319A4FC858393F7F70F230E2E
:10C59000F4FC8607BD0793F7073F3301F1408A8A11
:10C5A00001498347C4FD6367F902CE85130584FC06
:10C5B000232C54FD97000000E780E0C55281130151
:10C5C00004FCF2506254D2544259B259225A925A3F
:10C5D00021618280268597000000E780C09C931728
:10C5E0001900D69705092390A7001379F90F55BFB5
:10C5F000828097A7FF1F938767809C43D847A167D6
:10C600009387C704631AF70A397106DE22DC26DA3B
:10C6100080004AD84ED652D456D23285B284970082
:10C620000000E7802096AA89268597000000E78011
:10C630008097FD572318A4FC2685231AF4FC970045
:10C640000000E780409683D744000A8A2319A4FC9F
:10C65000858393F7F70F230EF4FC8607BD0793F746
:10C66000073F3301F1408A8A01498347C4FD63676C
:10C67000F902CE85130584FC232C54FD970000009D
:10C68000E78060B95281130104FCF2506254D25425
:10C690004259B259225A925A2161828026859700C6
:10C6A0000000E780409093171900D6970509239062
:10C6B000A7001379F90F55BF82809797FF1F9387C3
:10C6C000E7739C43D847A167DD076317F704176337
:10C6D000FFFFE702C3A07971328532849700000022
:10C6E000E780408A2AC6228597000000E780A08B59
:10C6F0002311A102228597000000E780A088B2459F
:10C700002300A102280897000000E780C0B045611F
:10C710001763FFFF6700E39E82809797FF1F938751
:10C72000E76D9C43D847A167938787046317F70495
:10C730001763FFFFE702A39A79713285328497006D
:10C740000000E78020842AC6228597000000E78049
:10C7500080852311A102228597000000E780808256
:10C76000B2452300A102280897000000E780A0AA94
:10C7700045611763FFFF6700C39882809797FF1F8B
:10C780009387C7679C43D847A1679387A704631221
:10C79000F7021763FFFFE702839401112800814528
:10C7A00097000000E78020A705611763FFFF67007F
:10C7B000439582809797FF1F938747649C43D84790
:10C7C000A167938757026319F7021763FFFFE70218
:10C7D00003910111328597F0FFFFE780A07A2308CB
:10C7E000A1008145280097000000E780C0A20561F4
:10C7F0001763FFFF6700E39082809797FF1F93877F
:10C80000E75F9C43D847A1679387E702631BF70460
:10C810001763FFFFE702A38C01113285328497F082
:10C82000FFFFE7804078AA84228597F0FFFFE7802A
:10C830008077854709E9228597F0FFFFE7808074BC
:10C840004205B337A00028008145231891003ECA55
:10C8500097000000E780209C05611763FFFF6700D9
:10C86000438A82809797FF1F938747599C43D847F5
:10C8700099476313F7081763FFFFE702438679714F
:10C880003285328497F0FFFFE780C06F2AC6228589
:10C8900097F0FFFFE78020712310A102228597F017
:10C8A000FFFFE780206E2301A102228597F0FFFFA2
:10C8B000E780406DA301A102228597F0FFFFE7808A
:10C8C000606C2302A102228597F0FFFFE780806B56
:10C8D0002313A102228597F0FFFFE780A06AB245EB
:10C8E0002314A102280897000000E780C092456148
:10C8F0001763FFFF6700E38082809797FF1F93878E
:10C90000E74F9C43D847A1679387C7036313F70892
:10C910001753FFFFE702A37C79713285328497F0C9
:10C92000FFFFE78020662AC6228597F0FFFFE78099
:10C9300080672310A102228597F0FFFFE780A066A1
:10C940002311A102228597F0FFFFE780A063230255
:10C95000A102228597F0FFFFE780C062A302A10237
:10C96000228597F0FFFFE780E0612303A102228583
:10C9700097F0FFFFE7800061B245A303A1022808FA
:10C9800097000000E780208945611753FFFF67008B
:10C99000437782801753FFFFE702637401112A84F3
:10C9A00097F0FFFFE780005EAA84228597F0FFFFE3
:10C9B000E780605F228597F0FFFFE780C05E035746
:10C9C00044008D4763F7E700228597F0FFFFE7807B
:10C9D000805D228597F0FFFFE780E05C2800A68558
:10C9E00097000000E780208305611753FFFF670071
:10C9F00043719797FF1F938767409C43D847A16770
:10CA0000FD07631FF7001753FFFFE702436D3285F1
:10CA100097000000E78040F81753FFFF6700636E40
:10CA200082809797FF1F9387673D9C43D847A167F4
:10CA3000E5076315F7081753FFFFE702436A7971AB
:10CA40003285328497F0FFFFE780C0532AC62285E3
:10CA500097F0FFFFE7802055228597F0FFFFE780E2
:10CA600080542310A102228597F0FFFFE780A05396
:10CA7000520551812311A10222852302010297F060
:10CA8000FFFFE7802050A302A102228597F0FFFF5D
:10CA9000E780404F2303A102228597F0FFFFE78044
:10CAA000604EB245A303A102280897F0FFFFE7807C
:10CAB000807645611753FFFF6700A36482809797D4
:10CAC000FF1F9387A7339C43D847A1679387E7034A
:10CAD000631FF7001753FFFFE7026360328597007B
:10CAE0000000E78060EB1753FFFF670083618280DF
:10CAF0009797FF1F938787309C43D847A1679387F9
:10CB00004704631EF7021753FFFFE702435D797185
:10CB10003285328497F0FFFFE780C0462AC622851F
:10CB200097F0FFFFE7802048B245280897F0FFFF05
:10CB3000E780606E45611753FFFF6700835C82806A
:10CB40009797FF1F9387872B9C43D847A1679387AD
:10CB500087026310F7041753FFFFE7024358797108
:10CB60003285328497F0FFFFE780C0412AC62285D4
:10CB700097F0FFFFE7800041B2452300A10228089B
:10CB800097F0FFFFE780206945611753FFFF6700BB
:10CB9000435782801753FFFFE7026354011197F058
:10CBA000FFFFE780203EAA85280097F0FFFFE7807F
:10CBB000806605611753FFFF6700A3549797FF1F17
:10CBC0009387C7239C43D847A167D107631FF7000A
:10CBD0001753FFFFE702A350328597000000E7805C
:10CBE000A0FB1753FFFF6700C35182809797FF1F79
:10CBF0009387C7209C43D847A167C507631FF700E9
:10CC00001753FFFFE702A34D328597000000E7802E
:10CC1000A0F81753FFFF6700C34E82809797FF1F4E
:10CC20009387C71D9C43D847A167B907631FF700C7
:10CC30001753FFFFE702A34A328597000000E78001
:10CC4000A0F51753FFFF6700C34B82809797FF1F24
:10CC50009387C71A9C43D847A167AD07631FF700A6
:10CC60001753FFFFE702A347328597000000E780D4
:10CC7000A0F21753FFFF6700C34882809797FF1FFA
:10CC80009387C7179C43D84789476318F702175300
:10CC9000FFFFE702C3440111328532C897F0FFFF5E
:10CCA000E780402EAA85280097F0FFFFE780A05676
:10CCB00005611753FFFF6700C34482809797FF1FEA
:10CCC0009387C7139C43D847A1678D076311F70467
:10CCD0001753FFFFE702A34001113285328497F01A
:10CCE000FFFFE780202A13066100AA844C002285FA
:10CCF00097300000E780C0232800A68597F0FFFF4B
:10CD0000E780605105611753FFFF6700833F828012
:10CD10009797FF1F9387C70E9C4381CFDC4391CB2E
:10CD20001753FFFFE702A33B82971753FFFF6700EC
:10CD3000433D82801753FFFFE702633A79713C0855
:10CD4000AE843ED2A165B7070A002A843ED44810BB
:10CD50003C08DD053ED636C432C63AC297D0FFFF46
:10CD6000E780402C12474810BA8597F0FFFFE78014
:10CD7000C01332464810B28597F0FFFFE780E014F9
:10CD8000A2464810B68597F0FFFFE78000125010CA
:10CD900001478146A685228597D0FFFFE780E04DB9
:10CDA00045611753FFFF6700C3351753FFFFE702C5
:10CDB000033301117C000329C501AE843ECAA1657D
:10CDC000B70707002A843ECC48087C00C5053ECE44
:10CDD00097D0FFFFE78000258345D900480897F0EA
:10CDE000FFFFE780800C500801478146A685228519
:10CDF00097D0FFFFE780604805611753FFFF67008A
:10CE000043301753FFFFE702832D83C7950093F745
:10CE1000F707A384F50097000000E78040F9175357
:10CE2000FFFF6700032E1753FFFFE702432B7971C3
:10CE30003C08AE843ED2A165B70709002A843ED4DF
:10CE400048103C08938545043ED632C636C497D078
:10CE5000FFFFE780201DA2464810B68597F0FFFF30
:10CE6000E780A00432464810B28597F0FFFFE780C4
:10CE7000C005501001478146A685228597D0FFFF47
:10CE8000E780A03F45611753FFFF670083271753D3
:10CE9000FFFFE702C32483C7950041112A8493F75B
:10CEA000F707A384F50032852EC697F0FFFFE780D1
:10CEB000800F85672AC46370F50297700000E780D1
:10CEC00020E92246B24509ED1147814622859700A7
:10CED0000000E78060E641011753FFFF670063220F
:10CEE00001478346F501DDB71753FFFFE702831DB6
:10CEF00001113C003ECAB7070A003ECC3C003ECEC2
:10CF000083C79500AA89328593F7F707A384F500B4
:10CF10002E8497F0FFFFE78000098567637DF504A5
:10CF2000A165AA8493858504480897D0FFFFE78010
:10CF3000600F268597700000E78080E12A8929E14B
:10CF40009145480897F0FFFFE78020F6A68548083E
:10CF500097F0FFFFE78060F7CA85480897F0FFFF6A
:10CF6000E780A0F4014781465008A2854E8597D0FE
:10CF7000FFFFE780803005611753FFFF6700C3178D
:10CF80008145480897F0FFFFE78020F20349090236
:10CF900075BF1753FFFFE702E31279711C103ECAF9
:10CFA000B7070F003ECC404D1C10AA84AE8948083C
:10CFB000994532C636893ECE97D0FFFFE78080067E
:10CFC00032464808B28597F0FFFFE78000EE630C19
:10CFD0000902A545480897F0FFFFE780C0E625460F
:10CFE000CA8597200100E78020A4500801478146A8
:10CFF000CE85268597D0FFFFE7802028456117530F
:10D00000FFFF6700630F8355C402480897F0FFFFD6
:10D01000E780A0EB0355E402814505C585478545BA
:10D020006301F502C167FD179305F00F630BF5006F
:10D030007D1597700000E780208E9305150093F50D
:10D04000F50F480897F0FFFFE78020E683450403CB
:10D05000480897F0FFFFE78040E583451403480840
:10D0600097F0FFFFE78060E483552403480897F0BA
:10D07000FFFFE78080E583554403480897F0FFFFF2
:10D08000E780A0E49DB71753FFFFE702430583C77E
:10D0900095008146014693F7F707A384F5009700B2
:10D0A0000000E78040EF1753FFFF67008305175329
:10D0B000FFFFE702C30279713E841C103ECA2E892D
:10D0C000B7070F00A1653ECCFD051C10AA844808D7
:10D0D00042C03AC23ECE36C432C697D0FFFFE78088
:10D0E00060F432464808B28597F0FFFFE780E0DB46
:10D0F000A2464808B68597F0FFFFE78000DD12479B
:10D100004808BA8597F0FFFFE78020DC0248630CEF
:10D1100008029145480897F0FFFFE780C0D211460A
:10D12000A28597200100E7802090500801478146A2
:10D13000CA85268597D0FFFFE780201445611753E5
:10D14000FFFF670003FC8945480897F0FFFFE78071
:10D1500080CF834704002300F50083471400A30019
:10D16000F500E1B71753FFFFE702C3F583C795004A
:10D1700001112A8A93F7F707A384F5003285AE845C
:10D1800032C697F0FFFFE78000E232462A893285F7
:10D1900097F0FFFFE78000DF85676373F902AA89D4
:10D1A0004A8597700000E780A0BA2A8419ED1147DC
:10D1B00081464A86A685528597000000E780C0B761
:10D1C00005611753FFFF670023F39387E9FF93F788
:10D1D000F70F0547E366F7FE8347F50195EB8947AF
:10D1E000E380F9FE8346F401528501474A86A6850D
:10D1F00097000000E78040B4A167D90748083ECCFB
:10D20000230A010002CE97000000E780A0B04DBFC6
:10D21000639EE7008947639EF90093071020231F50
:10D22000F50097700000E780C0B76DBF0947E39B2A
:10D23000E7FA8D47E398F9FA228597700000E780B6
:10D2400080DF9797FF1F9387A7DA9C4399E797970B
:10D25000FF1F9387A7C39C4399C703D504009780FA
:10D260000000E780A0CE231F040022855DBF175376
:10D27000FFFFE702C3E601113C003ECAB7070B00FF
:10D280003ECC3C003ECE83C795002A89328593F779
:10D29000F707A384F500AE8497F0FFFFE780A0D0E6
:10D2A00093170501C187635AF006A1652A84938507
:10D2B000E502480897D0FFFFE780C0D6A28548085E
:10D2C00097F0FFFFE78060C09797FF1F938707BC29
:10D2D0009C43A9EB01449375F40F480897F0FFFFB6
:10D2E000E780A0BC9355844093F5F50F480897F06C
:10D2F000FFFFE78080BB9355044193F5F50F480885
:10D3000097F0FFFFE78060BA014781465008A68585
:10D310004A8597D0FFFFE78040F605611753FFFF6E
:10D32000670023DE416585460546A2857D15975039
:10D330000000E78060BD59DD510597000100E780DE
:10D34000808F130440063344850271B71753FFFFE3
:10D35000E702E3D80111B70706003EC683C7950070
:10D3600021642A8993F7F707A384F500AE84280087
:10D370009305A4040AC40AC897D0FFFFE78080CAB7
:10D38000300001478146A6854A8597D0FFFFE78098
:10D39000C0EE97E0FFFFE780E01113049404480813
:10D3A00022CC230A010002CE97000000E78080967D
:10D3B00005611753FFFF6700C3D41753FFFFE70250
:10D3C00063D0C1642A8901449799FF1F9389C9C317
:10D3D000130A8002FD1497E0FFFFE780E0BD63477A
:10D3E000A40001451753FFFF670003D1B3074403AF
:10D3F00003A7C90ABA9703D707006306970083D724
:10D400002700638427010504F9B70545E1BF1753D9
:10D41000FFFFE70223CB2A8A2E8999C123A00500AA
:10D4200081498144979AFF1F938ACA9D614B97E077
:10D43000FFFFE780A0BE63C7A4004E851753FFFF20
:10D44000670083CB3384640383A70A003E94835729
:10D45000040099E763040900232089008504C1BF03
:10D460004146D2851305440097100100E7806059BA
:10D4700075F5A289E5B71753FFFFE702A3C4397119
:10D480007C083ED4B7070A003ED67C083ED883C746
:10D4900095002A8A328593F7F707A384F5002E8931
:10D4A00032C697F0FFFFE78000B085676373F50829
:10D4B0003246AA84328597F0FFFFE780A0AC85470B
:10D4C000AA8963E8A706A16593858504281097D0EB
:10D4D000FFFFE78020B5268597700000E780408732
:10D4E0002A8429ED9145281097F0FFFFE780E09B03
:10D4F000A685281097F0FFFFE780209DCE85281095
:10D5000097F0FFFFE780609A014781463010CA8597
:10D51000528597D0FFFFE78040D6A16793877704B5
:10D5200048183EDC230A010202DE97F0FFFFE78085
:10D53000607E21611753FFFF670003BC81452810FF
:10D5400097F0FFFFE7806096A685281097F0FFFF11
:10D55000E780A0979797FF1F938787E19C4381CB34
:10D5600022856389090097D00000E7804024834525
:10D57000040271B797D00000E780C022CDBF1753D7
:10D58000FFFFE70223B483C795004111AA8993F7EF
:10D59000F707A384F5003285AE84328A97F0FFFF47
:10D5A000E78060A08567637FF5022A8997600000A5
:10D5B000E780007A2A84914631C58347F501054703
:10D5C0006387E70291C70D476366F704AD461DA860
:10D5D0009305050303250A00414697100100E780E3
:10D5E00040420DE941011753FFFF6700E3B0930587
:10D5F000950803250A00414697100100E780604026
:10D60000814669F54A86A6854E8597000000E78029
:10D61000C081C9BF83250A001305940897700000D4
:10D62000E780A02919C1C146F1BF9797FF1F9387D3
:10D63000279C9C4399E79797FF1F938727859C43D7
:10D6400099C7228597800000E780208A69FD854779
:10D65000A30FF400228597B00000E7806084228544
:10D6600097600000E780E0734E8581464A86A68574
:10D6700097F0FFFFE780607BA1679387570448001E
:10D680003EC42302010002C697F0FFFFE7808068D6
:10D6900091BF1753FFFFE70203A283C79500411113
:10D6A000AA8993F7F707A384F50032852E89B28AF9
:10D6B00097F0FFFFE780208F85676374F50EAA84DB
:10D6C00097600000E780C0682A840DED416B014A35
:10D6D000979BFF1F938B4B93130C400E7D1B19A838
:10D6E00033048A0383A70B0B3E948357C4016383DF
:10D6F0006705050A97E0FFFFE780008BE342AAFE7B
:10D7000095460DA08357C5016396970293050503BF
:10D7100003A50A00414697100100E780802E994634
:10D7200011E181462686CA854E8597F0FFFFE78086
:10D73000C06F85A883A50A00130504039770000035
:10D74000E780A017C14679FD2285231E940097A08B
:10D750000000E780E074228597600000E780606445
:10D760009797FF1F9387C7C09C43A9C32300040258
:10D77000228597D00000E78040F04E8581462686BE
:10D78000CA8597F0FFFFE780406AA1679387070487
:10D7900048003EC42302010002C697F0FFFFE78065
:10D7A000605741011753FFFF6700639489472300C7
:10D7B000F402E1B7397106DE22DC4AD8800052D487
:10D7C00056D25AD026DA4ED65ECE2E8A32892A8B8F
:10D7D00097D0FFFFE780407A0605710541998A8A54
:10D7E0003301A140232224FC231404FC97D0FFFF23
:10D7F000E780807883479A000605350593F7F70799
:10D800002315A4FCA304FA004A85232624FC97E0F0
:10D81000FFFFE780407993170501C1876340F0025D
:10D820005681130104FCF2506254D2544259B25949
:10D83000225A925A025BF24B21618280AA844A8565
:10D8400097E0FFFFE7802076AA894A8597E0FFFFEF
:10D85000E7806075A1659385C5022A89130544FC9C
:10D8600097C0FFFFE780007C268597C0FFFFE78019
:10D870004070854511C94A86CE8597C0FFFFE78075
:10D88000C069AA8B21E98945130544FC97E0FFFF95
:10D89000E780A061A685130544FC97E0FFFFE780C1
:10D8A000C062CE85130544FC97E0FFFFE780E0618E
:10D8B000CA85130544FC97E0FFFFE780006101473C
:10D8C0008146130644FCD2855A8597D0FFFFE78036
:10D8D000C09AB9B78145130544FC97E0FFFFE78084
:10D8E000C05CA685130544FC97E0FFFFE780E05D80
:10D8F000CE85130544FC97E0FFFFE780005DCA85F5
:10D90000130544FC97E0FFFFE780205C814497D03B
:10D91000FFFFE7806066E3D4A4FA83A70B011397A7
:10D920001400BA9783D5070099C5130544FC97E006
:10D93000FFFFE78080598504D9BF797106D622D4CC
:10D940004AD000184ECE52CC56CA26D25AC8AE89FA
:10D950003289AA8A97D0FFFFE78000620605690531
:10D9600041990A8A3301A140232A24FC231C04FC88
:10D9700097D0FFFFE780406083C7990006052D051B
:10D9800093F7F707231DA4FCA384F9004A85232EEF
:10D9900024FC97E0FFFFE780006193170501C18732
:10D9A000634FF0005281130104FDB250225492548F
:10D9B0000259F249624AD24A424B45618280AA84A6
:10D9C0004A8597E0FFFFE780005EA1659385A50289
:10D9D0002A89130544FD97C0FFFFE780A0642685D0
:10D9E00097C0FFFFE780E058854509C9CA8597C001
:10D9F000FFFFE78080552A8B29E18945130544FD07
:10DA000097E0FFFFE780604AA685130544FD97E095
:10DA1000FFFFE780804BCA85130544FD97E0FFFFB9
:10DA2000E780A04A01478146130644FDCE8556850E
:10DA300097D0FFFFE7806084B5B78145130544FDAB
:10DA400097E0FFFFE7806046A685130544FD97E059
:10DA5000FFFFE7808047CA85130544FD97E0FFFF7D
:10DA6000E780A046814497D0FFFFE780E050E3DBEA
:10DA7000A4FA83270B0113971400BA9783D50700E4
:10DA800099C5130544FD97E0FFFFE7800044850436
:10DA9000D9BF1743FFFFE702836483474500404D2A
:10DAA000D5EFFD575DC48346940009476363D70AE9
:10DAB0000346B400854663EEC6088306E40063CAE5
:10DAC00006085C45F9562390D7009787FF1F83C748
:10DAD000A73399E3A304E4009787FF1F9387073BCD
:10DAE0009C4381E78947A306F4009797FF1F93871C
:10DAF00027889C4381E789472306F40097050000A7
:10DB000093854506AA841305040197F00000E78079
:10DB10002010FD57231AF40281471CDC0148978727
:10DB2000FF1F23AF872C9787FF1F9387A72D232ED7
:10DB3000040304C0804397D0FFFFE780204E614676
:10DB40003306C502814522859740FFFFE780205CB0
:10DB500081473E851743FFFF6700A35AFD57D5BF96
:10DB60001743FFFFE702A3572A8403554502976036
:10DB70000000E780E01D19E5231E04001743FFFFA6
:10DB8000670023588357E401F5DB930504FF17452D
:10DB900001001305A5E397E00000E780E014F9BF5A
:10DBA0001743FFFFE702A3532E89A1654111938517
:10DBB000E5032A8436C432C6BE843AC297C0FFFF4A
:10DBC000E780404612472285BA8597E0FFFFE7804D
:10DBD000C02D32462285B28597E0FFFFE780E02E18
:10DBE000A2462285B68597E0FFFFE780002E6303FB
:10DBF00009029145228597E0FFFFE780C024114686
:10DC0000A68597100100E78020E241011743FFFF3E
:10DC10006700234F8945228597E0FFFFE780A02218
:10DC200083C704002300F50083C71400A300F50098
:10DC3000E9BF1743FFFFE702834A83C79500444DBE
:10DC4000054793F7F707A384F5001C42411183C7EA
:10DC500007006367F7062E842A89B1C003C7D40082
:10DC6000630FF7021787FF1F13074722184305C3E7
:10DC7000A386F40097A00000E780404A83C7D40041
:10DC800099E741657D1597400000E780403083D7D4
:10DC90002403918B89C797E00000E780C0134A8571
:10DCA000A28597F0FFFFE7808010A167C1074800B9
:10DCB0003EC42302010002C697F0FFFFE780800503
:10DCC00041011743FFFF6700C3431743FFFFE7020C
:10DCD000034103D745008D47AA8441112E84328920
:10DCE0002E8563E3E70297E0FFFFE780C02BAA855C
:10DCF00023000900268597C0FFFFE780002541012A
:10DD00001743FFFF6700E33F97E0FFFFE780A0298D
:10DD10002AC6228597E0FFFFE780E028B2458547C5
:10DD20002A862300F900268597C0FFFFE780E01EC2
:10DD3000F9B7397106DE22DC26DA80004ED652D4DD
:10DD400056D24AD85AD05ECEAE89B284AA8A97D02B
:10DD5000FFFFE780602106051305250241990A8A25
:10DD60003301A140232224FC231404FC97D0FFFF9D
:10DD7000E780801F83C7990006054D0593F7F707D5
:10DD80002315A4FCA384F9002685232624FC97E010
:10DD9000FFFFE780402193170501C1876340F00230
:10DDA0005281130104FCF2506254D2544259B259C8
:10DDB000225A925A025BF24B21618280AA8B03ABFA
:10DDC000040097C0FFFFE780C01A51E583D74400E5
:10DDD00001498544F11793B71700A301F4FC834769
:10DDE00034FCA165C9C79385E504130544FC97C0BD
:10DDF000FFFFE7802023A685130544FC97E0FFFF83
:10DE0000E780A00ADE85130544FC97E0FFFFE7806A
:10DE1000C00B834734FC114691E30946DA851305AC
:10DE200044FC97E0FFFFE78060058144630A090036
:10DE3000416B7D1B97D0FFFFE780001363CCA402EA
:10DE400001478146130644FCCE85568597C0FFFFE7
:10DE5000E780A042B1B7A685130634FC9700000006
:10DE6000E780E0E6933415002A8986048DBF938508
:10DE7000C504A5BF8327C90013971400BA9783D59B
:10DE8000070063886501130544FC97E0FFFFE78006
:10DE9000C003850445B71743FFFFE702C32179712B
:10DEA0001C103EC4B7070F003EC61C103EC883C7F7
:10DEB0009500AA8A328593F7F707A384F500AE8907
:10DEC000328497E0FFFFE780000E93170501C187BA
:10DED000635AF0062A8A228597E0FFFFE780A00CAC
:10DEE0002A895285032B040097C0FFFFE780600852
:10DEF00039ED8357440081440544F11793B7170067
:10DF0000A303F10083457100DA872287CA8652860F
:10DF1000280097000000E780E0C8014781463000F4
:10DF2000CE85568597C0FFFFE7802035A167938790
:10DF3000D70348083ECC230A810026CE97F0FFFF86
:10DF4000E78040DD45611743FFFF6700431AA28564
:10DF50001306710097000000E78060D7AA84094487
:10DF600055D13544E30055FB4A8597F0FFFFE78024
:10DF700000450D4441D9014497D0FFFFE780C0FE22
:10DF8000634DA400C16B0144FD1B97D0FFFFE780E8
:10DF9000A0FD634EA4001544B5B7DC44131714006C
:10DFA000BA9783D70700638327030504F1B7D844E2
:10DFB00093171400BA9703D70700631B77012390C8
:10DFC0002701268597A00000E78080DB01441DBF64
:10DFD000050465BF1743FFFFE702C30E83C7950023
:10DFE00041112A8A93F7F707A384F50032852E8919
:10DFF000328497E0FFFFE78000FB93170501C1879C
:10E000006353F006AA89228597E0FFFFE780A0F915
:10E010002311A1004E85832A040097C0FFFFE780EB
:10E0200040F539E58357440085440144F11793B71F
:10E030001700A300F1000348110003572100D68701
:10E040005285CE862686CA8597F0FFFFE780600658
:10E05000A167F10748003EC42302910022C697F051
:10E06000FFFFE78020CB41011743FFFF6700C30894
:10E07000A2851306110097000000E78040C52A849E
:10E08000894455D98357210011678544BA97C2073F
:10E090001167C1831307F7EFE36FF7F89787FF1F47
:10E0A000938707F59C4381CB854513052100975045
:10E0B0000000E7802075835521002285814497C0A8
:10E0C000FFFFE780A0E125D923100500228597A056
:10E0D0000000E78040CD85B71743FFFFE702A3FDAF
:10E0E00083C7950041112A8B93F7F707A384F500A6
:10E0F00032852E8A328497E0FFFFE780C0EA9317CB
:10E100000501C1876351F006AA8A228597E0FFFFC7
:10E11000E78060E92A895685832B040097C0FFFFBA
:10E12000E78020E531E58357440081440544F11739
:10E1300093B71700A301F10003483100DE875A8529
:10E140004A87D6862286D28597F0FFFFE78060F661
:10E15000A167ED0748003EC42302810026C697F060
:10E16000FFFFE78020BB41011743FFFF670023F853
:10E17000A2851306310097000000E78040B5AA840D
:10E1800009445DD99167CA97C2071167C183130714
:10E19000F7EF0544E362F7FACA8597C0FFFFE7800F
:10E1A000E0D3014451F9814997D0FFFFE780C0DCFB
:10E1B00063DBA900984893971900BA9703D7070023
:10E1C00005EF2390270197D0FFFFE780E0DA1544A1
:10E1D000E384A9F6268597A00000E780C0BC978756
:10E1E000FF1F9387E7E09C430144B9D74A859750C6
:10E1F0000000E780C05889B785097DB71743FFFF46
:10E20000E70243EC79713E847C083EC82E8AB7074A
:10E210001400A1653ECAE5057C08AA89080836C431
:10E22000428932C6BA8AC6843ECC97C0FFFFE780D7
:10E2300060DFCA85080897E0FFFFE78000C7324625
:10E240000808B28597E0FFFFE78020C8A246630A6E
:10E2500009049D45080897E0FFFFE780C0BE1D4602
:10E2600081459740FFFFE78080EA63890A0891456E
:10E27000080897E0FFFFE78000BD1146A6859700DC
:10E280000100E780607A100801478146D2854E85FB
:10E2900097C0FFFFE78060FE45611743FFFF6700FF
:10E2A000A3E5B685080897E0FFFFE78000C21C40A1
:10E2B0000808D8439355C701858912075183B205D1
:10E2C000D98D97E0FFFFE78040C01C40080883C558
:10E2D000870097E0FFFFE78040BD1C40080883C52A
:10E2E000A70097E0FFFFE78040BC1C40080883C5FB
:10E2F000970097E0FFFFE78040BB85BF894508088E
:10E3000097E0FFFFE78020B483C704002300F500F7
:10E3100083C71400A300F500BDB71743FFFFE70252
:10E3200063DA83C795004111AA8993F7F707A3849D
:10E33000F5003285AE84328497E0FFFFE780A0C607
:10E3400093170501C187635DF0042A89032A04003D
:10E3500097C0FFFFE780E0C119E9835744000548F3
:10E36000F11793B71700A307F100814631A81306F0
:10E37000F100A28597000000E78060951DC51C454F
:10E380009DC783D6470001480347F10093078500E6
:10E39000D2884A86A6854E8597000000E78040E631
:10E3A00041011743FFFF670023D509487DBF1D4882
:10E3B0006DBF1743FFFFE702E3D065715C083EC401
:10E3C000B7077B013EC65C083EC883C795002A8A12
:10E3D000328593F7F707A384F500AE8997E0FFFF36
:10E3E000E78040BA8357E100E1C78945280097C01C
:10E3F000FFFFE78020C38145280097E0FFFFE7800B
:10E40000C0AA97C0FFFFE78000C99787FF1F9387C7
:10E4100027F69C431784FF1F0344049FAA843334C8
:10E42000800099C3136424009787FF1F938707A672
:10E430009C4399C3136444009787FF1F938747BB8E
:10E440009C4399C31364840083D5040028000149C8
:10E4500097E0FFFFE78060A783D52400280097E0BE
:10E46000FFFFE78080A683D54400280097E0FFFFE8
:10E47000E780A0A597D0FFFFE78000AB93150501CB
:10E48000C181280097E0FFFFE78020A4A285280033
:10E4900097E0FFFFE78060A39C446360F9020147B7
:10E4A00081463000CE85528597C0FFFFE780E0DCD3
:10E4B00059611743FFFF670023C4DC44131449006C
:10E4C00028003E9497E0FFFFE78060968347440072
:10E4D0000347540089070607BA978607E36AF5FCE5
:10E4E000835524002800814A97E0FFFFE780E09DE4
:10E4F00083454400280097E0FFFFE780009B8345A9
:10E500005400280097E0FFFFE780209A83474400EB
:10E5100063C9FA00814A8347540063C1FA020509BE
:10E52000A5BF1C4413975A002800BA9783D507004B
:10E53000850A97E0FFFFE7804099C9BF032BC4001D
:10E5400093975A0028003E9B83552B00850A97E03D
:10E55000FFFFE780809783550B00280097E0FFFFBF
:10E56000E780A0964DBF1743FFFFE70243B75C4922
:10E5700093E717005CC997A00000E78020B6174317
:10E58000FFFF670003B81743FFFFE70243B52E8480
:10E59000814597F0FFFFE780C0E705C58357050079
:10E5A000FD172310F50009C4835725002310F4003C
:10E5B00097000000E78060FB01451743FFFF6700FD
:10E5C00043B431457DD823100400C5BF1743FFFF76
:10E5D000E70243AF83C7950041112A8A93F7F707F3
:10E5E000A384F50032852E89328497E0FFFFE7800F
:10E5F000809B93170501C1876356F006AA89C14520
:10E60000228597E0FFFFE780A0802A8B4E85832A32
:10E61000040097C0FFFFE780C09531E983574400AD
:10E62000231101000544F11793B71700A300F1006F
:10E6300081440348110003572100D6875285CE86B6
:10E640002286CA8597F0FFFFE780A0A6A16793877F
:10E65000170248003EC42302810026C697E0FFFF50
:10E66000E780406B41011743FFFF6700E3A81306F3
:10E670001100A28597F0FFFFE7806065AA8409E595
:10E6800023110100094475B7930521005A859700AD
:10E690000000E78080EF835721002A84D9DB978729
:10E6A000FF1F9387E7949C4381CB85451305210089
:10E6B00097500000E78000158355210026853144DE
:10E6C00097C0FFFFE78080812DD5231005002685A8
:10E6D00097900000E780206D0144A1BF1743FFFF22
:10E6E000E702E39F41112E896C00AA8402C697F0CD
:10E6F000FFFFE78000D20DC1035705000507231077
:10E70000E50097000000E78040E681473E85410133
:10E710001743FFFF6700E39E3247954765DBCA85D5
:10E72000268597300000E780400DC147E34005FE95
:10E730003244854741462310F40083570900A685DB
:10E74000130544002311F40097000100E780C02D59
:10E75000228545BF1743FFFFE702C39683C7950095
:10E760004111AA8A93F7F707A384F5003285AE8991
:10E77000328497E0FFFFE780008393170501C1878C
:10E780006356F0062A8AC145228597D0FFFFE780AD
:10E790002068AA845285032B040097B0FFFFE7800E
:10E7A000407D31E983574400231101008544F1176E
:10E7B00093B71700A300F100014403481100035769
:10E7C0002100DA875685D2862686CE8597F0FFFF10
:10E7D000E780208EA1679387070248003EC423028A
:10E7E000910022C697E0FFFFE780C0524101174326
:10E7F000FFFF67006390A2851306110097F0FFFFEB
:10E80000E780E04C2A8409E523110100894475B7AB
:10E8100026859305210097000000E78060ECAA841C
:10E8200049FD83552100228597B0FFFFE780006BEB
:10E8300049F5014997C0FFFFE7800074635DA900B7
:10E84000184893171900BA9703D707000DEF03571D
:10E8500021002390E70097C0FFFFE780E071630687
:10E8600025039777FF1F9387A7789C4399C7035584
:10E87000210097500000E78080F0228597900000EB
:10E88000E78060521DBF050975B795443DB705C1C6
:10E890009307F00F630FF500C547630CF50093076E
:10E8A000F5FF05453315F50042054181828001459C
:10E8B000828041657D158280B9E91743FFFFE70239
:10E8C000038203450603328497000000E78060FC62
:10E8D0009305803EB305B502C205C18181CD0357C2
:10E8E000E402854763F8E7001305040197E00000A0
:10E8F000E78020428357E40241677D176385E70084
:10E90000FD172317F4021733FFFF6700837F828010
:10E910001733FFFFE702237A004283C79500444D77
:10E920000349140093F7F707A384F5008347040015
:10E93000220911673369F900A167B347F900411152
:10E940002A8BAE8A63ECE70E834724001307C00EC0
:10E95000B91793F7F70F6373F71003473400C147F4
:10E9600063EEE70E834744001307E00793C70708E9
:10E970006371F70C8349840083477400A209B3E9EB
:10E98000F900856763F7F90A034A64008347540076
:10E990004E85220A336AFA0097500000E780403B18
:10E9A00061C123962403834B3400137AFA00239A1F
:10E9B0003403238874032399440393890401631C5B
:10E9C000090023A60402239804024E8597E0000064
:10E9D000E78060363DA0034924004A859700000087
:10E9E000E78020EB2397A402834744004E85A38849
:10E9F000F402E38D0BFCE30B09FC97E00000E780D9
:10EA0000202F97900000E780007381460146D6854D
:10EA10005A8597E0FFFFE7800058A1679387970327
:10EA20003EC423020100480002C697E0FFFFE780D2
:10EA3000602E41011733FFFF6700636B8544A28698
:10EA40002686D6855A8597E0FFFFE780C054A167E8
:10EA5000938797033EC423029100F1B7BD44C5B725
:10EA60009144F1BF1733FFFFE702C36501111C0892
:10EA7000404D3EC2B7070F003EC41C083EC62A895F
:10EA8000AE8997C0FFFFE78000D7585C1C5C6346E7
:10EA9000B70E6394E50063E2A70E3385A740B3B7D2
:10EAA000A700B305B7401306803E81469D8D9700B1
:10EAB0000100E78080B793140501C180A1659385AB
:10EAC000C503480097B0FFFFE780C0558145480067
:10EAD00097D0FFFFE780603D83550404480097D03E
:10EAE000FFFFE780803E83552404480097D0FFFF56
:10EAF000E780A03D814589CCC167FD179305F00FE4
:10EB00006388F400268597500000E780E0E0AA853E
:10EB1000480097D0FFFFE780403903554404814502
:10EB200001CDC167FD179305F00F6307F5009750FE
:10EB30000000E78060DEAA85480097D0FFFFE780ED
:10EB4000C03683456404480097D0FFFFE780E03576
:10EB500083457404480097D0FFFFE78000355000DC
:10EB600001478146CE854A8597B0FFFFE780E07078
:10EB700005611733FFFF67002358814481B71733BE
:10EB8000FFFFE702C35583C7950093F7F707A384F8
:10EB9000F50097000000E78020ED1733FFFF6700C6
:10EBA00043561733FFFFE702E35183C79500411136
:10EBB000404D93F7F707A384F5002A8A3285B28483
:10EBC000AE8997D0FFFFE780003E2A8B268597D03D
:10EBD000FFFFE780403D2A89268597D0FFFFE78029
:10EBE000603A93170B0163CA0702E177CA97C2071D
:10EBF000C183116763E3E70293070910C207C1836A
:10EC00001307B00F637BF70093170901C187AA8A26
:10EC1000634AF000C54763FE570141011733FFFF08
:10EC20006700834D97B0FFFFE7802025E31725FF9E
:10EC3000D5B763080B0263060902814463890A029F
:10EC4000B7077F0023106405231124057CC0568577
:10EC500097000000E780E0C39304803EB304950270
:10EC600039A0B7077F00232004047CC081440355EA
:10EC7000240497E00000E780A0A3A1C497C0FFFF91
:10EC8000E78060B7269593D7F44133379500AE9768
:10EC9000BA9708DC5CDCCE85528597000000E780DF
:10ECA000A0DC99E023220404A1679387B7034800FE
:10ECB0003EC42302010002C697E0FFFFE780800503
:10ECC000A9BF814701481CDC232E0403E9B7173391
:10ECD000FFFFE702C34097C0FFFFE7802034E14712
:10ECE0003305F502914597500000E78000C5E557D0
:10ECF00011C59777FF1F23A7A71081473E851733BC
:10ED0000FFFF6700034085471777FF1F230EF70EAD
:10ED100082801733FFFFE702833C9777FF1F9387BB
:10ED2000270E80433DC0835704046390A706835792
:10ED30002404639CB7043689B28497C0FFFFE78040
:10ED400080AB5C5C63C3B7046395B7001C5C63EE87
:10ED5000A7028347640463F3F400A6872303F40443
:10ED60008347740463F39700A687A303F4048357CF
:10ED7000440441677D176385E70085072312F40487
:10ED80003C4481C7CA85268582971733FFFF6700F9
:10ED900043379777FF1F9387A7069C43014599C385
:10EDA00003C5870082801733FFFFE7024333011159
:10EDB000B70707003EC683C79500584D0AC493F7AE
:10EDC000F7070AC8A384F5002A89AE8411CB1C4238
:10EDD00083C707002304F70097900000E780003402
:10EDE000216493055402280097B0FFFFE780802339
:10EDF00097000000E78020FAAA85280097D0FFFF3F
:10EE0000E780A00A300001478146A6854A8597B071
:10EE1000FFFFE780804613044402480822CC230AFF
:10EE2000010002CE97E0FFFFE780C0EE05611733D7
:10EE3000FFFF6700032D1733FFFFE702432A01118D
:10EE40007C003ECAB70707003ECC7C003ECE83C79D
:10EE500095002E84AA8493F7F707A384F500A16593
:10EE600093855502480897B0FFFFE780A01B9700E5
:10EE70000000E78040F2AA85480897D0FFFFE780AE
:10EE8000C002500801478146A285268597B0FFFF42
:10EE9000E780A03E05611733FFFF67008326977761
:10EEA000FF1F9387E7F59C43094599C303C5970066
:10EEB00082809777FF1F9387A7F49C43094599C3E6
:10EEC00003C5D70082809777FF1F938767F39C4322
:10EED000014599C303C5A70082801733FFFFE702EE
:10EEE000631E0111B70708003EC683C79500404D59
:10EEF0000AC493F7F7070AC8A384F5002A89AE84E9
:10EF000029C41442854703C7060063E0E70A834724
:10EF10009400094681496380C702B307F740A30400
:10EF2000E400B339F00083C716002305F40097907E
:10EF30000000E780A01E03572403058B19C76386D2
:10EF4000090097D00000E78000E92164930584025E
:10EF5000280097B0FFFFE780E00C97000000E780F3
:10EF600040F4AA85280097D0FFFFE78000F49700BF
:10EF70000000E78080F5AA85280097D0FFFFE78092
:10EF8000C0F2014781463000A6854A8597B0FFFF51
:10EF9000E780A02E13047402480822CC230A010043
:10EFA00002CE97E0FFFFE780E0D605611733FFFF51
:10EFB000670083141733FFFFE702631201117C001F
:10EFC0003ECAB70708003ECC7C003ECE83C7950002
:10EFD0002E84AA8493F7F707A384F500A16593858F
:10EFE0008502480897B0FFFFE780C0039700000044
:10EFF000E78020EBAA85480897D0FFFFE780E0EA8A
:10F0000097000000E78060ECAA85480897D0FFFFD2
:10F01000E780A0E9500801478146A285268597B080
:10F02000FFFFE780802505611733FFFF6700630D51
:10F030009777FF1F9387C7DC9C43014599C303C59E
:10F04000B70082801733FFFFE70263090111B7079A
:10F0500007003EC683C79500404D0AC493F7F707E3
:10F060000AC8A384F5002A89AE8405C81C42054756
:10F0700083C707006368F7060347B400630FF70010
:10F08000A305F40097900000E78040098347B4008F
:10F09000B9CF97D0FFFFE78040BE21649305B4004D
:10F0A000280097B0FFFFE780E0F797000000E780B7
:10F0B00060F8AA85280097D0FFFFE78000DF0147AE
:10F0C00081463000A6854A8597B0FFFFE780E01AA9
:10F0D0002904480822CC230A010002CE97E0FFFF52
:10F0E000E78040C305611733FFFF6700830197D0B6
:10F0F000FFFFE78020BF55B71733FFFFE70223FE6E
:10F1000001117C003ECAB70707003ECC7C003ECE12
:10F1100083C795002E84AA8493F7F707A384F5008C
:10F12000A165AD05480897B0FFFFE780A0EF970005
:10F130000000E78020F0AA85480897D0FFFFE7800D
:10F14000C0D6500801478146A285268597B0FFFFAB
:10F15000E780A01205611733FFFF670083FA9777F6
:10F16000FF1F9387E7C99C43094599C303C5C7009F
:10F1700082801733FFFFE70283F601117C00AE8423
:10F180003ECAA165B70707002A843ECCD1057C00A2
:10F1900048083ECE97B0FFFFE780C0E89700000028
:10F1A000E78020FCAA85480897D0FFFFE780E0CFE2
:10F1B000500801478146A685228597B0FFFFE7806A
:10F1C000C00B05611733FFFF6700A3F31733FFFF81
:10F1D000E702E3F083C7950093F7F707A384F500F0
:10F1E00097000000E78020F91733FFFF670063F105
:10F1F0001733FFFFE70203ED83C795000329C5011D
:10F20000411193F7F707A384F5001C4283C9070057
:10F21000854763E637079777FF1F938767159C43FA
:10F220002E84AA8485CF97000000E78080F3894769
:10F230006306F502630409028347C900638037034C
:10F240002306390197900000E78040ED835729039A
:10F25000898B89C797D00000E780E0B72685A28513
:10F2600097000000E78020F1A167CD0748003EC469
:10F270002302010002C697E0FFFFE780A0A9410139
:10F280001733FFFF670043E79777FF1F938747B761
:10F290009C431D4599C303C5E70082801733FFFFD8
:10F2A000E702E3E30111B70707003EC683C79500F5
:10F2B000584D0AC493F7F7070AC8A384F5002A89B2
:10F2C000AE8415C71C4283C7070093968701E18669
:10F2D00063C4060685466381D7068346E7006388D4
:10F2E000F6002307F70097900000E78020E32164F1
:10F2F0009305E400280097B0FFFFE780A0D29700B5
:10F300000000E780A0F8AA85280097D0FFFFE780DB
:10F31000C0B9014781463000A6854A8597B0FFFFF6
:10F32000E780A0F53504480822CC230A010002CE6C
:10F3300097E0FFFFE780009E05611733FFFF67003E
:10F3400043DC1733FFFFE70283D901117C003ECA7B
:10F35000B70707003ECC7C003ECE83C795002E84C5
:10F36000AA8493F7F707A384F500A165B9054808B7
:10F3700097B0FFFFE78000CB97000000E78000F127
:10F38000AA85480897D0FFFFE78020B250080147C0
:10F390008146A285268597B0FFFFE78000EE0561D4
:10F3A0001733FFFF6700E3D51733FFFFE70283D171
:10F3B000AA8401441779FF1F1309C9A4E14997C022
:10F3C000FFFFE780A0C56344A400014519A83305E9
:10F3D0003403832709003E958357250063979700E0
:10F3E00011051733FFFF670023D10504C9BF032EA2
:10F3F0008500630A0E121773FF1F130363BF0323F5
:10F4000003006315030029436390061203234E0192
:10F41000631503001D43639907101733FFFFE702CD
:10F4200083C9C689428A3E89BA8AB684328BAE8B3A
:10F430002A84B5E103554E0019E501431A851733B7
:10F44000FFFF6700C3CAA167A98F116763FBE700CD
:10F4500097000000E78080F5814597F0FFFFE78087
:10F46000C0120844B70700E05841F98F18455CC145
:10F47000B707001FF98F1CC55C4991C7610597E06C
:10F480000000E780408BE38A09FA2285979000000C
:10F49000E78060C65DB7328597C00000E7804043D3
:10F4A0000D4349DD1C44116703D54700A167A98FAF
:10F4B00063FBE70097000000E78040EF814597F08D
:10F4C000FFFFE780800C0323840093164B01D18259
:10F4D0008347B300035663008588FD8BA305F300C3
:10F4E000FD777D8E558EFD76FD16B204F18E832755
:10F4F0004301C58E231273012313D3002304530148
:10F5000023052301A3044301BDDF228597B0FFFF3C
:10F51000E78080C9AA850844B5D1610597D000006D
:10F52000E780207F8DB71D431A8582801733FFFF48
:10F53000E70243B90569AA84AE89328A0144FD5ABB
:10F540007D1997C0FFFFE78020A26347A400014513
:10F550001733FFFF670043BAD84493171400BA97D4
:10F5600003D70700631F37032390570163070A007F
:10F57000268597900000E780A0809C449DC383D798
:10F580006700B3F72701639E3701D288014881479E
:10F590000147814601468145268597000000E780A6
:10F5A00040E5050479BF1733FFFFE702A3B1797186
:10F5B0001C103EC4B7070F003EC61C103EC883C7D0
:10F5C0009500AA8A328593F7F707A384F5002E8960
:10F5D000328497D0FFFFE780009D93170501C18714
:10F5E000635AF006AA89228597D0FFFFE780A09B87
:10F5F0002A8A4E85032B040097B0FFFFE7806097AF
:10F6000039ED8357440081440544F11793B717003F
:10F61000A303F10083457100DA872287D2864E86E4
:10F62000280097E0FFFFE780E05701478146300060
:10F63000CA85568597B0FFFFE78020C4A1679387EE
:10F64000F70348083ECC230A810026CE97D0FFFF5F
:10F65000E780406C45611733FFFF6700E3A9A2858F
:10F660001306710097E0FFFFE7806066AA840944F3
:10F6700055D1528597E0FFFFE78060D40D4459D9FA
:10F680000546D285268597000000E78060EA2A8437
:10F6900051B71733FFFFE70283A4835507000346E2
:10F6A000270041112A842E8532C62EC497E0FFFF21
:10F6B000E780E0D001C93246A245228597000000CC
:10F6C000E78000E741011733FFFF670083A317338B
:10F6D000FFFFE702439E83C795004111AA8A93F773
:10F6E000F707A384F5003285AE89328497D0FFFFF7
:10F6F000E780608B93170501C1876357F00AC14506
:10F700002A8A228597C0FFFFE78080702A8D228594
:10F7100097D0FFFFE78020892A89228597D0FFFFB5
:10F72000E7804086930705F893F7F70F1307E00784
:10F73000AA8B637BF706228597D0FFFFE780808442
:10F740002A8C228597D0FFFFE780C083AA8C528540
:10F75000032B040097B0FFFFE780A08139E98357AE
:10F760004400231101008144F11793B71700A3004F
:10F77000F10005440347110083562100938784005C
:10F780005685DA8822885286CE8597F0FFFFE7807B
:10F7900020A7A167E90748003EC42302810026C6CE
:10F7A00097D0FFFFE780005741011733FFFF670045
:10F7B000039413061100A28597E0FFFFE780205114
:10F7C000AA8409E52311010009446DB793052100BE
:10F7D0006A8597F0FFFFE780A0F02A8441FD8355FA
:10F7E00021009356C9001316490185486688E287AF
:10F7F0005E87858A5182268597000000E78060BF7A
:10F800002A848DBF1733FFFFE702E38A83C7950081
:10F8100041112A8B93F7F707A384F5003285AE894F
:10F82000328497C0FFFFE780007893170501C187F6
:10F830006352F00A2A8A228597C0FFFFE780A076EC
:10F84000AA8A228597C0FFFFE780E0752A89228572
:10F8500097C0FFFFE7800073930705F893F7F70F52
:10F860001307E0072A8C6377F706228597C0FFFF0E
:10F87000E7804071AA8C228597C0FFFFE7808070E7
:10F880002A8D5285832B040097A0FFFFE780606ECE
:10F8900039E58357440085440144F11793B71700B5
:10F8A000A301F10003473100930784005A85DE88E5
:10F8B0002688D6865286CE8597F0FFFFE780409453
:10F8C0008D4748003EC42302910022C697D0FFFF17
:10F8D000E780404441011733FFFF67004381A28561
:10F8E0001306310097E0FFFFE780603E2A848944D9
:10F8F00055D99356C9001316490185486A88E68789
:10F900006287858A5182D68597000000E78060AEC5
:10F91000AA8449BF1723FFFFE702C37A2A898144DB
:10F920000144617A916A176BFF1F130B6B6C97B0E0
:10F93000FFFFE780606463C7A40022851723FFFFF1
:10F940006700837B8327090093991400CE9703D522
:10F95000070033074501420741836364570305C12C
:10F9600003270B0019C785453E8597400000E780B7
:10F9700060E9832709000504CE97239007008504DA
:10F980007DB797000000E78060A283270900050487
:10F99000CE972390070065D5814597F0FFFFE7805C
:10F9A000C0BEF1BF1723FFFFE702C37183C79500F5
:10F9B00041112A8A93F7F707A384F50032852E892F
:10F9C000328497C0FFFFE780005E93170501C1876F
:10F9D000635AF004AA89832A040097A0FFFFE780F6
:10F9E000405931E58357440085440144F11793B7EA
:10F9F0001700A301F10003483100D6875285014763
:10FA0000CE862686CA8597D0FFFFE780806AA167E9
:10FA1000F50748003EC42302910022C697D0FFFF9D
:10FA2000E780402F41011723FFFF6700E36CA285A9
:10FA30001306310097E0FFFFE78060292A8489449C
:10FA40005DD99767FF1F9387A75A9C4381CF0449CD
:10FA500097B0FFFFE7804052AA85268597400000B7
:10FA6000E78040DA1305040197000000E780C0EA50
:10FA7000228597800000E78000338144ADBF1723C3
:10FA8000FFFFE702436383C795004111AA8A93F7FA
:10FA9000F707A384F5003285AE8932842311010073
:10FAA00097C0FFFFE780205093170501C18763547B
:10FAB000F0062A8AC145228597C0FFFFE7804035BE
:10FAC000AA8B5285032B040097A0FFFFE780604AB2
:10FAD00021E98357440085440144F11793B7170087
:10FAE000A300F1000348110003572100DA8756856F
:10FAF000D2862686CE8597D0FFFFE780805BA16700
:10FB00009387270248003EC42302910022C697D063
:10FB1000FFFFE780202041011723FFFF6700235DDF
:10FB2000A2851306110097E0FFFFE780401A2A84A0
:10FB300089444DD99767FF1F9387874B98433E8928
:10FB400001CF044997B0FFFFE7800043AA852685CF
:10FB500097400000E78000CB1305040197000000E8
:10FB6000E78080DB97B0FFFFE780004195443DD9F7
:10FB7000930521005E8597F0FFFFE78060B6AA84B9
:10FB800035F11C480357210022852390E700978018
:10FB90000000E780402183270900A9D703552100F1
:10FBA00097400000E780A0BD35BF1723FFFFE702A5
:10FBB000835083C795004111AA8A93F7F707A3845E
:10FBC000F5003285AE89328497C0FFFFE780A03D03
:10FBD00093170501C1876351F0062A8A228597C0D1
:10FBE000FFFFE780403C2A895285032B040097A041
:10FBF000FFFFE780003831E5835744008544014426
:10FC0000F11793B71700A301F10003483100DA8719
:10FC100056854A87D2862686CE8597D0FFFFE78015
:10FC20004049A167F90748003EC42302910022C65B
:10FC300097D0FFFFE780000E41011723FFFF670009
:10FC4000034BA2851306310097E0FFFFE7802008F1
:10FC50002A8489445DD99167CA97C2071167C18315
:10FC60001307F7EF8544E362F7FA9767FF1F93875F
:10FC700027389843BE8B01CF044997B0FFFFE78038
:10FC8000A02FAA85268597400000E780A0B713051E
:10FC9000040197000000E78020C897B0FFFFE780CD
:10FCA000A02D95443DD11C482285814423902701F5
:10FCB00097800000E780200F83A70B00B9D74A8503
:10FCC00097400000E780A0AB89B71723FFFFE7024A
:10FCD00003412A844105B28497000000E780C0C335
:10FCE00011C5228597800000E780E00B8146014620
:10FCF000A685228597800000E780C04E1C4C89C7EE
:10FD0000DC4799C3228582971723FFFF6700633F73
:10FD10009767FF1F9387C70E9C43014599C31385BF
:10FD2000070182809767FF1F9387870D8843828032
:10FD30001723FFFFE702A33A9317C600DD8DC20524
:10FD40004111C1812A8432C697C0FFFFE780E017C6
:10FD50003246228511829375F60F97C0FFFFE78028
:10FD6000C01441011723FFFF6700A3391723FFFFCA
:10FD7000E702433579713C083ED2B7070C003ED408
:10FD80003C083ED683C79500AE842A8993F7F707CF
:10FD9000A384F500A16593853504481097A0FFFF63
:10FDA000E7804028C165FD150144176AFF1F130A4B
:10FDB000AA25930A400EAE892E8B2EC697B0FFFF60
:10FDC000E780801E4205931704014181C183B2453B
:10FDD00063E9A702C167FD176387F500481097C064
:10FDE000FFFFE780800E501001478146A6854A85B7
:10FDF00097A0FFFFE780604845611723FFFF67007A
:10FE0000A32F3307540383270A0BBA9703D6C701DE
:10FE1000630A3601638A3501481097000000E780C5
:10FE200060F1DA85050451BFB285EDBF1723FFFFEE
:10FE3000E702632879717C083EC8B70711003ECA03
:10FE40007C083ECC83C79500AA89328593F7F707D3
:10FE5000A384F5002E8997C0FFFFE780C014856753
:10FE60006378F504A165AA848905080897A0FFFFB7
:10FE7000E780401B268597400000E78060ED133443
:10FE800015000A04A285080897C0FFFFE780E0017B
:10FE9000A685080897C0FFFFE780200325CC01470F
:10FEA00081461008CA854E8597A0FFFFE780E03C99
:10FEB00045611723FFFF67008323B307540303271C
:10FEC000CA0ABA9703D70700631C970003D6270016
:10FED00063806505080897000000E780A0E5DE85DF
:10FEE00005042EC697B0FFFFE780000D420593176B
:10FEF00004014181C183B245E3E1A7FCC167FD175D
:10FF0000E38FF5F8080897C0FFFFE78000FC41BFCA
:10FF1000B285F9B7C165FD150144176AFF1F130AC1
:10FF2000AA0E930A80022E8BAE8B65BF1723FFFFAC
:10FF3000E702E31A18418347170083460700A20728
:10FF4000D58FD207D1832390F5008347270003473D
:10FF500017008D45A207D98F91832310F60097C013
:10FF6000FFFFE780A0E91723FFFF6700831917232E
:10FF7000FFFFE7022315C16401441769FF1F13093E
:10FF8000A90893098002FD1497B0FFFFE780C00223
:10FF90006347A40001451723FFFF6700E3153305FE
:10FFA00034038327C90A3E9583570500E38597FEEE
:10FFB0000504D9BF1723FFFFE702C3102A8AAE89C1
:10FFC000B284B68A97400000E78080D819E591474F
:10FFD0003E851723FFFF670023122A894E8597C0AD
:10FFE0000000E780E08E2A84638E0A048D476DD17D
:10FFF00003570500C547E31D47FD0347F901854643
:020000040001F9
:10000000AD47E317D7FC8347450081CF4146A6851E
:100010005D0597F00000E780C09E814755D9AD4748
:1000200045BF130965012302E500CA85268597109F
:100030000000E780606231C1A547E38B0AF8230224
:10004000040079B705C183570500E39247F941469B
:10005000A685190597F00000E780A09A81472DD961
:100060009947BDB74E8597000000E78080F02A844D
:10007000954739DD130955004DBF4146A68523102C
:100080004401231134011305190097F00000E780A3
:10009000A099228597800000E780A0EA81470DBFE4
:1000A0001723FFFFE702A30379717C003ECCB7075B
:1000B0000A003ECE7C003ED083C79500B2842E84D9
:1000C00093F7F707A384F5001306A1002A892C00F3
:1000D000268597000000E780A0E5A16528088D052A
:1000E00097A0FFFFE78000F490408355A1000355DF
:1000F0008100854697000000E78000ECAA84AA856D
:10010000280897C0FFFFE78040DA0356A100835517
:100110008100280897000000E780C0C1300801472F
:100120008146A2854A8597A0FFFFE7800015854795
:1001300048103ED42302910202D697D0FFFFE780F9
:1001400060BD45611723FFFF6700A3FB1723FFFF77
:10015000E702E3F879717C003ECCB7070A003ECE97
:100160007C003ED083C79500B2842E8493F7F707B6
:10017000A384F5001306A1002A892C002685970088
:100180000000E780E0DAA16528088D0597A0FFFF51
:10019000E78040E990408355A100035581008146E6
:1001A00097000000E78040E1AA84AA85280897C04C
:1001B000FFFFE78080CF0356A10083558100280808
:1001C00097000000E78000B7300801478146A2850C
:1001D0004A8597A0FFFFE780400A4810230291025A
:1001E00002D402D697D0FFFFE780C0B24561172343
:1001F000FFFF670003F11723FFFFE70243EE9700BD
:100200000000E78060DB1723FFFF670083EF97673D
:10021000FF1F938727BF884382801723FFFFE702D2
:1002200003EC835725004111AE842A842307B100D3
:1002300017F5FFFF130525466C002316F10097A064
:10024000FFFFE780804591C4228597800000E7800A
:10025000E0D6FD572310F400130620028145130554
:1002600054009720FFFFE78080EA41011723FFFF3A
:10027000670023E91723FFFFE702C3E479717C00DD
:100280003ECCB7070A003ECE7C003ED083C7950027
:10029000AA89AE8493F7F7073285A384F500130685
:1002A000A1002C0097000000E78080C80355810062
:1002B000114497400000E780A0A915C50355A1008F
:1002C000014497B00000E780A06011CD03570500FE
:1002D0008357810045446318F70085459700000067
:1002E000E780E0F30144216993053900280897A0CD
:1002F000FFFFE78020D3A285280897C0FFFFE78093
:10030000C0BA0356A1008355810028089700000059
:10031000E78040A2300801478146A6854E8597A018
:10032000FFFFE78080F548104AD42302810202D6FD
:1003300097D0FFFFE780009E45611723FFFF67000E
:10034000A3DB1723FFFFE702E3D79767FF1F93871E
:1003500027AB2A8488432E8915C503574503835745
:10036000C4016311F7022326050223180502410583
:1003700097D00000E780209C63060900978000006A
:10038000E78060DB81449769FF1F9389E9C7130AFF
:10039000800297B0FFFFE78020C263C4A404976780
:1003A000FF1F9387A7AE9C4399C70355C4019720AD
:1003B0000000E780C0BD6307090022859780000028
:1003C000E780C0A01306400E814522859720FFFFDD
:1003D000E780E0D3FD57231EF4001723FFFF6700DB
:1003E000A3D13385440383A7C90A3E95035705006B
:1003F0008357C4016317F700CA8597000000E780A0
:1004000000E2850479B71723FFFFE702A3CB83C778
:1004100095004111AA8993F7F707A384F500328567
:10042000AE8497C0FFFFE78000B885676378F50466
:100430002A8997400000E780A091014401CD83D72D
:100440000400314463882701854597000000E78058
:1004500080EF01444E85A2864A86A68597D0FFFF8D
:10046000E780A09CA1679387170448003EC423023D
:10047000810002C697D0FFFFE780C08941011723A2
:10048000FFFF670063C71723FFFFE702A3C3976758
:10049000FF1F9387E796804329C4014597C000005A
:1004A000E780002181470148C1641CDC232E04033E
:1004B000232004041769FF1F130909B50144930998
:1004C000400EFD1497B0FFFFE78000AE634FA4001D
:1004D000814517F5FFFF1305857F97A0FFFFE78094
:1004E000C01B1723FFFF670023C133053403832795
:1004F000090B3E958357C501638797008545970093
:100500000000E78040E4050475BF9357050113D749
:100510008700A380F50093170501C183A183238081
:10052000E5002381F500A381A50082801723FFFF4A
:10053000E702E3BA2300050083C71500A300F50016
:1005400083C725002301F50083C73500A301F5000B
:1005500083C745002302F50083C75500A302F500B9
:1005600083C7650093059500A30305002303F500E9
:1005700023040500328597000000E78040F9172327
:10058000FFFF670003B81723FFFFE702A3B3411182
:10059000E9540DCD85CD93F9C5FF2E842A89AA840F
:1005A000338AA900B7EA040063189A020D888544CB
:1005B00011CCB7E704009C5F82972AC622866C00A4
:1005C0003305390197E00000E780004626854101A8
:1005D0001723FFFF670043B283A78A039104829722
:1005E00093170501C183A183A38EF4FE93570501E0
:1005F000238FF4FEA183238EA4FEA38FF4FE6DB798
:1006000063E6D5021723FFFFE70263ADB28741110E
:100610003686BE8536C697E00000E780E040B246E9
:10062000410136851723FFFF6700A3AD814636855C
:100630008280838705001387F5003D05FD8793F7CA
:100640007708834607007D158606B58FA300F50061
:100650006307B7007D17834717009D83DDB782804E
:100660001723FFFFE702A3A7B7E7040083A7070943
:1006700032872A863A858297133515001723FFFFA4
:10068000670023A815C181478DC11723FFFFE7022B
:1006900003A5414697E00000E780003985473E8585
:1006A0001723FFFF6700E3A581473E8582801DCDAC
:1006B0001723FFFFE702A3A2414681452A84972022
:1006C000FFFFE780C0A4414681451305040397203E
:1006D000FFFFE780C0A30147C1672322040438C895
:1006E0007CC805451723FFFF6700A3A10145828051
:1006F00081473DCDB5CD1723FFFFE702439EB2846E
:100700002E891306800581452A849720FFFFE78004
:1007100000A0CA8524C4268597000000E780C0F6A3
:100720004146814522859720FFFFE780409E304467
:10073000A285228597000000E780C0F2930404019F
:10074000A285268597000000E780E0EEA6851305C8
:10075000040297000000E78000EE22859700000069
:10076000E78020F585473E851723FFFF67006399E3
:100770003E8582801723FFFFE702C3944111E954AD
:100780000DCD85CD93F9C5FF2E842A89AA84338A9D
:10079000A900B7EA0400639844030D88814411CC92
:1007A000B7E704009C5F82972AC622866C00330557
:1007B000390197E00000E7802027268541011723B3
:1007C000FFFF6700639383A78A03910482979317BF
:1007D0000501C183A183A38EF4FE93570501238FE6
:1007E000F4FEA183238EA4FEA38FF4FE6DB765CD26
:1007F0001723FFFFE702038DB28411E60545172397
:10080000FFFF6700638F2A842E890145EDD93C489C
:100810007848B3E6E700E5D69386F7FFB3B7F6006E
:100820007D17032A4404BA9734C87CC863050A06B6
:10083000C14913050A03B38949412295637D3601F5
:10084000B2862E86A68597000000E780A0DB7C405C
:10085000BE9464C065B7CE862E86CE859700000014
:10086000E78040DAC114D2944E9923220404A2876F
:100870009306040103C7070003C607038507318FEA
:10088000A38FE7FEE398F6FE3044A2852285970009
:100890000000E78020DD2699C1493306994063ECCA
:1008A0009900A9DCA686A68513050403970000001D
:1008B000E78040D579BF8147B306F4003307F600DF
:1008C0000347070083C5060085072D8F2380E600B8
:1008D000E39437FF3044A285228597000000E7802B
:1008E00060D8C1145DBF014582800DC11713FFFFA1
:1008F000E702E37E1306800581459720FFFFE7802E
:10090000008105451713FFFF6700A37F0145828023
:10091000814749C5C1C51713FFFFE702437CFC416E
:1009200041462E84AA846399C70413860501A287D1
:100930008146C14503C7070003C507038507298F03
:100940003305D600034505008506298FA38FE7FEF2
:10095000E392B6FE3044A285268597000000E7802A
:1009600060D0228597000000E78060F885473E85CB
:100970001713FFFF6700E378138507031D8E81457A
:1009800022959710FFFFE78080787C40130700F8DE
:1009900013060402A2972388E70251BF3E85828096
:1009A0001713FFFFE702A3736D712E84B284AA852B
:1009B00090102800368997000000E780A0D309ED49
:1009C000D55725A050400C40280097000000E78034
:1009D00040E27DD5FD142104F5F42C004A859700F2
:1009E0000000E78020F3814761DD3E8551611713E8
:1009F000FFFF670003711713FFFFE702436E41110A
:100A00002EC432C62C00054697000000E78080F90E
:100A100041011713FFFF6700C36E1713FFFFE702C3
:100A2000036C01112A842EC602C802CA02CC02CE6F
:100A300097E00000E780C023B2462A86A285080816
:100A400097000000E78060FB1375F50F0561171331
:100A5000FFFF6700036B1713FFFFE702436879711D
:100A6000B2872A8421462308B10013051101BE85EF
:100A70003AC436C697E00000E78000FBB246930513
:100A80009101368597000000E78060A82285141048
:100A900035460C0897000000E78020F62A8422479C
:100AA00001E921460C103A8597E00000E780C0F785
:100AB000228545611713FFFF6700A3641713FFFF2B
:100AC000E702E3617171AE84AA850A8532849700DA
:100AD0000000E78060BB11C90A86A68522859700C1
:100AE0000000E78020B8814711E1C5473E854D6190
:100AF0001713FFFF6700E3601713FFFFE702235B95
:100B00001D712A8AB289BE843546854713051101B5
:100B10002E8CB68A3A8BC28C468D2308F10097E062
:100B20000000E78060F010100C085285231F0100C0
:100B300097000000E780C0F82A843DEDA1476313C9
:100B4000FD089307900591E0E5473546E2851305DA
:100B5000110113990A012308F1001359090197E0C3
:100B60000000E78060EC1357890093978A00D98FC3
:100B700090080C085285231FF10097000000E780C1
:100B800020F42A8415E9A1E49387FA00918313796C
:100B9000F9003EC6631309004149668B8144C14B8D
:100BA000854DB247639F970C6A868C0033855C0144
:100BB00097E00000E78040E7228525611713FFFFDB
:100BC0006700A35293079004C9F0A547BDBF8347B0
:100BD00001050947C14B2308F10083471105A58F83
:100BE000A308F10093872400814463E1FB040147DB
:100BF00014083386E6008C08B386E400BA95DA96CA
:100C000083C6060083C505000507AD8E2300D60008
:100C1000E390E7FE4147639CE70490080C08528587
:100C200097000000E780C0E925D181A0B3069B00B2
:100C3000BA871008B305F60090083E9603C5060073
:100C40000346060085078506298E2380C500E392AA
:100C500077FF998F90080C085285BE94970000008A
:100C6000E78000E68947014749D12A84B1B7900857
:100C70003E96034606001408BE962380C6008507EC
:100C800059BFB24785046387971481471808B30694
:100C9000F70098083E973386F9000347070003469C
:100CA00006008507318F2380E600E39177FF9008E7
:100CB0000C08528597000000E78080E05DF535461E
:100CC000E285130511012308B10197E00000E780D8
:100CD000A0D5139704014183939784002183D98F72
:100CE00010180C085285231FF10097000000E780C0
:100CF00020DD25FD814710183387F9003E96034714
:100D0000070003460600B306FB008507318F2380EA
:100D1000E600E39277FF65A81808B306F700980885
:100D20003E973386F9000347070003460600850710
:100D3000318F2380E600E3E127FFCA87639E7709AE
:100D400090080C08528597000000E78060D711FDDD
:100D500081479800B306F700900818103E973E961A
:100D600003470700034606008507318F2380E6000E
:100D7000E39177FF3546E285130511012308B101A0
:100D800097E00000E78040CA1397040141839397DE
:100D900084002183D98F10180C085285231FF1007D
:100DA00097000000E780C0D1E31105EC81471018DF
:100DB0003387F9003E960347070003460600B30653
:100DC000FB008507318F2380E600E3E227FFC1099E
:100DD000410BC1BB814785B79408BE9683C6060008
:100DE00018083E972300D700850789BF6380063225
:100DF0001713FFFFE702A32B59712A84BE89B28B18
:100E000085473546130511022E8B468C4289BA8AD6
:100E1000368A2300F10297E00000E780E0C0101856
:100E20000C1022852317010297000000E78040C9BB
:100E300063180512A147631FFC069307900563938F
:100E40000900E5473546DA851305110293140A01B6
:100E50002300F102C18097E00000E780E0BC931717
:100E60008A0013D78400D98F90080C10228523178D
:100E7000F10297000000E780A0C47DE163920904BD
:100E80009307FA00BD88918391E0C144C207C183F2
:100E9000DE8C814A3EC6414DB24763E2FA0E62865D
:100EA000B3854B01881097E00000E78080B54DC9FD
:100EB0003D557DA093079004E39609F8A54759B7DF
:100EC000834701050947C14C2300F10283471105FF
:100ED000B3C7F900A300F10293872900814963E1B8
:100EE000FC04814618103306D7008C083387D900DC
:100EF000B69556970347070083C5050085062D8FD5
:100F00002300E600E390D7FE41476390E706900890
:100F10000C10228597000000E78080BA35D189A0A7
:100F2000B3863A01BA871010B305F60090083E96D2
:100F300003C506000346060085078506298E238023
:100F4000C500E39297FF3387EC4090080C10228590
:100F5000BA9997000000E780A0B68947014741D1C0
:100F600065611713FFFF6700431890083E9603461C
:100F700006001410BE962380C600850779B7B247D5
:100F8000850A93990A01939D8A0093D90901639177
:100F9000570F85473546DA85130511022300F10204
:100FA00093D9890097E00000E78000A8B3ED3D01E8
:100FB00090000C1022852317B10397000000E780F2
:100FC00020B059FD8147A68963EA970626860C085A
:100FD0004A8597E00000E78020A581471810B306F6
:100FE000F700100898083E973E960347070003460F
:100FF00006008507318F2380E600E3E197FE639FBB
:10100000A90590080C10228597000000E78040ABEE
:1010100021F981479810B306F700900818183E97F9
:101020003E9603470700034606008507318F23805D
:10103000E600E391A7FF4109C10CB9BD1808900073
:10104000B306F7003E963387FC00034707000346CC
:1010500006008507318F2380E600B5B798084E97C4
:10106000034707001C10CE972380E700850941BF86
:1010700085473546DA85130511022300F10293D91D
:10108000890097E00000E780209AB3ED3D019000D1
:101090000C1022852317B10397000000E78040A2BF
:1010A000E31005EC814718089000B306F7003E9660
:1010B0003387FC0003470700034606008507318F8E
:1010C0002380E600E391A7FF41460C084A8597E09C
:1010D0000000E780609581471810B306F7001008FC
:1010E00098083E973E96034707000346060085078B
:1010F000318F2380E600E391A7FF90080C10228532
:1011000097000000E780C09B1DD599BD7D5582806A
:101110001713FFFFE702A3FC01112A842E85930514
:101120005100328902C002C202C402C69304740094
:1011300097F0FFFFE780A03D1D46A68513059100AF
:1011400097E00000E780408E10088A854A85970066
:101150000000E780E09619ED93071400180883C695
:1011600007000346070085070507B18EA38FD7FE4A
:10117000E397F4FE05611713FFFF670083F8171369
:10118000FFFFE70223F42E848C414111AA89838753
:1011900015003289914463D30700A1449757FF1F7C
:1011A0009387071D9C43A1C7C1CA8D472310F10037
:1011B00083C725004A852301F10083C73500A301B9
:1011C000F10083C745002302F10083C75500A30245
:1011D000F10083C7650093059100A3030100230379
:1011E000F1002304010097F0FFFFE78040320C403C
:1011F0004A860A8597F0FFFFE780803303280400C2
:1012000083564400A6881D0881470147E51642869B
:101210008A854E8597000000E780408E2A8919E56F
:10122000A685228597B0FFFFE780E0C14A8541018E
:101230001713FFFF670043EC4A860A8597F0FFFF0C
:10124000E780002F6DB71713FFFFE702A3E72E8497
:101250008C414111AA89838715003289914463D357
:101260000700A1449757FF1F938787109C43A1C78E
:10127000C1C68D472310F10083C725004A8523018D
:10128000F10083C73500A301F10083C745002302A5
:10129000F10083C75500A302F10083C765009305E1
:1012A0009100A30301002303F1002304010097F040
:1012B000FFFFE780C0250C404A860A8597F0FFFFB4
:1012C000E780002783564400032804008A85858E22
:1012D000C2061D08C1822312D400A6888147014797
:1012E000E51642864E8597000000E78060B0410118
:1012F0001713FFFF670043E04A860A8597F0FFFF58
:10130000E78000234DBF1713FFFFE70243DDB3352E
:10131000B000011185052A891315F6013365150101
:101320002308B1009305110136843AC632C03EC489
:1013300042C297F0FFFFE780801DA2471248425546
:1013400093D68700230BF1009305910193578800F2
:10135000A30AD100A30BF100230C010197F0FFFFBA
:10136000E780E01A3247024603280400B337E00062
:10137000835644009207914411C2A1444A85A6882D
:1013800042860C0897F0FFFFE78040772A8919E52D
:10139000A685228597B0FFFFE780E0AA4A85056110
:1013A0001713FFFF6700E3D51713FFFFE70283D191
:1013B00001113EC68647B335B0008505AA891315CD
:1013C000F6015D8D2308B1009305110136843A8939
:1013D000B28442C446C297F0FFFFE7804013224820
:1013E0009248164593578800A30AF100930591018E
:1013F00093D78800230B0101A30BF100230C1101EB
:1014000097F0FFFFE780A01032471040835644005A
:10141000B337E000920703280900914891C0A14822
:101420000C084E8597000000E780809CAA8401E9A3
:10143000835544004A8597B0FFFFE780C0A026850A
:1014400005611713FFFF670023CBAA959307F00FE1
:10145000170701001307075B6317B50013C5F7FFF4
:101460001375F50F828005058346F5FFB58FBA9792
:1014700083C70700D5B70357450014419307F00F02
:101480001706010013060658369742074183139545
:1014900006014181631BE500AD8FB29703C50700CC
:1014A000130515F3133515008280850603C5F6FF75
:1014B000A98FB29783C70700D9BF1713FFFFE702B1
:1014C00003C2B28736842E86BA86AA853E85BA8440
:1014D00097F0FFFFE7806052634F0500228597D0A9
:1014E0000000E780E0782A86A686A285268597F008
:1014F000FFFFE78080501713FFFF670083C01713BB
:10150000FFFFE70223BC5D712A8BAE8A170501003D
:101510001305C54C2C00B284368ABA893E8997F0EF
:10152000FFFFE780C04F2A845DE134104146DA8531
:10153000280097F0FFFFE780404C2A8449E985475F
:10154000A303F100A6C2930771002408BEC4A686B7
:1015500085470D462C18281002DC02DED6C0BEC618
:1015600097F0FFFFE78000442A8435E1834771024A
:10157000A6860D4693F7F7072300FA00C1473EDE23
:101580002C188947281026DCA303F10097F0FFFFF1
:10159000E78040412A8405ED4146A6854E8597D0D7
:1015A0000000E78060488D47A6860D462C1828105D
:1015B000A303F10097F0FFFFE780C03E2A8401E912
:1015C0004146A6854A8597D00000E780E045228500
:1015D00061611713FFFF670023B21713FFFFE702D4
:1015E00003B097F700009387E7A0984383C74700AD
:1015F00079712A89AE84170501001305A53E0C08F0
:101600003AC42306F10097F0FFFFE78040412A84A7
:1016100005ED14104146CA85080897F0FFFFE780E2
:10162000C03D2A8415E1140815462C00081097F0D7
:10163000FFFFE780803C2A8401E921462C082685AB
:1016400097D00000E780403E228545611713FFFFD9
:10165000670023AB1713FFFFE70263A897F70000AB
:10166000938747999C477971AA842E8417050100B6
:101670001305C5370C083EC697F0FFFFE780203AF8
:101680000DE914104146A685080897F0FFFFE78092
:10169000C03605E1140811466C00081097F0FFFFF2
:1016A000E780A03519E58347F10193F7F70323009D
:1016B000F40045611713FFFF6700A3A41713FFFF92
:1016C000E702E3A13688A14881470147E54697F044
:1016D000FFFFE780A0421713FFFF670083A21713E5
:1016E000FFFFE702C39F3688A14881470147E546CF
:1016F00097F0FFFFE780C06F1713FFFF670063A03D
:101700001713FFFFE702A39D01112A842E850C0801
:1017100032C697F0FFFFE780803009ED3247970629
:1017200001009386262B1008C145228597000000F2
:10173000E780E0D805611713FFFF6700839C17134C
:10174000FFFFE702C3994111C1472EC032C48A8509
:1017500009463EC23EC697F0FFFFE780A024410144
:101760001713FFFF6700E3991713FFFFE7022397A3
:101770004111AE8613061009AA850A8502C002C26D
:1017800002C402C697F0FFFFE7802027410117132C
:10179000FFFF670003971713FFFFE70243943287A9
:1017A00097060100938606252E8693050002970072
:1017B0000000E780C0D01713FFFF67008394171362
:1017C000FFFFE702C3917971C1472ACC2ED032D4F2
:1017D0002C080D4628003ECE3ED23ED602C402C69C
:1017E00002C802CA97F0FFFFE780C01B45611713CC
:1017F000FFFF670003911713FFFFE702438E0111FC
:10180000AA842E84170501001305451F8A8597F0C9
:10181000FFFFE780C02015E514084146A6850A852C
:1018200097F0FFFFE780601D09ED8347E101034763
:10183000F101A207D98FCA07C9836177D98F231015
:10184000F40005611713FFFF6700A38B15CD171375
:10185000FFFFE702C3889747FF1F9387275F9043E7
:101860009745FF1F9385C55E1745FF1F1305055A52
:1018700097D00000E78000C51745FF1F13050559E5
:101880001713FFFF6700E3871745FF1F1305055870
:1018900082808DCD1713FFFFE70263849747FF1FF8
:1018A0009387C75A944301112E840A869745FF1FD8
:1018B0009385055A97D00000E78040C60A850294B8
:1018C000014505611713FFFF6700A3837D558280E3
:1018D0001713FFFFE702A38097D00000E78080D1B5
:1018E0009747FF1F23A4A75617F5FFFF1305E5C968
:1018F00097B00000E780C0741713FFFF6700638094
:101900001747FF1F1307C7569317150008433E9547
:10191000FD572310F50082801703FFFFE702237CA9
:101920002A84084009E51703FFFF6700837D1C41F7
:1019300058401CC06313E5005CC08347550023205A
:101940000500F99BA302F50097A0FFFFE780207C2C
:10195000C9BF1703FFFFE702E3769747FF1F93878F
:10196000275398432A8411CB8347350093F7070206
:1019700089C703550500894502971305440197B0AF
:101980000000E780403B835504000355E400973096
:101990000000E780A00C485819C597A0FFFFE7801A
:1019A0000077232A04021305840397000000E780D0
:1019B000E0F68144B1499790FFFFE780206A63CB4E
:1019C000A402834734002320040493F727FCA301D7
:1019D000F40000489790FFFFE78040691316150058
:1019E000814522859700FFFFE78060721703FFFFA4
:1019F00067008370B38734030329040385043E9989
:101A00004A8597000000E78060F12304090065B76C
:101A10008347350093F7070299E301458280835796
:101A2000E500E39CB7FEC167FD176316F6000545A8
:101A30008280054599A81703FFFFE702436A9317C1
:101A40000601C187B2842A8401496359F002835791
:101A500005009DCB01456367F600034584003E9574
:101A60003325A6001375F50F0DA01C481317190098
:101A7000BA9783D70700E38E97FA05099790FFFF7F
:101A8000E780C05EE343A9FE01451703FFFF67003F
:101A900043671703FFFFE702E362AE89AA849790CA
:101AA000FFFFE78060522A8497D0FFFFE780A02ED7
:101AB000AA8601471306840197050000938585E4F3
:101AC0001745FF1F1305053B9790FFFFE780E018C0
:101AD0002A8925C98C441304C50022859E0593F5E7
:101AE000050897A0FFFFE780403CCC408387740047
:101AF000E18163DD070493E50508228597A0FFFFD8
:101B0000E780A03A0D4693854400228597A0FFFF09
:101B1000E780C03683D50400228597A0FFFFE780C9
:101B2000E03D83D52400228597A0FFFFE780003D9C
:101B300003D6490083A50900228597A0FFFFE7800F
:101B4000E0334A851703FFFF6700035B93F5F50752
:101B50006DB71703FFFFE702835801112A8432850E
:101B600032C697A0FFFFE780E0279780FFFFE7805E
:101B7000C030835704001747FF1F1307E74832465A
:101B8000231BF100930700F8A30DF1001C47184335
:101B9000231AA1008983858BB307F740B2854808D3
:101BA0003ECE231C0100230D010097000000E780BA
:101BB00080EE05611703FFFF6700A3541703FFFFC3
:101BC000E7024350004101453DC49304C40026850B
:101BD0003289AE8997A0FFFFE780C02495452A8A05
:101BE0002685035B040197A0FFFFE780202126855F
:101BF00097A0FFFFE780603E8D45AA8A268597A0C3
:101C0000FFFFE780A01F268597A0FFFFE780E03C4D
:101C10005C48420A135A0A01D2975CC42318640133
:101C2000814763983A0146054D8133062541933734
:101C3000160013F5F70F1703FFFF6700E34B1703B9
:101C4000FFFFE702434789692A8BAE8B328AB68A47
:101C500081440144314CFD199790FFFFE78000401B
:101C600063CDA4009790FFFFE7804042018D33B51C
:101C7000AA001703FFFF6700834733898403832784
:101C80000B003E9963170A008347890085043E9440
:101C9000E1B703560A00DE854A8533F6C90097008E
:101CA0000000E780E0F16DD10545E1B71703FFFFC4
:101CB000E702E34201112A847C000355E5003ECA95
:101CC000B70707003ECC7C003ECE97200000E7809F
:101CD00020082A898545480897A0FFFFE78020391A
:101CE0009945480897A0FFFFE780E015AA844A8538
:101CF00097200000E780A0082380A4009747FF1FDB
:101D0000938787309C434166130606F093968701BC
:101D100013D78701558F93D68700F18E558FA20771
:101D2000B706FF00F58FD98F11462C0013851400DC
:101D30003EC497D00000E78020CF5008A382040063
:101D40008945228597000000E780E0E019C9AA854F
:101D50001305840397A0FFFFE780E0313C4085072F
:101D60003CC005611703FFFF6700A3391703FFFF9E
:101D7000E702E3369790FFFFE78040312A840504AD
:101D80009790FFFFE780802F3305A402F14791452C
:101D90003305F50297200000E78020BA11E565556C
:101DA0001703FFFF6700E3359747FF1F23AAA70C20
:101DB0009790FFFFE780802D2A8405049790FFFF0E
:101DC000E780C02B3305A402894506059720000053
:101DD000E780A0B669D59747FF1F23ABA708979068
:101DE000FFFFE780A02A2A8405049790FFFFE78081
:101DF000E0283304A4029747FF1F239D870697908E
:101E0000FFFFE780A0282A849790FFFFE780002744
:101E1000930714003385A7029747FF1F239DA7044C
:101E200097070100938747811747FF1F2328F7046F
:101E30000145BDB71703FFFFE702C328AA842E8917
:101E400001449749FF1F9389291C130A8006979024
:101E5000FFFFE780A0226347A40001451703FFFFAF
:101E6000670083293305440383A709024A86A685B0
:101E70003E9597000000E780E0B919E10504C1BF75
:101E80000545E9BF1703FFFFE702E322AA8A2E8B6D
:101E9000B28B368C3A8A814401448149974CFF1FAA
:101EA000938C8C16130D80069790FFFFE780001D22
:101EB00063C9A40011E085494E851703FFFF670041
:101EC00003233389A40383A70C025E86D6853E993B
:101ED0004A8597000000E780E0B31DC19790FFFF9F
:101EE000E780C01A0544636D4501D2866286DA85B3
:101EF0001305090397000000E780A0D411C18549AC
:101F000085045DB71703FFFFE702C31BC1644111DE
:101F10002A8901449749FF1F9389090F130A8006F4
:101F2000FD1436C632C42EC29790FFFFE78000151D
:101F300092452246B2466348A40001454101170379
:101F4000FFFF6700631B3305440383A709023E9527
:101F500009C683473500C18B9DC791C683473500AD
:101F600093F707028DC3630699008357E500639CCE
:101F700027010357050001CB63E7E5008347850090
:101F8000BA97E3CDF5FA050469BF1703FFFFE7022F
:101F90006313C1642A8901449749FF1F9389C906C5
:101FA000130A8006FD149790FFFFE780200D63461B
:101FB000A4001703FFFF670023143305440383A71E
:101FC00009023E958357E500638A970063049900F0
:101FD0006396270197000000E780E0970504E1B7CA
:101FE0001703FFFFE702A30C89692A8AAE8A328BA6
:101FF000B68B8144174CFF1F130C0C01930C800609
:10200000314DFD199790FFFFE780400763C6A4009C
:102010001703FFFF6700630D3389940383270C02C6
:102020008355CA015A863E994A8597000000E78089
:10203000609E31C1814D15A03384AD038327090310
:1020400003D60B00D68533F6C9003E94228597004F
:102050000000E780E0B609E9850D9790FFFFE78073
:10206000E0FFE3CBADFC01A8228597000000E780EC
:10207000E08A23040400850471B71703FFFFE70219
:1020800083034169AA8A014A174BFF1F130BCBF741
:102090007D19C14B054C9790FFFFE78020FE6346FA
:1020A000AA001703FFFF6700830493098006B307A4
:1020B0003A0383290B02BE9983D7E900638E270177
:1020C00063842A01639A570103A4890301E84E85BA
:1020D00097000000E780C0BD050A75BF8357040163
:1020E000639977099304C400268597A0FFFFE780D2
:1020F00060D385452A8D2685835C040197A0FFFF68
:10210000E780C0CF268597A0FFFFE780A0E76205A4
:102110006185635905048D45268597A0FFFFE780FB
:10212000E0CD8945268597A0FFFFE78020CD894532
:10213000268597A0FFFFE78060CC8545268597A080
:10214000FFFFE780E0CC83470500094793F7F707D7
:10215000639AE7009945268597A0FFFFE78040CB6B
:10216000A30285014848337D2D01231894016A9507
:1021700048C40040A1BF1703FFFFE70243F637E45E
:1021800004008327041D82979747FF1F83C7C7D486
:102190001715FF1F13058539A300F5008327441C7D
:1021A00082978327841C81461306F00F81450145E1
:1021B00082971703FFFF6700C3F41747FF1F13073A
:1021C000A7C118439745FF1F83C505D19747FF1F38
:1021D000938707CF83468703034697036397D5000A
:1021E0009747FF1F238AC7CE828083C58701034795
:1021F000A7036317B6009747FF1F238FE7CC8280A2
:1022000003C687016317C7009747FF1F2386D7CCF4
:10221000828083C68701130750026319D700930792
:1022200060021747FF1F2309F7CA828083C6870110
:10223000130660026315D60093077002DDB783C7EB
:10224000870155BF9747FF1F938787C7D44B09471F
:10225000638DE6081703FFFFE70263E81749FF1FD6
:10226000130949C33E8483470900918B9DCFB7E48E
:10227000040083A7041D829783A7441C1745FF1FF2
:102280001305C5C1829783A7841C81461746FF1F8B
:102290000346C6C281450145829721C5834709008F
:1022A000ED9B1747FF1F2307F7BE8347040093F7F3
:1022B000F70F85CB91471747FF1F232DF7C09700D6
:1022C0000000E78080EB97000000E78040EFB7E771
:1022D0000400BC4F414691451745FF1F0345C5BE4D
:1022E00082971703FFFF6700C3E182801703FFFF98
:1022F000E702E3DE8D4741116306F504C547630835
:10230000F50285476310F5029747FF1F2388A7BC96
:10231000B7E70400BC4B930500101745FF1F0345AA
:10232000A5BA829741011703FFFF670083DD854748
:102330001747FF1F2304F7BAB7E70400BC4B930508
:102340000020E1BF9747FF1F938787B7D44B114702
:10235000638DE600B7E7040083A7071D8297B7E700
:102360000400BC4B930500044DBF05491747FF1FF0
:10237000232227B783C7070032C62E8493F7F70FAF
:10238000D5D3B7E4040083A7041D7D141374F40FA0
:102390008297E37689FCB245994703C61500E3F0BE
:1023A000C7FCFC4409061745FF1F130565B3829758
:1023B000BC48930500081745FF1F0345E5B0829709
:1023C00079BF1703FFFFE70283D11747FF1F1307EA
:1023D00027AF4047184B1C409746FF1F23A8F6AE77
:1023E0006316E4001747FF1F2324F7AE130584FE8E
:1023F0009790FFFFE78060A6035564FF9780FFFF7B
:10240000E780E06E97A0FFFFE78060D01703FFFF33
:10241000670023CF1703FFFFE70263CC9747FF1F37
:10242000938707AAD84BDC4789C797000000E7804D
:1024300080F985471747FF1F232EF7A89747FF1FEF
:10244000938787999C43930500021745FF1F034517
:10245000A5A783C787031747FF1F230FF7A6B7E773
:102460000400BC4B82971703FFFF670083C997479F
:10247000FF1F23A9A7A482801703FFFFE70283C4DD
:1024800037E404007C4CA1451745FF1F0345C5A355
:1024900082977C48A1451745FF1F0345E5A2974455
:1024A000FF1F9384E4A18297DC4489EB970000002E
:1024B000E78080D91703FFFF670003C403D567FFD8
:1024C0009780FFFFE780A062AA896DD1D848914725
:1024D0006310F7027C4C91451745FF1F0345C59ECD
:1024E00082977C4891451745FF1F0345E59D8297DC
:1024F00003A9490103D409018947B7E90400174733
:10250000FF1F2329F79C83A7091D210442048297FA
:1025100083C784011715FF1F13054501611917179C
:10252000FF1FA305F70083A7491C418082979747A7
:10253000FF1F2385079A83A7C91C81460946937507
:10254000F40F4A85829711E99747FF1F83C747A970
:1025500089C79700FF1FE780E069B7E70400BC4F19
:102560002146A1451745FF1F03450596829799B758
:102570001703FFFFE702A3B693F7052001112E848E
:1025800081CF97000000E78020E913450420056112
:102590001703FFFF6700E3B693F70510A9CF974431
:1025A000FF1F9384E491DC4897000000E78020C17E
:1025B0001747FF1F13074782184383C78401034748
:1025C00087036318F700DC4489C797000000E780A1
:1025D00080DF85471747FF1F232EF78EB7E70400DC
:1025E000BC4B930500021745FF1F0345E58D8297FD
:1025F0001345041069BF93F70508BDC79747FF1F30
:1026000083C7178EE91719469745FF1F9385658D78
:102610001305D10093F4F70F1749FF1F0349498CA5
:1026200097C00000E780404093970401C18317479B
:10263000FF1F1307678B231DF100231CF100974731
:10264000FF1F9387E7873ACE3ACAD8432306010093
:1026500009CBDC439315890154080D46E1856800D8
:1026600082971345040825B793F72500A5C397471C
:10267000FF1F9387E784D84B89476306F702974784
:10268000FF1F83C7278113F7270011EF918B99CF85
:10269000B7E70400BC4F1306000A89451745FF1F22
:1026A00003458582829713452400D5B59737FF1FD0
:1026B000938787729C4383C787031747FF1F230DA8
:1026C000F78097000000E78060DBF1BF93F7050219
:1026D00081CB97000000E78060DA1345040245BD16
:1026E00093F7850081CB97000000E780E0D2134587
:1026F000840071BD93F7150081CB97000000E7803F
:10270000A0B41345140061B593F7450081CB970041
:102710000000E78060B31345440095BD93F70504BE
:1027200095C39737FF1F83C7A77991CB9700000008
:10273000E780A0A491471737FF1F232DF778134593
:102740000404B1B593F705010145E38207E4973727
:10275000FF1F9387E776D84B91476310F7049737AD
:10276000FF1F938727739C4313D727008583D98F37
:10277000858B91E7B7E7040083A7071D8297B7E72A
:102780000400FC4F91451735FF1F0345E573829701
:1027900085471737FF1F232FF77213450401C5BB69
:1027A0009747FF1F238EA78282801703FFFFE70250
:1027B00003939737FF1F23AB07709737FF1F23A99A
:1027C000077085471734FF1F130404611737FF1F75
:1027D0002322F7701C4083C787031737FF1F230D81
:1027E000F76E9790FFFFE780A08F29C59717FF1F0F
:1027F00023A2A7D41C40170500001305A5D783C743
:1028000087031737FF1F2309F76C1717FF1FA30F45
:10281000F7D09737FF1FA385076AB7E7040083A7A0
:10282000070882979737FF1F2380A76A1703FFFFC8
:102830006700238DB7C7898E938767ED1717FF1F32
:10284000232AF7CE45BF1737FF1F03476767795520
:1028500055E79737FF1F9387A76603C7170005073C
:102860009736FF1FA38EE66403C717008D463377A4
:10287000D7029736FF1FA385E66483C61700173774
:10288000FF1F13076755184393F6F60FA9EE83470A
:1028900087031737FF1F2301F76485471737FF1F8B
:1028A0002300F7629737FF1F9387C75E9C4301455C
:1028B000998BA9E71703FFFFE702638237E404005F
:1028C0007C48C1451735FF1F0345056082973C488A
:1028D00085451735FF1F0345255F8297014517037F
:1028E000FFFF6700038283C7170085466395F600E4
:1028F0008347970379BF8347A70361BF82809737D8
:10290000FF1F83C7E75BA1CF17F3FEFFE702237D1D
:1029100037E404009737FF1F2384075A7C48854516
:102920001735FF1F0345455A82977C4C9145173553
:10293000FF1F0345655982977C4891451735FF1F56
:102940000345855882973C48C1451735FF1F03450D
:10295000A5578297014517F3FEFF6700837A7955E3
:10296000828017F3FEFFE70283772A84035565FF11
:102970009780FFFFE780A0179737FF1F9387475483
:10298000D847BE841DEF9790FFFFE78080779C4873
:10299000232004009DEB9737FF1F23AB8752973707
:1029A000FF1F23A58752B7E70400BC4B89451735A5
:1029B000FF1F034565518297014517F3FEFF67002E
:1029C0004374630A8700184375BF80C39737FF1F9E
:1029D00023A08750C9BF7955CDB717F3FEFFE70293
:1029E00003709737FF1F9387E75F8843232605000F
:1029F00023240500510597A00000E780C03317F39A
:102A0000FEFF6700037017F3FEFFE702436D173404
:102A1000FF1F1304245D1C40411199CF9C472302E2
:102A2000B5002AC61CC197000000E78040FB1C408F
:102A30009C4B99C332458297410117F3FEFF670013
:102A4000436C17F3FEFFE70283694111444D328561
:102A500032842EC69790FFFFE780C0522AC4228599
:102A60009790FFFFE780205403A84400630C080000
:102A7000B245835744001840224683D54500AA86B4
:102A800026850298410117F3FEFF6700836717F35D
:102A9000FEFFE702C364404D1DC808C09705000053
:102AA000938565031305440197A00000E780401655
:102AB0009737FF1F938707539C43014589E7973753
:102AC000FF1F23A1875217F3FEFF670083637D5525
:102AD000DDBF17F3FEFFE702836001116800930575
:102AE000F00F02C602C802CA02CC02CE9700000054
:102AF000E780A0F1056117F3FEFF67008360973759
:102B0000FF1F9387274E9C43D847A1679D076319F2
:102B1000F70217F3FEFFE702835C011132859790FD
:102B2000FFFFE7802046230AA10081456800970047
:102B30000000E78080ED056117F3FEFF6700635C2E
:102B400082809737FF1F9387E7499C43D847A16747
:102B5000938777036319F70217F3FEFFE702235801
:102B6000011132859790FFFFE780C041230AA10041
:102B70008145680097000000E78020E9056117F3B0
:102B8000FEFF6700035882809737FF1F93878745B2
:102B90009C43D84795476316F70417F3FEFFE702F7
:102BA00003540111328532849790FFFFE780803D06
:102BB000230AA10022859790FFFFE780C03E83573C
:102BC0004400231BA10081453ECC1C4068003ECE42
:102BD00097000000E78060E3056117F3FEFF6700E0
:102BE00043528280930785FF8DC38327C5FF91CF12
:102BF000DC4B81CF17F3FEFFE702634E032585FF11
